:020000040801F1
:1000000000800120B5BF04080000000000000000CF
:1000100069C1040869C1040869C10408000000003E
:100020000000000000000000000000009D02010828
:1000300069C104080000000085040108D904010812
:1000400069C1040869C1040869C1040869C10408D8
:1000500069C1040869C1040869C1040869C10408C8
:1000600069C10408C5490408ADE5030869C104086D
:100070003146040869C10408A96E040869C104086E
:1000800069C1040869C1040869C1040869C1040898
:100090002D7C040869C1040869C10408FDE5030852
:1000A000DDEE030869C1040869C1040869C10408D8
:1000B00069C1040869C10408552F020869C1040810
:1000C00069C1040869C1040869C1040869C1040858
:1000D00069C10408792E0408C9340408C53A040823
:1000E00069C1040869C1040869C1040869C1040838
:1000F00069C1040869C1040869C1040869C1040828
:1001000069C1040861F4040869C1040869C10408EC
:1001100069C10408B140040869C1040869C1040840
:1001200069C1040869C1040869C1040869C10408F7
:1001300000000000000000000000000000000000BF
:1001400000000000000000000000000000000000AF
:10015000000000000000000000000000000000009F
:10016000000000000000000000000000000000008F
:10017000000000000000000000000000000000007F
:10018000000000000000000000000000000000006F
:10019000000000000000000000000000000000005F
:1001A000000000000000000000000000000000004F
:1001B000000000000000000000000000000000003F
:1001C000000000000000000000000000000000002F
:1001D0000000000000000000000000005FF8E0F1F7
:1001E000DFF854040068006880F308880B4B196836
:1001F000086801F10401DFF84424B1E8F00FA2E837
:10020000F00FB0E8F80F83F3148880F309884FF0FB
:10021000000080F31188DFF828E470470400002014
:1002200030B44FF0807500E922000446012B14BF62
:1002300003230223002140F80C1C40F8202C44F832
:10024000443D204630BC704708B5836913F8020C62
:10025000012811D004D3022816D00F4B984708BDAF
:100260004EF61C53CEF200031A6842F07F421A6029
:10027000BDE80840FFF7B4BF4EF60453CEF20003CA
:100280004FF080521A6008BDEFF3148121F0010194
:1002900081F3148808BD00BFC17104081EF0040F6B
:1002A0000CBFEFF30880EFF30980FFF7CDBF00200C
:1002B000FFF7CABF4EF62053CEF20003196830B4E0
:1002C00041F47F01196019684EF6905241F07F4168
:1002D000CEF2000219601368B3F5006F15D04EF22C
:1002E000140241F63F11CEF20002C0F201014EF2BB
:1002F00010031160CEF2000307221A605A4B00224D
:100300001A6000DF002030BC7047584958484EF64C
:100310009C53401A41F01002CEF2000320281A60CC
:1003200040F29A804023052203E001321F2A00F0A8
:10033000838098424FEA4303F7D8012302FA03F27D
:10034000C0F2076313434B4D41F011044EF6A05029
:100350004EF69C52691ACEF20000CEF2000220291D
:100360000360146074D94023052202E001321F2A81
:1003700066D099424FEA4303F8D8012302FA03F208
:10038000C0F2075313433C493C4D41F012044EF672
:10039000A0504EF69C52691ACEF20000CEF2000236
:1003A0002029036014605BD94023052202E001325A
:1003B0001F2A49D099424FEA4303F8D8540044F029
:1003C000837444F001144EF6A0524EF69C53132051
:1003D000CEF20002CEF20003C4F200004FF6FE712E
:1003E0001460C1F6FF7118604022052301E08A42C3
:1003F0001CD8013352001F2BF9D13F21C1F200312B
:100400004EF6A053CEF200034EF624521960CEF2FF
:10041000000211684EF6945341F480311160CEF21F
:1004200000031A6842F005021A6058E7590041F0CB
:10043000985141F00101E3E73F23C0F2076382E7EF
:100440003F23C0F207539EE73F24C0F20714BAE7E8
:100450000923C0F2075396E70923C0F2076372E746
:100460000924C0F20714AEE7880C00200000010840
:1004700000001008004001080000002000020020D9
:10048000704700BFEFF30980124B1A68EFF3148135
:1004900020E9F20F10602DE908404FF0BF0080F313
:1004A000118801F07DFA4FF0000080F31188BDE85B
:1004B00008401968086801F10401604AB1E8F00FCA
:1004C000A2E8F00FB0E8F80F83F3148880F30988EE
:1004D000704700BF0400002008B54FF0BF0080F354
:1004E000118841F29563C0F6010398474FF0000070
:1004F00080F3118808BD00BF30B4002945D0002B1F
:1005000027D105254C68ECB10B6845F01002134368
:10051000202C83607AD94023052202E001321F2A71
:1005200015D09C424FEA4303F8D852008B6843F041
:1005300001031343C36001350C310830082DE1D1AC
:1005400030BC704745F010038360C460F3E73E227F
:10055000ECE79B0042F01402202B026058D94022A5
:10056000052402E001341F2C0BD093424FEA4202D3
:10057000F8D8012304FA03F4C0F20733234343609D
:10058000BFE73F23C0F20733F9E7274B274943F082
:100590001402C91A2029026042D94023052202E030
:1005A00001321F2A2AD099424FEA4303F8D8012387
:1005B00002FA03F2C0F2073313431D4A1D4942F009
:1005C0001504891A20294360846025D94023052217
:1005D00002E001321F2A15D08B424FEA4303F8D3C1
:1005E000520042F0837242F00112C26016220023D0
:1005F0000261172243618261C361A1E73F23C0F218
:100600000733DAE73F22C0F20712EEE708228DE750
:100610000923C0F20733B2E70922C0F20712E4E768
:100620000923C0F20733C8E7000000200080012042
:10063000000000200002002008ED00E09CED00E03A
:10064000FDFFFFFF2DE9F84306460F4638B34C2067
:10065000174DA847044610B306FB07F808F1010040
:10066000A84705462060E8B1721E07FB020200EBB6
:1006700008014FF0FF336160002104F11000DFF842
:100680003890A163E2606364A364A560E6632764B5
:10069000C84704F12400C8472046BDE8F88300207D
:1006A000BDE8F8832046034B98472846BDE8F88309
:1006B000611C0108A51C0108717704082DE9F04FA1
:1006C000824687B0A14F039202930191B847DAF8AE
:1006D0003820DAF83C3000259A42DFF88482DFF8CF
:1006E00084B29B4CC0F09780039E002E00F01B81CB
:1006F000002D00F0088104ADC047D847B847DAF8AC
:100700004430013300F00B81DAF84830013300F057
:100710000281C04741F6F523284603A9C0F601032C
:100720009847002840F00481B847DAF83860DAF8D2
:100730003C5047F2F913C0F604039847AE4240F02C
:100740008C800AF1100528460399824B984747F29E
:10075000C513C0F604039847DAF84830002B1DDDB6
:10076000DAF82430D3B10AF12406DFF8EC9109E07D
:10077000DAF84830013B002BCAF848300EDDDAF8D1
:1007800024305BB13046A0470028F1D0C847DAF8E2
:100790004830013B002BCAF84830F0DC4FF0FF3303
:1007A000CAF84830C047B847DAF84430002B1ADDA1
:1007B000DAF81030BBB1684E09E0DAF84430013B9A
:1007C000002BCAF844300EDDDAF810305BB1284651
:1007D000A0470028F1D0B047DAF84430013B002BA5
:1007E000CAF84430F0DC4FF0FF33CAF84430C04759
:1007F0005A4B984730B94EF60453CEF200034FF0EF
:1008000080521A600125B847DAF83820DAF83C300F
:100810009A42BFF469AFDAF84020002A40F0EB803A
:10082000DAF80040002C00F01581DAF83830013396
:10083000CAF83830DAF8243063B1454B0AF12400A5
:100840009847012801BF4EF60453CEF200034FF043
:1008500080521A60C047012067E047F2C513C0F616
:1008600004039847DAF84830002B1CDDDAF824300E
:10087000CBB10AF12406384D09E0DAF84830013BE3
:10088000002BCAF848300EDDDAF824305BB1304670
:10089000A0470028F1D0A847DAF84830013B002BE8
:1008A000CAF84830F0DC4FF0FF33CAF84830C04790
:1008B000B847DAF84430002B1CDDDAF81030CBB141
:1008C0000AF11005244E09E0DAF84430013B002B10
:1008D000CAF844300EDDDAF810305BB12846A04784
:1008E0000028F1D0B047DAF84430013B002BCAF8B9
:1008F0004430F0DC4FF0FF33CAF84430C047174BA8
:10090000984701257FE704AD41F6DD232846C0F670
:1009100001039847F0E60023CAF84830F9E60023BF
:10092000CAF84430F0E6C047304607B0BDE8F08F63
:10093000B847DAF84830002B2CDDDAF824304BB316
:100940000AF12405024C044E18E000BFC5710408EA
:10095000711A0108011A0108611B0108AD1701088D
:10096000F97104082D160108DAF84830013B002B14
:10097000CAF848300EDDDAF824305BB12846A047CB
:100980000028F1D0B047DAF84830013B002BCAF814
:100990004830F0DC4FF0FF33CAF84830C047B84762
:1009A000DAF84430002B1DDDDAF81030D3B12D4CCD
:1009B0000AF110052C4E09E0DAF84430013B002B17
:1009C000CAF844300EDDDAF810305BB12846A04793
:1009D0000028F1D0B047DAF84430013B002BCAF8C8
:1009E0004430F0DC4FF0FF33CAF84430C0471F4BAF
:1009F0009847002099E7029BABB901991C4BDAF8A4
:100A000008009847DAF80810DAF84030DAF80420DD
:100A1000CB189342CAF80830FFF407AFDAF8003079
:100A2000CAF8083001E70199114BDAF80C00984731
:100A3000DAF84030DAF80C205B42DAF80010D2180D
:100A40008A42CAF80C203EBFDAF80420D318CAF84C
:100A50000C30EAE6DAF80400064B9847CAF804407E
:100A6000E3E600BF711A0108611B0108AD17010818
:100A7000755F01080D1C010838B50A4B456804462E
:100A80009847854201D0002038BDE1680139E16016
:100A900009B1012038BD20460A460B46FFF70EFE7D
:100AA000012038BD951B010870B54C200F4B9847AD
:100AB0000446C8B100254FF0FF330122E2636364AE
:100AC000A36400F110000A4E65602560A560E56032
:100AD000A5632564B04704F12400B04720462946A9
:100AE0002A462B46FFF7EAFD204670BD611C01082F
:100AF0007177040870B5044616464FF0BF0080F3C6
:100B00001188A56BE06B854206D300234FF00000EF
:100B100080F31188184670BD226C62B92568002DDB
:100B200032D0A26BA36C0132A2635A1C11D00133E4
:100B3000A3640123EAE7C3B9164BA0689847A168EC
:100B4000236C6268CB189342A360EAD32368A36046
:100B5000E7E7636A002BECD004F124000E4B9847C2
:100B60000028E6D001233360D0E70A4BE0689847BD
:100B7000226CE368524221689B188B42E3603EBFBF
:100B800063689B18E360CCE76068044B9847656036
:100B9000C7E700BF755F0108711A01080D1C010845
:100BA0002DE9F04F814687B0A74E0193A74F0291E0
:100BB0000392B047D9F838300025DFF8A8A2B8462C
:100BC000A34C002B40F091800398002800F0368160
:100BD000002D00F0C08004ADB847D047B047D9F829
:100BE0004430013300F01B81D9F84830013300F064
:100BF0001281B84741F6F523284603A9C0F6010340
:100C00009847002840F03281B047D9F83850C047A3
:100C1000002D40F0A880D9F80030002B00F00381AF
:100C200009F124058B4B284603999847B047D9F81A
:100C30004830002B1BDDD9F82430C3B1DFF828B2CF
:100C400009E0D9F84830013B002BC9F848300EDDE7
:100C5000D9F824305BB12846A0470028F1D0D84706
:100C6000D9F84830013B002BC9F84830F0DC4FF090
:100C7000FF33C9F84830B847B047D9F84430002BA3
:100C80001DDDD9F81030D3B109F11005DFF8D8B166
:100C900009E0D9F84430013B002BC9F844300EDD9F
:100CA000D9F810305BB12846A0470028F1D0D847CA
:100CB000D9F84430013B002BC9F84430F0DC4FF048
:100CC000FF33C9F84430B847634B984730B94EF604
:100CD0000453CEF200034FF080521A600125B04752
:100CE000D9F83830002B3FF46FAFD9F80030D9F87D
:100CF0000C4073B1D9F84020D9F80400A118814202
:100D0000C9F80C10029824BFC9F80C301946534B8F
:100D10009847019B002B40F0FE80D9F83820D9F885
:100D20000030013AC9F83820002B00F00481D9F8CE
:100D30001030002B00F0F48009F11000444B98476C
:100D4000012840F0ED804EF60453CEF200034FF040
:100D500080521A60E4E004AD41F6DD232846C0F677
:100D60000103984738E747F2C513C0F604039847D4
:100D7000D9F84830002B1DDDD9F82430D3B109F162
:100D80002405DFF8E4B009E0D9F84830013B002B36
:100D9000C9F848300EDDD9F824305BB12846A047A9
:100DA0000028F1D0D847D9F84830013B002BC9F8CA
:100DB0004830F0DC4FF0FF33C9F84830B847B0474F
:100DC000D9F84430002B1DDDD9F81030D3B109F12A
:100DD0001005DFF894B009E0D9F84430013B002B4E
:100DE000C9F844300EDDD9F810305BB12846A04771
:100DF0000028F1D0D847D9F84430013B002BC9F87E
:100E00004430F0DC4FF0FF33C9F84430B847124BA0
:100E10009847012563E70023C9F84830E9E6002335
:100E2000C9F84430E0E647F2C513C0F6040398471A
:100E3000D9F804000A4B9847C047F1E60090B8473C
:100E4000009807B0BDE8F08FC5710408F971040877
:100E5000711A0108011A0108AD170108755F010830
:100E6000A11B01082D160108611B0108B047D9F824
:100E70004830002B1EDDD9F82430DBB1304C09F1AD
:100E80002405DFF8C08009E0D9F84830013B002B89
:100E9000C9F848300EDDD9F824305BB12846A047A8
:100EA0000028F1D0C047D9F84830013B002BC9F8E1
:100EB0004830F0DC4FF0FF33C9F84830B847B0474E
:100EC000D9F84430002B1DDDD9F81030D3B109F129
:100ED00010051B4C1B4E09E0D9F84430013B002B98
:100EE000C9F844300EDDD9F810305BB12846A04770
:100EF0000028F1D0B047D9F84430013B002BC9F8A5
:100F00004430F0DC4FF0FF33C9F84430B8470E4BA3
:100F10009847002095E7D9F82430C9F80C4013B958
:100F2000B84701208DE709F12400054B98470028B8
:100F30007FF409AFF4E7054B9847C9F80400F6E6DB
:100F4000711A0108611B0108AD170108951B010802
:100F500070B50C4B456804460E46984785420CD048
:100F60000021204632460B46FFF71AFE012800D02A
:100F700070BDE3680133E36070BDE36801201B18B6
:100F8000E36070BD951B010870B5044616464FF02E
:100F9000BF0080F31188A36B2BB94FF0000080F3E2
:100FA0001188184670BD206860B1E368226C6568DE
:100FB0009B18AB42E36024BF0346E0600846194635
:100FC0000B4B9847A26B636C013A591CA26303D088
:100FD000013363640123E0E72369002BFAD004F1B5
:100FE0001000044B98470028F4D001233360D4E765
:100FF000755F0108711A010847F2C51310B5C0F6F4
:10100000040304469847A46B47F2F913C0F604039F
:101010009847204610BD00BF806B704738B541F639
:10102000A5440546C0F601040068A0472846A0472D
:1010300038BD00BF806BD0F1010038BF0020704781
:10104000826BC06BB2EB000CDCF1000050EB0C00CB
:10105000704700BF2DE9F04F814683B0684F68208C
:101060008B4616469A460E9DB8470446002800F067
:10107000C380002D00F0B3800565B200A52128468D
:10108000604B9847236D06F1FF3C03EB8C030C9DEE
:101090005946102223F0070704F154005A4B984791
:1010A00025F0004B594B0022BBF1040F34BF5D46C5
:1010B000042504F1240884F86320E564656640464D
:1010C00001939847C5F1050504F13800019B984745
:1010D0003346A563201D0F99226D4D4D2463646432
:1010E000A8470C9D3846EB0F49464A4D5246A84743
:1010F0000D9D206005B12C60474D484B98472B68EB
:1011000001332B606B68002B3ED0D5F8D8308BB301
:1011100005F10806E36CD5F8DC20D5F8E41093421D
:1011200088BF3D4A03EB830088BFC2F8DC30D5F8A6
:10113000E02006EB800001328B42C5F8E02088BF3A
:10114000354A414688BFC2F8E430354B9847354BA5
:101150009847D5F8D8309BB12F4B5B68DB6C9B452B
:101160000ED94EF60453CEF200034FF080521A60AF
:10117000012006E06B68DB6C9B4528BF6C60C7E70D
:10118000012003B0BDE8F08F6C602B6805F1080604
:10119000012BBFD1244F3046B84705F11C00B8479A
:1011A00005F13000B84705F14400B84705F16C0A75
:1011B00005F15800B84705F180095046B847484640
:1011C000B84705F19400B84705F1A800B84705F104
:1011D000BC00B847C5F8D0A0C5F8D4909AE7B200D3
:1011E00010460192B847019A0546206500287FF411
:1011F00045AF20460D4B98474FF0FF30C1E700BF89
:10120000611C010809600108696301088977040805
:10121000F90401082102010800000020C57104083A
:1012200091770408F971040871770408A51C010876
:101230002DE9F0411A4C1B4B0546984763689D42C7
:101240002BD02E464DB306F124073846DFF86480D4
:10125000C047B36C13B106F13800C0471248394695
:10126000124B9847D4F8E030D4F8E820013301322B
:10127000C4F8E0300E4BC4F8E8209847D4F8D830D2
:1012800003B10DB1BDE8F0814EF60453CEF2000378
:101290004FF080521A60BDE8F08166680025D2E701
:1012A00000000020C5710408A80000209177040800
:1012B000F9710408E577040810B5064B0446984711
:1012C00024B1E46C044B9847204610BD034B5C6886
:1012D000F7E700BFC5710408F97104080000002099
:1012E0002DE9F041274B0546042934BF0E4604265C
:1012F0009847254B5A68954240D02C46002D3DD04A
:10130000636EB3421ED021D3D5F1010538BF00254D
:10131000E26C1D4F934207F1080803EB8303626BF5
:1013200008EB830308BFE664C6F105019A426666CE
:10133000A1630FD035B14EF60453CEF200034FF047
:1013400080521A60114B9847BDE8F081003518BFF4
:101350000125DDE704F1240630460D4B9847E36C88
:10136000D7F8E42003EB8300934288BFC7F8E4304A
:1013700008EB80003146074B9847DBE75C680025A7
:10138000BEE700BFC571040800000020F971040821
:10139000E5770408917704082DE9F041344D354B89
:1013A000044698476B689C4254D02646002C51D086
:1013B00006F124073846DFF8CC80C047B36C13B180
:1013C00006F13800C0472A4E2B4B394606F1BC00C7
:1013D00098472A4B98470CB1BDE8F081D6F8D83031
:1013E0007BBBD6F8BC2033689A4239D0D6F8EC30B3
:1013F000002B38D1D6F8E43003EB830306EB8306E9
:10140000B3686BB9D5F8E430013BC5F8E430D5F8E2
:10141000E43003EB830305EB83039B68002BF1D0DF
:10142000D5F8E420164B02EB820203EB82025368EC
:1014300002F108015B688B4253600ED0DB686B6081
:10144000CAE74EF60453CEF200034FF080521A6002
:10145000BDE8F0816E680024AAE75B685360EDE7A1
:101460007460BDE8F0810123C6F8F030BDE8F0817A
:1014700000000020C571040891770408F971040880
:1014800008000020E5770408436B074A934201D027
:1014900000207047806C283B9842F9D0D0F10100C1
:1014A00038BF0020704700BFBC00002070B5044664
:1014B00060B11B4D6B68984208D01A4B9847636B1C
:1014C00005F1BC02934202D0174B984770BDA36C44
:1014D00005F194029342F7D0002BF5D104F12406D4
:1014E0003046124B9847D5F8E420E36C10489342FD
:1014F00088BFC5F8E43003EB830300EB830031467B
:101500000C4B98476B68E26CDB6C9A4221BF4EF63D
:101510000453CEF200034FF080521A60D4E700BFAC
:1015200000000020C5710408F9710408E57704087B
:101530000800002091770408F8B51B4C436B04F1B8
:10154000BC029342054602D000263046F8BD866CA8
:1015500004F194008642F7D0002EF5D1D4F8EC3097
:10156000E3B96268EB6CD66C05F12407B3423846E8
:101570000E4B34BF002601269847EB6CD4F8E420CC
:101580000B48934288BFC4F8E43003EB830300EBBD
:1015900083003946074B98473046F8BD05F13801BE
:1015A000044B98473046F8BD00000020E57704085A
:1015B000080000209177040810B54FF00043002484
:1015C00084B08DE8180080222346029403940A48D0
:1015D0000A49FFF73FFD0128034601D004B010BDC2
:1015E0004FF0BF0080F31188054AC2F8D830054B90
:1015F000C2F8F4409847F1E7F176040898810508AD
:1016000000000020B502010808B54FF0BF0080F3CC
:10161000118840F2000240F28143C2F20002002130
:10162000C0F60103C2F8D810984708BD40F2000385
:10163000C2F20003D3F8EC200132C3F8EC2070476B
:1016400047F2C51310B5C0F60403984740F20002F4
:10165000C2F20002D2F8F44047F2F913C0F60403D4
:101660009847204610BD00BF4FF0BF0080F311889F
:1016700040F20003C2F20003D3F8F4304FF0000050
:1016800080F311881846704740F20003C2F200034D
:10169000186870472DE9F84F404DD5F8EC30002B15
:1016A00069D1D5F8F4300133C5F8F430D5F8F43009
:1016B000002B4AD0D5F8F830D5F8F420374E9A42AE
:1016C0003CD3D6F8D0301B68002B33D0D6F8D030BE
:1016D000DB68DC68D6F8F420636A93425BD8304F4D
:1016E00006F10809DFF8C080BA4608E0D6F8D03025
:1016F000DB68DC68D6F8F420636A93424BD804F1C7
:10170000240B5846B847A36C04F1380003B1D04706
:10171000E36CD5F8E42003EB8300934209EB8000EF
:10172000594688BFC6F8E430C047D5F8D0301B68AA
:10173000002BDBD14FF0FF33C5F8F830D5F800317E
:101740000BB9184B9847BDE8F88FD5F8D030D5F8CD
:10175000D420C5F8D020C5F8D430D5F8FC300133FA
:10176000C5F8FC30D5F8D0301B6863B94FF0FF33B3
:10177000C5F8F830A0E7D5F800310133C5F80031DD
:10178000084B9847DAE7D5F8D030DB68DB685B6A4E
:10179000C5F8F83090E7C5F8F830CFE70000002032
:1017A000E577040811C00408917704082DE9F84F83
:1017B000324C334B9847D4F8EC30013BC4F8EC3052
:1017C000D4F8EC30002B46D12268002A43D0DFF851
:1017D000B890DFF8B8B09846274604F1080A1DE033
:1017E000D7F8A030DD6805F1380005F12406C847B8
:1017F0003046C847EB6CD7F8E42003EB83009342F4
:101800000AEB8000314688BFC7F8E430D8476368E8
:10181000EA6CDB6C9A4228BF4FF00108D4F8943090
:10182000164A002BDCD1D2F800316BB1D2F800316E
:1018300053B1FFF72FFFD4F80031013BC4F800315A
:10184000D4F80031002BF4D1B8F1010F09D0D4F84D
:10185000F030012B05D000240A4B98472046BDE804
:10186000F88F00224EF60453C4F8F020CEF20003A5
:101870004FF0805201241A60EEE700BF0000002004
:10188000C5710408F9710408E57704089177040824
:1018900038B538B94EF60453CEF200034FF08052FB
:1018A0001A6038BD154CD4F8EC300133C4F8EC3074
:1018B000D4F8F4506368451903F12400104B98479D
:1018C0006268D4F8F43055629D4210D3D4F8D00049
:1018D00061680C4B24319847D4F8F8309D4238BFEA
:1018E000C4F8F850FFF762FF0028D3D038BDD4F811
:1018F000D4006168034B24319847F3E700000020CF
:10190000E5770408AD77040838B5224C0368D4F8AD
:10191000EC20CD180132C4F8EC20D4F8F420934226
:101920000DD9AB420DD80560FFF740FF50BB4EF616
:101930000453CEF200034FF080521A6038BDAB4220
:1019400003D8D4F8F4309D42EDD96368056003F103
:101950002400114B98476268D4F8F43055629D42D8
:101960000C4C10D3D4F8D00061680C4B243198474C
:10197000D4F8F8309D4238BFC4F8F850FFF716FF8E
:101980000028D4D038BDD4F8D4006168034B24318A
:101990009847C9E700000020E5770408AD77040800
:1019A000154BD3F8EC202AB11EE0D3F8E420013A1D
:1019B000C3F8E420D3F8E42002EB820203EB8202B6
:1019C0009268002AF1D0D3F8E4100C4A01EB8101AF
:1019D00002EB81014A6801F10800526882424A60C4
:1019E00006D0D2685A6070470122C3F8F0207047D1
:1019F00052684A60F5E700BF0000002008000020A0
:101A000070B5174C0D466168164E3831B0476068A6
:101A1000154B243098476B1C1AD0D4F8F410626828
:101A2000D4F8F4306D189D4255620BD3D4F8D00031
:101A300061682431B047D4F8F8309D4238BFC4F80B
:101A4000F85070BDD4F8D40061682431B04770BD3F
:101A5000616804F1BC002431044B984770BD00BF9D
:101A600000000020AD770408E577040891770408AA
:101A7000F8B5C368154CDD68154F05F138063046DA
:101A8000B847D4F8EC30D3B905F124063046B8474E
:101A9000EB6CD4F8E4200F48934288BFC4F8E430DC
:101AA00003EB830300EB830031460B4B98476368DD
:101AB000E86CDB6C984234BF00200120F8BD04F1D3
:101AC00094003146044B9847F1E700BF0000002026
:101AD000E5770408080000209177040840F200032D
:101AE000C2F20003D3F8FC20D3F8F43080E80C00F5
:101AF000704700BF70B5174B0D46044698472B68DA
:101B00005A1C24D0144A2168D2F8FC00814208BF34
:101B1000616804D0D2F8F4006168814215D9D2F826
:101B2000F4000D4A401A83420FD9D2F8F460D2F87B
:101B3000FC009B1BD2F8F4205918296084E80500AA
:101B40000025064B9847284670BD0125F9E700257A
:101B5000F7E700BFC571040800000020F971040810
:101B600040F20003C2F200030122C3F8F0207047E4
:101B7000064B10B55A68904206D028B100220430B6
:101B80001346034CA04710BD5868F7E7000000203B
:101B9000F904010840F20003C2F2000358687047DC
:101BA000F8B5174CC36C62680546D26C934210D2EC
:101BB000626804F10806D16C03EB8303426B06EB09
:101BC0008303C1F105019A42816303D06368DB6C32
:101BD000C364F8BD00F1240738460A4B9847636890
:101BE000D4F8E420DB6C3946934203EB8300EB64CA
:101BF00088BFC4F8E43006EB8000034B9847F8BD7B
:101C000000000020E57704089177040838B5044601
:101C1000E0B1C26C436E9A4218D000F12405284608
:101C20000B4B98470B4A636ED2F8E410C3F10500E2
:101C30008B42A0630848E36488BFC2F8E43003EB3A
:101C4000830300EB83002946044B984738BD00BF4F
:101C5000E5770408000000200800002091770408C0
:101C6000430710B50B4B04461CBF20F00704083493
:101C70009847094A1368E418B4F5C04F08D2A34244
:101C800006D21460054CE418054B9847204610BD59
:101C90000024F9E72D160108A80E0020B00E002040
:101CA000AD170108704700BF40F6A863C2F20003F9
:101CB00000221A60704700BF40F6A863C2F200031A
:081CC0001868C0F5C040704730
:105CC8002DE9F0478AB004460D4600F04DF8DFF89C
:105CD80094A09AF90030013306460F460FD02046AB
:105CE800294600F007F950B14FF000084FF00009BD
:105CF8002046294642464B4604F066FA20B930460B
:105D080039460AB0BDE8F08701230093144B9AF88E
:105D18000060CDE9044501930023CDE902450893CD
:105D280056B9CDE90689684600F00CF970B1089BB0
:105D38008BB9DDE90667E2E74046494642464B46ED
:105D480004F0FAF8022ECDE90601ECD100F008F9CA
:105D580021230360EBE700F003F9089B0360E8E701
:105D680000830508080300202DE9F8430027B946F9
:105D7800C7F6F077C7F6F0790F404F4504460D4651
:105D880002460B460E46804600F09980002976DDD3
:105D98005FEA215C00F0818026F07F43ACF2FF3C93
:105DA80023F470031CF0010F43F480131CBF4FEA67
:105DB800D8724FEA48084FEA6C0C18BF02EB43034D
:105DC80000274FEAD872162402EB430338464FEAFD
:105DD80048024FF400114518D60F9D424FEA42027F
:105DE800DEBFC5EB030368187F184908013C06EBC2
:105DF8004303F0D12026A0464FF000410EE0814633
:105E08001B1A954288BF013B521B64184846D50FA0
:105E180049085200013E05EB430315D0984201EBB7
:105E2800080503DB954298BF8342F0D105F000498D
:105E380005EB0108B9F1004FE1D1B8F1000FA8BF97
:105E480000F10109DCDADAE7134310D166087B10A8
:105E5800FA0703F17F5348BF46F0004603F50013E5
:105E6800344603EB0C5520462946BDE8F883611CEF
:105E78001CBF04F001031C19E8D10137E7E721F042
:105E880000460643EFD049BB8C464FEAD826ACF112
:105E9800150C4FEA4858002EF7D016F4801319D184
:105EA80076000133F002FBD5C3F10101C3F12002F2
:105EB80028FA02F28C44164308FA03F86CE703F058
:105EC80011FF02460B462046294603F059FD0446B9
:105ED8000D46C8E7202201210023E9E702460B46C8
:105EE80003F04CFD02460B4604F026F804460D4626
:105EF800B9E700BF50EA010201D102207047D0F192
:105F0800010238BF0022B1F1004F08BF0028F4D0C9
:105F180021F000434FF6FF71A3F58010C7F6DF713B
:105F2800884201D804207047B3F5801F01D20320AE
:105F380070470020C7F6F070834214BF002002F0BB
:105F48000100704700207047002101F0FFBB00BF2F
:105F580000210A2201F0BCBC00220A2301F018BC6F
:105F680040F21033C2F20003186870470F2AF0B4E9
:105F780040D941EA00039B073ED10C46034615462B
:105F88002668103D1E6066685E60A6689E60E668CA
:105F98001034DE6010330F2DF2D8A2F1100502F094
:105FA8000F0425F00F051035032C00EB05032944D9
:105FB80024D9A4F1040C1D460C464FEA9C0C01EBB5
:105FC8008C07043754F8046BBC4245F8046BF9D1CC
:105FD8000CF1010402F00302A40009191B193AB1DB
:105FE80001399A1811F8014F03F8014B9342F9D17E
:105FF800F0BC70470346F2E70346F1E72246EEE7B6
:1060080070B48407034644D0541E002A3FD0CEB251
:1060180002E0002C3BD0144603F8016B13F0030F89
:106028001D4604F1FF32F4D1032C29D9CAB20F2C32
:1060380084BF2B46264642EA022242EA024211D98E
:10604800103E1A605A609A60DA6010330F2EF7D843
:10605800A4F1100304F00F0423F00F031033032CF2
:106068001D440DD92E462346043B46F8042B032B2A
:10607800FAD8231F04F0030423F003030433ED18B4
:106088002CB1C9B22C1905F8011BA542FBD170BC73
:10609800704705461446C7E740F210330022C2F2A3
:1060A80000031B68C3F8A800C3F8AC20704700BF02
:1060B80040F210330122C2F20003F0B44FF22D4730
:1060C8001E6847F62D74C5F65107C4F6954400239B
:1060D800D6F8A850D6F8AC1007FB05F704FB0177F3
:1060E800A5FB044512193D4443EB0503C6E92A23E1
:1060F80023F00040F0BC7047830770B5064614D102
:106108000368A3F1013222EA030313F0803F0CD1A4
:10611800031D1A4653F8044BA4F1013525EA04047B
:1061280014F0803FF5D0104600E0304603782BB1DC
:10613800431C184601330478002CFAD100F082F889
:10614800304670BDC9B2F0B400294BD083070FD0D8
:106158000378002B73D0994242D0431C05E013F812
:10616800012B002A3BD091423AD09A071846F6D123
:10617800036841EA0127A3F1013247EA074722EA07
:10618800030212F0803F1CD17B40A3F1013222EAC6
:10619800030313F0803F14D1021D02E014F0803F86
:1061A8000FD1104652F8043BA3F1013687EA0304E5
:1061B80026EA0303A4F1013513F0803F25EA04041D
:1061C800ECD00378002B3AD0994209D0431C01E067
:1061D800914205D0184613F8012B002AF8D1104631
:1061E800F0BC704781070DD00378002BF8D0431C12
:1061F80002E00278002AF3D013F0030F184603F1E7
:106208000103F6D10368A3F1013222EA030313F074
:10621800803F0AD1021D104652F8041BA1F1013437
:1062280024EA010111F0803FF5D00378002BD7D084
:10623800431C184601330278002AFAD1D0E71846E1
:10624800CEE700BF80EA0102844612F0030F4FD167
:1062580011F0030F32D14DF8044D11F0040F51F82D
:10626800043B0BD0A3F101329A4312F0803F04BFE4
:106278004CF8043B51F8043B16D100BF51F8044BCD
:10628800A3F101329A4312F0803FA4F101320BD1FD
:106298004CF8043BA24312F0803F04BF51F8043B82
:1062A8004CF8044BEAD023460CF8013B13F0FF0FDF
:1062B8004FEA3323F8D15DF8044B704711F0010F12
:1062C80006D011F8012B0CF8012B002A08BF7047E3
:1062D80011F0020FBFD031F8022B12F0FF0F16BFDA
:1062E8002CF8022B8CF8002012F47F4FB3D17047A2
:1062F80011F8012B0CF8012B002AF9D1704700BFC7
:1063080020F0030110F00300C0F1000051F8043B35
:1063180000F1040C4FEACC0C6FF000021CBF22FA0B
:106328000CF213434FF0010C4CEA0C2C4CEA0C4CC9
:10633800A3EB0C0222EA030212EACC1204BF51F8C2
:10634800043B0430F4D013F0FF0F1FBF013013F4E7
:106358007F4F013013F47F0F18BF0130704700BF23
:1063680041EA000313F0030F034670B425D0AAB125
:106378000C78013A03F8014B4CB11C4672B111F884
:10638800015F013A04F8015B2346002DF6D12AB1DA
:106398009A18002103F8011B9342FBD170BC704787
:1063A8000E4651F8044BA4F1013525EA040515F011
:1063B800803F05D1043A43F8044B032AF0D8D6E7C6
:1063C8003146D4E72DE9F00701273C4600254FF078
:1063D800FF36631900EB060C8B420DD21CF804C083
:1063E80010F80380E0452ED201241D469F1B631937
:1063F8008B4200EB060CF1D34FF0010A00255446FE
:106408004FF0FF3C1760631900EB0C0899420ED956
:1064180018F8048010F80390C1451AD901241D46C4
:10642800CCEB030A6319994200EB0C08F0D80CF185
:1064380001000136B0423CBFBA463046C2F800A05F
:10644800BDE8F00770470BD001272E463C46ED19F2
:10645800BFE709D04FF0010AAC4654465544D2E78D
:10646800BC4205D00134B4E7544505D00134CAE72D
:1064780027461D460124ACE7A2461D460124C2E773
:106488002DE9F04FADF2244D164680460D461046D4
:10649800194607AA1C46FFF795FF07AB0DF21C42E9
:1064A800039043F8044F9342FBD1671E002308A8CA
:1064B80034B1F25CF91A0133A34240F82210F8D142
:1064C80007993046039A711801F0A6FE00287FD17B
:1064D800DDF80CC02A468246671E0CF1FF3CCDF859
:1064E80008C0B444CDF814C0DDF80CC005460194CA
:1064F800CCF1010CCDF810C009E02DB1079A9342F8
:106508003CBF0199C2EB01039A4400252246019B36
:1065180008EB020000210AEB0304A21A01F032FE84
:1065280000284FD1002C4DD008EB040308A913F81C
:10653800013C51F82330002BDFD1039A954228BF44
:106548002A46BA4211D208EB0A0316F802C0B1185B
:10655800985C844506D02FE011F8010F13F802C0AB
:10656800844529D10132BA42F6D3039B02989D4251
:1065780028BF184618D2DDF808C008EB0A0316F839
:106588000C1013F80C20914240F08680059A06EB17
:10659800050B06E013F801C012F8019DE14503D18F
:1065A8000846411E5A45F5D10135854276D8079DE2
:1065B800019BAA445D1BA9E7DDF810C00025E24451
:1065C8009244A3E7002009B00DF5806DBDE8F08F77
:1065D800DDF80CC02A46DDF80CA04FF0000BCCEB20
:1065E80004030DF12009634538BF6346671E013374
:1065F800254607930CF1FF330193B444039BCDF870
:1066080008C0C3F1010304930BEB050408EB020077
:106618000021A21A01F0B6FD0028D3D1002CD1D058
:1066280008EB040313F8013C59F8233063BBBA455F
:1066380008EB0B0015D2DDF808C010F80A309CF8FA
:1066480000209A4218BF534621D1029A534605E0CA
:1066580012F8011F10F803C08C4518D10133BB4252
:10666800F6D3019B5A1CAED0DDF804C016F80C1006
:1066780010F80C20914206D113F1FF33A3D3F15C3B
:10668800C25C9142F8D0079B9B442246BCE7DDF8E8
:1066980010C0E3449B44F8E7039885E708EB0A0039
:1066A80091E700BF2DE9F04F8046037887B00E468A
:1066B800002B00F0F7800A789AB18446013101274F
:1066C80002E011F8012B5AB1934214BF002707F0DA
:1066D80001071CF8013F0D46002BF2D12B7803BBB4
:1066E8001FB1404607B0BDE8F08F08F101003178CE
:1066F800FFF728FDAD1B012D18BF0028074608BF6E
:106708008046EED0A844404594BFC0EB080401245D
:106718001F2D09D9214632462B46FFF7B1FE804688
:10672800DFE74FF00008DCE7294605AA3046FFF707
:1067380049FE0599711801903046019A01F06CFDE7
:10674800002852D1019B83468046013B0093F318F1
:106758000393019BC3F101030293224608EB05044E
:10676800B8180021A21A01F00DFD0028D9D1002C7B
:10677800D7D0019B9B4528BF5B469D4213D9F9188A
:10678800F05CF21811F80810884240F0858007EB99
:10679800080C05E012F8011F1CF8030088427BD1A1
:1067A80001339D42F6D89DE80A005B457DD907EB89
:1067B8000809725C19F801309A4276D1039B06EBFE
:1067C8000B0A06E019F8020013F801CD844503D13D
:1067D80011464A1E5345F5D10BF1010B8B4566D87E
:1067E800059B9844C3EB050BB7E701984FF0000BE6
:1067F80022462B1A06EB000900F1FF388246834235
:1068080038BF03463918013300910593C0F10103DD
:1068180002930BEB0504B8180021A21A01F0B2FC90
:1068280000287FF47EAF002C3FF47BAF554598BF1E
:1068380007EB0B0014D9009899F8002010F80B30DA
:106848009A4224D14A46534607EB0B0005E012F85A
:10685800011F10F803C08C451AD101339D42F6D8A8
:10686800B8F1FF3F43463FF45AAF16F8081010F846
:106878000820914207D113F1FF33FFF450AFF15CC8
:10688800C25C9142F7D0059B9B442246C1E7534620
:10689800029A93449B44F8E702994FF0000B88440E
:1068A80098445AE70D46012718E7019994E7B84438
:1068B80017E700BF000000002DE9F04F9DB08946A2
:1068C800834610924A4600200021CDF85C90CDE91D
:1068D8000801114612F8013B2D2B40D8DFE803F0E0
:1068E8003A3F3F3F3F3F3F3F3F38383838383F3FD8
:1068F8003F3F3F3F3F3F3F3F3F3F3F3F3F3F3F3FA0
:10690800383F3F3F3F3F3F3F3F3F3F353F1701261F
:10691800129601F10108CDF85C804B78002B21D14B
:106928009A4604930026CDF85C901296109D0DB1FE
:10693800179B2B60129E1EB1049F07F10047049716
:10694800504604991DB0BDE8F08F00271297E0E784
:106958001792BEE74FF0000ACDF810A0E2E788468C
:1069680000251295302B00F0D980002604960026C9
:106978002F2B1D4640F3E584392B00F3E28408F100
:1069880001023746344601E0392B17DC0F2C0DDCA9
:1069980007EB870006EB8601082C03EB400003EBAE
:1069A8004103D4BFA0F13007A3F1300617929246F5
:1069B80012F8013B01342F2B1D46E5DC584601F047
:1069C800CFFB01685846039101F0CAFB0068FFF746
:1069D80097FC03990246504602F0B2F98246002815
:1069E80000F0B480002107940A46084625F02003E9
:1069F800452B0BD1079D45EA0103049D1D4340F03B
:106A0800CD80099EDDF820A004968BE74FF0000C9E
:106A1800079B002B3FD007993846C2EB0C09079D0E
:106A2800002C08BF0C4603F0E7F8102DA8BF10256E
:106A3800092D02460B46CDE9082313DDA04B03EBD5
:106A4800C50353E9122303F04DF9CDE9040130469B
:106A580003F0D2F802460B46DDE9040102F090FF8C
:106A6800CDE90801079E0F2E00F3F380B9F1000F5E
:106A78004FD040F38485B9F1160F00F3388590495B
:106A8800DDE9082301EBC909D9E9000103F02AF976
:106A9800824604914AE7049E0E433AD1002840F00A
:106AA8009882493D252D00F2F782DFE815F0FA02B9
:106AB800F502F502F502F5028102F502F502F5028A
:106AC800F502F502F502F502F502F502F502F50206
:106AD800F502F502F502F502F502F502F502F502F6
:106AE800F502F502F502F502F502F502F502FA02E1
:106AF800F502F502F502F5028102531C179353784B
:106B0800282B00F0F685002208921346CFF6F8737A
:106B18000993099FDDF820A0049707E798F801304A
:106B2800582B00F0B883782B18BF08F1010200F049
:106B3800B2831146179212F8013B302BF9D08846E0
:106B4800002B00F02B820125049510E75846179D6D
:106B580001F006FB0068FFF7D3FB2B1817932D5C99
:106B6800002C40F0D881302D214605D101331793F0
:106B780001311D78302DF9D0A5F13103082B00F231
:106B88002D82303DDDF85C8040F0A1840A46404605
:106B980001210795431C17934578BFE1DDF85C9008
:106BA80009F10103179399F801502B2D00F0CE83BA
:106BB8002D2D00F0698200230A93A5F13003092BDB
:106BC80084BFCDF85C904FF0000C3FF621AF302D1C
:106BD80006D1179B0133179313F8015B302DFAD0B8
:106BE800A5F13103082B3FF611AF179BA5F1300C27
:106BF80003F1010ACDF85CA05D780B932F2D13DD0E
:106C0800392D11DC03F1020A534601E0392D0BDC62
:106C18000CEB8C0C17939A4605EB4C0C1D78013342
:106C2800ACF1300C2F2DF1DC0B9BC3EB0A0ABAF147
:106C3800080FC8BF44F61F6C04DC44F61F639C456C
:106C4800A8BF9C460A9B002B3FF4E2AECCF1000C97
:106C5800DEE6079E751B4D44002D40F30E8415F0AB
:106C68000F010AD01648DDE9082300EBC101D1E97C
:106C7800000103F037F8CDE9080135F00F0540F0C1
:106C8800B1810998DDF820A00B950490009758462B
:106C980041462246079B01F06FFBB9F1000F1190A6
:106CA800C0F2688400270D97119E29EAE977DDE98B
:106CB80008450C360E971396CDF828A076E000BF4D
:106CC800A07C05080F9B002B00F0018200270026FE
:106CD800C3F6F077AC460020CDF830A0C3F6F070CC
:106CE80008904FF0000A5346C7F6F07AC7F6E073EB
:106CF8000CEA0A0A9A4500F01C820B9DBAF1D46F7F
:106D08008CBF00230123002D08BF0023FBB10C9882
:106D1800A5A3D3E90023089903F060FA98B10C9869
:106D2800089903F0A1FA002800F0A88202F064FF95
:106D38000C9008910F9F002F40F08A82089D05F162
:106D480000430C9E1F4607F1D663CAEB03070A9857
:106D5800049901F091FD02460B463046394602F08F
:106D6800C1FF02460B460A98049902F009FE044640
:106D78000D468C460A9004910B9E3EB90023C7F637
:106D8800F0730CEA03039A4500F00A8258461899F2
:106D980001F09CFA5846414601F098FA584649468F
:106DA80001F094FA5846079901F090FA119E584656
:106DB80016AF716801F062FA336913999A1C920050
:106DC800804600F10C00FFF7D1F8049B009719A842
:106DD8000A9A0190584601F0C9FD012118905846B9
:106DE80001F064FB1699199B0029AABF0D9F0E9EFE
:106DF8007E180B9FB4BFC1EB060EDDF838E0C7EB79
:106E08000101B8BF0D9ECF1881466FF47F7087428D
:106E18000B98B4BF01F23343C3F1360306EB030A00
:106E280073441F18B245B4BF53463346BB42A8BF8C
:106E38003B460D99002BC2BFC3EB0A0AC3EB0707F9
:106E4800C3EB060691B10A465846494601F0D6FBFF
:106E5800189A81465846494601F032FB189903466C
:106E68005846039301F032FA039B1893BAF1000FC6
:106E780005DD58461899524601F00AFC18900E9AFA
:106E880022B14146584601F0B9FB8046002F05DD86
:106E9800414658463A4601F0FBFB8046002E05DD88
:106EA80049465846324601F0F3FB81461899424656
:106EB80058464FF0000A01F069FC4946C668C0F818
:106EC8000CA007900F9601F043FC5045C0F2418298
:106ED80000F091820798494601F0A2FD00224FF088
:106EE800804306460F4603F079F900287FF4EAAE9E
:106EF80000233946C3F6E0733046002202F0F2FE62
:106F08000F9F0C9001F10043089107B1089B0C9E5C
:106F1800AC461F46E5E6514652460794A5F13003B4
:106F28000120092B3FF662AD01F1010C1D461798AF
:106F38006146002B3FF42EAE012900F0D883079B51
:106F48000A9203F1010AC9181A4653460B94102AEB
:106F580008DC07EB870A06EB8604092BD4BF4FEA47
:106F68004A07660001338B42F1D10A9A63460B9CAB
:106F78000799102900F314838C44D218BCF1090F27
:106F8800D5BF07EB870706EB860605EB470705EB3A
:106F98004606079D0021ED180795FBE59A460493E0
:106FA800C4E400BFAFF300800000C0FFFFFFDF4173
:106FB800AF48179A10F8011F134600293FF49DADFA
:106FC8005B780132402B02DD5A2BD8BF20338B422D
:106FD800F0D00998DDF820A00490A3E40022012055
:106FE800079203E5B5F59A7F00F33A822D11012D3A
:106FF80040F378839F4E4FF0000ADDE9082304969A
:1070080015F0010F104619464FEA65050AF1010A05
:1070180005D0D6E9002302F065FE02460B46083685
:10702800012DEDDC10461946CDE90801049E0998AA
:1070380006EBCA01A0F154700990DDE90823D1E9F3
:10704800000102F04FFE00230022C7F6F073C7F6D6
:10705800A042CDE9080109990B40934200F2008251
:107068000022C7F69042934240F29F824FF6FF718A
:107078004FF0FF300E460025C7F6EF760B950996C0
:1070880082460890049601E601250A9509F1020353
:10709800179399F8025090E5099ADDF820A0049218
:1070A80040E47548179A10F8011F1346002900F0AC
:1070B800EB825B780132402B02DD5A2BD8BF20339C
:1070C8008B42F0D0099BDDF820A004932AE4AC465B
:1070D800002C40F09D80C5F31303FBB90023304614
:1070E80039460022C3F6F073039503F06DF8DDF816
:1070F8000CC0002840F0DC8100230022C3F6E073B6
:107108003046394602F0EEFDDDF80CC0024601F1CA
:1071180000430C90089116461F46E2E50020002720
:1071280001460026C3F6F071CBF6F0770C90089173
:10713800D7E5ACF15475049B0A9A20462946CDE957
:10714800046716461F46CDE9146701F095FB024611
:107158000B46DDE9040102F0C5FD02460B46204658
:10716800294602F00DFC0023C7F6F0734FF6FF72B4
:10717800C7F69F420B400446934240F285804FF683
:10718800FF73159FC7F6EF739F4200F058814FF6C3
:10719800FF754FF0FF34C7F6EF750A940495F5E5CF
:1071A80008990C98CDF80CC003F036F802F034FDBD
:1071B80002460B460C98089902F0E0FB0F9ADDF89E
:1071C8000CC006460F467ABB74BBCCF313035BBBFB
:1071D80021A3D3E9002302F0F7FF00283FF4D6AD3E
:1071E800DDF828A05846189901F070F8584641462D
:1071F80001F06CF85846494601F068F8584611996C
:1072080001F064F85846079901F060F8FFF78EBB63
:10721800012C83D1002D81D14FF0000ACDF810A0A8
:107228002223CBF80030DDE7304639460CA3D3E9FA
:10723800002302F0C9FF0028D2D1304639460AA3FC
:10724800D3E9002302F0DEFF00283FF49FADC7E733
:10725800089B76E5AFF300809535A094FFFFCF3FFC
:107268009535A094FFFFDF3F35E5AF350000E03FDF
:1072780017830508907D05080B83050800260C90E8
:10728800C3F6F076089655E501F1547C0A906546F8
:10729800CDF810C070E5129E18ABA34D5846009368
:1072A80017A901962A4619AB00F0A0FB10F00706B3
:1072B800044604BFB246CDF810A03FF437AB062E03
:1072C80000F00C81189A3AB129681AA801F0F6FB67
:1072D8005846189900F0FAFF013E199B042E0AD867
:1072E800DFE806F0241F190324006FF000464FF072
:1072F800FF3709960897230755BF09980999DDF8BC
:1073080020A041F0004B52BF0490DDF820A0CDF83A
:1073180010B0FFF70BBB00231D46C7F6F0750995A3
:10732800E9E71A981B9908900991E4E71A9A03F279
:10733800334308921B9A22F4801242EA03520992BC
:10734800D9E7C24637463446FFF738BB00230A93CD
:107358009CE6CDE908457EBB089F6FBBC5F31303C8
:1073680053BB5346C7F6F0732B40B3F1D66F23D9FE
:10737800079D6B6913B92B69012B1DDD0122079944
:10738800584601F085F94946079001F0E1F90028CF
:1073980012DD0B9D002D40F09481099E26F00043DC
:1073A8001B0D1B05A3F580134FF0FF3008906FEA03
:1073B80013536FEA035309930B9D002D00F082804D
:1073C800002714973A46DDE90801C3F650121592D2
:1073D800DDE9142302F086FC0F460646CDE908676E
:1073E8008246099F0491002F7FF4FCAE089800287C
:1073F8007FF4F8AE14E70F9ECDE90845DDF828A024
:10740800002E00F095804FF6FF7225F07F4121F4A1
:107418007001C0F20F0291422B46089900F0CF800C
:10742800CB07C9D55046049901F026FA02460B4607
:107438005046049902F0A4FACDE90801BCE7149873
:1074480001307FF4A4AE0022089213469246C7F694
:10745800F0730993099E2223CBF800300496C1E605
:10746800002622233746CBF80030C7F6F077089677
:107478000997B2460497FFF759BA3FF402AC6D4238
:1074880015F00F030AD0294ADDE9080102EBC3030E
:10749800D3E9002302F050FDCDE908012D1140F099
:1074A800AC800999DDF820A00B950491FFF7EEBB9D
:1074B8000F9A00231E46CBF6E073C3F6E0760896D3
:1074C8000C9228E6099EDDF820A004968AE601239E
:1074D8000A46404600219C46079149E54FF0000ABC
:1074E80008F10103CDF810A01793FFF71FBA079E04
:1074F800C6F1250399453FF7ACABC6F10F0A0B4C13
:10750800CAEB0909DDE9082304EBCA0104EBC90445
:10751800D1E9000102F0E6FBD4E9002302F0E2FB26
:1075280082460491FFF702BA40070020A07C0508B4
:107538000999C1F31303002B35D1089B002B3FF4A5
:1075480028AFDA077FF538AF5046049901F094F96F
:1075580002460B465046049902F010FA02460B46C2
:10756800CDE908230022002302F024FE00287FF43E
:1075780053AE21E7C9F100050D95FFF795BB19F149
:10758800160FFFF666AB6C4BDDE90801A3EBC909E2
:10759800D9E9002302F0D0FC82460491FFF7C6B96E
:1075A8000021FFF7F7BA089BCBE701F154710025DA
:1075B80009910B950491DDF820A0FFF767BB0B9F9D
:1075C800002F7BD00022C7F6F0722A40B2F1D46FA8
:1075D80074D8120D4FF0FF30C2F16B0200FA02F2BC
:1075E80091427FF41DAF00220020C7F6F072089088
:1075F8001A4002F580120992DEE61F2D3BDC15F0D9
:10760800100F14BF6A260026002D0B9614DD4B4E72
:10761800DDE9082315F0010F1046194605D0D6E913
:10762800002302F05FFB02460B4608366D10F1D1CD
:1076380010461946CDE908010B9D7DB1099AC2F3A0
:107648000A53C3F16B03002B08DD1F2B63DD0021F8
:10765800342B089167DD4FF05C720992089E002276
:10766800099D00233046B2462946049502F0A2FD42
:1076780000283FF40BAB4FF0000A2223CDF810A0EE
:10768800CBF80030FFF752B92D4C1146179214F879
:10769800010F0B4618B35B780131402B02DD5A2BE2
:1076A800D8BF20338342F2D00132179200250895C3
:1076B8002E46C7F6F0760996FFF72BBA4FF0FF3241
:1076C8008EE7099F27F000431B0D1B05B3F1D66F0A
:1076D8003FF668AEB3F15C7F3FF672AE9CE50131D0
:1076E8001791E3E7174D4FF0000A04959EE40B4607
:1076F8003EE417A814491AAA00F022FC05287FF4D2
:1077080002AA1B9B1A9943F0FF4343F4E003099331
:107718000891FFF7FEB94FF0FF32089D02FA03F314
:107728001D4008959AE74FF0FF31203B01FA03F31B
:107738001340099392E700BFA07C0508687C050800
:107748000F830508907D05085407002040F2103388
:107758000A46C2F2000301461868FFF7ADB800BF39
:1077680038B50A46094B01461868FFF7A5F80446DC
:107778000D46FEF7BFFB20B12046294602F094FDD6
:1077880038BDBDE8384001F0E9B900BF100300205A
:107798002DE9F04F85B099460B4602914B4903906D
:1077A800D1F800801C4614F8015B08EB050123465C
:1077B800497801F00801C9B20029F3D12D2D7BD0F9
:1077C8002B2D05BF24460B460B4614F8015B39F0F8
:1077D800100112D1D9F1010038BF0020302D04D09A
:1077E80058B14FF00A09CB4608E0217801F0DF01D3
:1077F800582965D008B14FF00809CB46002B5946E7
:107808000CBF6FF000464FF000468DE80C00304684
:10781800002702F09FF830468A46594601F06CFF6F
:10782800BC469DE80C0016E0303DA94525DD8445A1
:1078380094BF0021012151EAD77729D15545D4BFFA
:1078480000210121844518BF002109BB0BFB0C5CFA
:10785800012714F8015B08EB0501497801F00406DB
:10786800F6B2002EE0D111F0030106D0012914BFB1
:10787800572137216D1AA945D9DC791C0BD0C3B91A
:10788800604612B197B9029B136005B0BDE8F08F4E
:107898004FF0FF37DDE70399002B0CBF6FF0004076
:1078A8004FF0004022230B60002AEED0013C0294E6
:1078B800E9E7CCF1000CE3E714F8015B012386E764
:1078C8004FF010096578CB46023497E70C03002087
:1078D80030B440F21034C2F200040D46134601469B
:1078E8002A46206830BCFFF753BF00BF02694B111E
:1078F8002DE9F001934200F114072DDA043300EB6F
:107908008202143211F01F0100EB830303F1040C0F
:1079180029D05C680CF104039A42C1F1200824FACA
:1079280001F438D93D461E6806FA08F6344345F88E
:10793800044B53F8044B9A4224FA01F4F3D8CCEBE5
:107948000203053B23F00303C31818331C60E4B19A
:107958000433DF1BBF101AE00023036100234361D7
:10796800BDE8F0017047624584BF63463946F3D9E4
:1079780053F8044B9A4241F8044BF9D86FEA0C03C8
:107988009B1823F00303C3181833DF1BBF100761CC
:10799800002FE5D1E2E73B46D8E700BF0F481021AA
:1079A8000F4B3022D154013110F8012FC9B2002AEF
:1079B800F8D10C481A216122D154013110F8012F55
:1079C800C9B2002AF8D108481A214122D1540131FC
:1079D80010F8012FC9B2002AF8D170472C83050886
:1079E800A8640120248305081C8305082DE9F04FAD
:1079F8008BB08846A14E06920993079000F0B0FB21
:107A080000680290FEF77CFC029B1A1896F830304A
:107A1800039012F801AC002B00F00981D8F800306F
:107A28009D1C9A78302A40F0FE81033300271D46BA
:107A380013F8012B0137302AF9D016F802B0DFF815
:107A48003C92BBF1000F00F0F5802B784FF0000B53
:107A580019F80340002C00F000826A1C1446013219
:107A68002378F35C002BF9D1994620460299039AB2
:107A780001F066F9E8B12378BBF1000F00F0C1818D
:107A8800C4EB0B0B4FEA8B020592502B00F09B8046
:107A9800702B00F098802246C8F80020B9F1000F3A
:107AA8000DD0002F0CBF0627002738460BB0BDE8C5
:107AB800F08FBBF1000F00F0BE812378E0E7631B75
:107AC8004946013B072B03DD5B100131072BFBDC2B
:107AD800079800F0D3FBA54200F114030490089323
:107AE80080F0DB819B46039B4FF000084746C3F1BB
:107AF800010C0FE0202F5FD03A46043714F8013C00
:107B08004C46A542F35C03F00F0303FA02F348EA7C
:107B1800030819D214F8013C04F1FF395345E9D19F
:107B280009EB0C039D42E5D818460299039A019384
:107B3800CDF800C001F004F9019BDDF800C0002871
:107B4800D8D11C46A542E5D3089B40464BF8048B88
:107B58000499C3EB0B0B4FEAAB030B615D0100F01B
:107B680059FC069A1468281AA04200F32581C0F22D
:107B78004B810025069805998368994200F3F680A1
:107B8800069805994368994280F200815E1AB442CA
:107B980076DCC268022A00F06F81032A00F098811F
:107BA800012A00F0868107985027049900F08EFB7F
:107BB80014980023036078E74BF8048B4FF0000813
:107BC800042742469AE763782B2B00F0F2802D2B8E
:107BD80000F0EA80601C4FF0000BF15C00293FF4D4
:107BE8005AAF19293FF757AF43781039DFF88CC0DF
:107BF800421C1CF8033093B1192B10DC023001E051
:107C0800192B0CDC024601EB8101013092F800C00F
:107C180003EB4101103916F80C30002BF0D1BBF101
:107C2800000F00D04942059B5B18059334E7FFF726
:107C3800B5FEF3E628460299039A01F081F8002878
:107C480040F09D8003982C182B5C19F80320002A1B
:107C580000F0EB80302B40F00B81631C1D4613F8BD
:107C6800012B302AFAD0B35C002B40F002814FF090
:107C78000109A3464F462C46F7E600BFA864012039
:107C8800771E002D40F0E780002F04DD0498394668
:107C980000F038FF054608997B11012207F01F07FD
:107CA8000498A41B51F8233002FA07F231461A420D
:107CB80018BF45F00205FFF719FE069B02275B680F
:107CC8000593002D69D00698C368022B00F0EA805E
:107CD800032B5DD0012B5ED1AA075CD508990B68F0
:107CE8002B43DB0757D5049B002604991D69089B85
:107CF80001EB85001430194653F8042BB2F1FF3F0D
:107D080040F0EB80984243F8046CF4D8049A9368E6
:107D18009D42B8BF2B4680F2F980049901EB83029B
:107D280001330B6101235361022F00F0D9800499BC
:107D38000B699D420EDB14F01F0400F0AC80049B1D
:107D480003EB8505286900F065FBC4F12003984220
:107D580080F2A18004980121FFF7C8FD069A0598D2
:107D6800936801300590984240F395800798A327BF
:107D7800049900F0ABFA149A0023136095E62B7867
:107D88002C46CDF814B04FF001097EE6012798E79C
:107D9800159B002BA7D147F01007049B149803608C
:107DA800059B0998036080E64FF0010BA378A01C9F
:107DB80013E74FF0000BF9E7061B0498314600F073
:107DC800A1FE0546A8B1731E0498012503F01F0102
:107DD8005A1105FA01F100EB82025269114208D0EA
:107DE800AB4205DD0498B11E00F08CFE032500B9F6
:107DF800022504983146FFF779FD059B9B190593E9
:107E0800B8E6CDF814B040E6251A04992A46079832
:107E180000F03EFC059B5B1B00250593049000F1D8
:107E280014030893A6E6002707E605924FF0010918
:107E38002BE62C468146039904EB010B635CF25C4C
:107E4800002A7AD00BF10102144612F8013BF15CCA
:107E58000029F9D114E601251DE728460299039A5D
:107E680000F06EFF0028E4D0A1462C46CB4602E67F
:107E78002546A3460127F0E5159800287FF493AE20
:107E8800099A62270498089913600123149A0361D8
:107E98000B60106009E621277FE7DDF820B04FF07E
:107EA800000851E6159AC2F10103002B3FF473AFA5
:107EB80019E7A6427FF477AE012CE1DD0498611E34
:107EC80000F020FE00283FF46EAE069A5368D7E70C
:107ED800159900293FF467AED2E701320A6023E71B
:107EE800069A22271368013BA3427FF456AF631119
:107EF8000498012204F01F0400EB830302FA04F241
:107F08005B691A4214BF2127222746E75168079860
:107F1800013100F0B3F90646049800F10C01036939
:107F280006F10C009A1C9200FEF720F804990798B5
:107F3800049600F0CBF93369EFE65C46A0E500BF94
:107F48002DE9F04F85B0DFF8B0810C4602909246DB
:107F580098F83030002B00F0AF8023685A1113F0E6
:107F68001F0303930AEB8202009201D004320092AD
:107F7800009A002399460099CB464E4642F8043CA5
:107F88000439029B0191DDF804C0196864464B78F6
:107F9800002B34D018F80320002A70D1202B00F2CF
:107FA80085805E4527DDB9F1070FCCBF002301238B
:107FB800644528BF002393B1C9F108092268234604
:107FC8004FEA8909C9F12007586800FA07F51543EF
:107FD80020FA09F21D6043F8042F9C45F4D8544553
:107FE80098BF4FF0080906D9002244F8042C043C35
:107FF800B346A446914601314B78002BCAD1002ED6
:1080080056D0B9F1070FCCBF00230123644528BF20
:10801800002393B1C9F10809226823464FEA890968
:10802800C9F12005596801FA05F0104321FA09F24F
:10803800186043F8042F6345F4D3A2453FD2019852
:10804800524654F8041B1346A04243F8041B1A4630
:10805800F7D20199002243F8042B9942FBD20099E8
:1080680051F8043C4BB9019B9A4502D139E09A4535
:1080780038D053F8042D002AF9D0052019E009F169
:1080880001090136B9F1080F07DC23681B0102F06A
:108098000F0201311A432260AEE75445ABD90023E1
:1080A8004FF0010944F8043C043CF0E7292B1DD0AB
:1080B800042005B0BDE8F08FFFF770FC4DE7039A88
:1080C800002ACCD0009A039952F8043CC1F120024E
:1080D8004FF0FF3121FA02F21340009A42F8043CB3
:1080E800C0E75346012205201A60E2E7029B0231ED
:1080F8001960002E85D1DBE7A864012010B514466D
:1081080022B110460A4900F02DFD08B9094810BDF2
:108118002046084900F026FD0028F7D020460649E9
:1081280000F020FD034B00280CBF1846002010BDAE
:1081380038830508088305089C81050840F26870A3
:10814800C2F20000704700BF40F26873C2F2000339
:10815800186A7047004870478C0700200020704755
:1081680000487047AC07002040F210330A46C2F2BC
:10817800000301461868FFF7C1BF00BF00487047F9
:10818800AC0700208307C9B270B440D0541E002A3F
:108198003FD003788B4221D0431C04E004B302781B
:1081A800013C8A421AD013F0030F184603F1010369
:1081B800F4D1032C16D8651E94B103788B420DD0E8
:1081C800421C002302E004788C4207D09D421046EE
:1081D80003F1010302F10102F5D1002070BC7047E0
:1081E8002046FBE741EA012646EA064602460430F5
:1081F80013687340A3F1013525EA030313F0803FA8
:1082080003D1043C032CF1D8D5E71046D3E7144634
:10821800CFE71046E2E700BF032A70B422D941EA4B
:1082280000039B0713D00578013A0C780023A54278
:1082380006D01BE010F8015F11F8014FA54215D1D7
:10824800934203F10103F5D1002070BC70470C463E
:108258000346043104301E682568AE4208D1043A4A
:10826800032AF4D8002ADED11046EEE7281BECE7F3
:1082780021461846002AD6D1F6E700BF38B505468C
:10828800C36C0C464BB153F8240080B1026843F824
:10829800242000230361C36038BD0421212200F09B
:1082A800A5FD0346E8640028EDD1002038BD012370
:1082B8002846194603FA04F56A1D920000F096FD57
:1082C8000028F2D044608560E3E700BF31B1C36C99
:1082D8004A6853F82200086043F82210704700BF2C
:1082E8002DE9F0478846D1F810A082B0814601F107
:1082F800140500242F680134BEB23F0C02FB063679
:1083080002FB07F303EB1643B6B206EB03461B0C5E
:10831800A24545F8046BEDDC53B1D8F80820924526
:108328000ADA08EB8A020AF10101C8F81010536151
:10833800404602B0BDE8F087D8F8041048460193DB
:108348000131FFF79BFFD8F8102008F10C01023229
:108358009200044600F10C00FDF708FED8F804105E
:10836800D9F84C20019B52F82100C8F8000042F8C7
:108378002180A046D5E700BF2DE9F84348F63965C6
:108388001F46C3F6E30503F1080306460C4690466C
:1083980085FB0310DB17C3EB6000012837DD0125DF
:1083A80000216D000131A842FBDC3046FFF766FF73
:1083B800089B43610123B8F1090F0146036122DDDF
:1083C80004F1090944444D4615F8013B0A22304698
:1083D800303BFFF785FFA5420146F5D109EB0804BC
:1083E800083C47450CDDC8EB0707E71914F8013BC3
:1083F8000A223046303BFFF773FFBC420146F5D1F5
:108408000846BDE8F8830A344FF00908E9E7002177
:10841800CBE700BF034600201A0C01D11B04102033
:1084280013F07F4F01D108301B0213F0704F01D1B8
:1084380004301B0113F0404F01D102309B00002B88
:1084480002DB5B0001D4202070470130704700BF79
:108458000368024613F0070007D0D9071FD498070E
:108468001FD49B0802201360704799B209B91B0CEE
:10847800102013F0FF0F01D108301B0A190701D192
:1084880004301B09990701D102309B08D90704D48D
:108498005B0801D12020704701301360704700202D
:1084A80070475B0801201360704700BF10B50C4689
:1084B8000121FFF7E3FE01224461026110BD00BF04
:1084C8002DE9F04F0C460E6985B015691746AE4286
:1084D80004DA32463C462E460F461546A36806EB9C
:1084E800050861689845C8BF0131FFF7C7FE00EB72
:1084F800880900F1140309F11409019000204B4583
:1085080003D243F8040B9945FBD807EB850504EB28
:1085180086061437143514341436AF4257D2019AEC
:10852800CDF80890A946CDF80C8002F1180CA046A9
:1085380057F8044BA0B2F0B14246ACF10403002452
:1085480052F8041B1D681FFA81FA090C1FFA85FBF3
:108558002D0C00FB0ABA00FB0151544401EB1441F5
:10856800A4B244EA01450C0C964243F8045BE7D8F0
:108578001C6057F8044C240C21D05CF8041C4246BB
:10858800634600250846B2F800A0000C89B29B4655
:1085980004FB0A00451941EA054143F8041C53F855
:1085A800040B52F8041B1FFA80FA090C04FB01A102
:1085B80001EB15410D0C9642E5D8CBF80010B945F2
:1085C8000CF1040CB4D8DDF80890DDF80C80B8F193
:1085D800000F0BDD59F8043CA9F104091BB105E0B3
:1085E80059F8043D13B9B8F10108F9D1019B1846AF
:1085F800C3F8108005B0BDE8F08F00BF12F0030388
:108608002DE9F041144680460F462BD1A4101BD00B
:10861800D8F848602EB92EE0641015D03568B5B189
:108628002E46E007F8D5394632464046FFF748FF60
:10863800B7B17A686410D8F84C3053F82210396012
:1086480043F822700746E9D13846BDE8F081314643
:1086580032464046FFF734FF306006460560E0E7E3
:108668000746D9E7094A5D1E002352F82520FFF77F
:1086780037FE0746CAE7404640F27121FFF716FF6A
:108688000023C8F8480006460360CAE7907C05083E
:108698002DE9F84F93460A6988464FEA6B158B68AF
:1086A80005EB020A81460AF1010649689E4203DD8C
:1086B8005B0001319E42FBDC4846FFF7DFFD002DE1
:1086C800024600F114040ADD00231F46013344F872
:1086D800047BAB42FAD102EB830303F11404D8F80C
:1086E800107008F1140508EB870714371BF01F0BEF
:1086F80021D0CBF120030021286800FA0BF00143B8
:1087080044F8041B55F8041BAF4221FA03F1F3D8CF
:10871800216009B10AF10206D9F84C30013ED8F8B7
:1087280004101046166153F82120C8F8002043F8B9
:108738002180BDE8F88F55F8043BAF4244F8043B6C
:10874800EAD955F8043BAF4244F8043BF3D8E3E7D1
:1087580003460A69006930B4801A0FD1043203F164
:10876800140592009B1889180433043153F8042D1A
:1087780051F8044DA24203D19D42F7D330BC704753
:10878800944294BF01204FF0FF30F7E72DE9F84FEE
:108798008B460446114658469146FFF7D9FF051EF9
:1087A80061D0BCBF5B46CB462046B8BF9946DBF8D4
:1087B8000410ACBF4FF000084FF00108FFF75EFD52
:1087C800DBF8107009F11405D9F810300BF1140614
:1087D80000240BEB870C09EB83090CF1140C09F14D
:1087E800140900F1140AC0F80C8056F8048B53469B
:1087F80055F804AB32461FFA88F109191FFA8AFBAB
:10880800CBEB01014FEA1A44C4EB184404EB2144B2
:1088180089B241EA04412414A94543F8041B9A4645
:10882800E3D8B445984614D952F8045BA9B22D0C84
:108838000C1905EB2445A4B244EA05412C149445CF
:1088480043F8041BF0D8F343634423F003030433D1
:108858004344043B21B953F8042D013F002AFAD0C0
:108868000761BDE8F88F20462946FFF707FD012379
:1088780045610361BDE8F88F0023C7F6F0730B402C
:10888800A3F15073002B02DD1946002070475B42AC
:1088980000211B15132B0BDD322B02DD012318469B
:1088A80070470122C3F1330302FA03F318467047F5
:1088B8004FF40022002042FA03F170472DE9F843F3
:1088C80000F1140806698946043600EB860634462A
:1088D800374654F8045B2846FFF79CFD0A28C0F188
:1088E8002003C9F8003018DCB045C0F10B0125FAA7
:1088F80001F738BF54F8084C47F07F5747F4401346
:1089080034BF24FA01F10021153005FA00F541EAD7
:10891800050210461946BDE8F8830021B04502D289
:1089280054F8081C371FB0F10B0418D005FA04F5E9
:10893800C0F12B00474545F07F5521FA00F645F474
:10894800401545EA060388BF57F8045C01FA04F1AC
:108958008CBF25FA00F0002040EA0102D9E745F073
:108968007F550A4645F44013D3E700BF2DE9F0418F
:10897800012182B01D461446FFF780FCC5F30A5753
:1089880025F07F43A84623F4700306460FB143F44D
:1089980080130193002C22D002A840F8084D6846A5
:1089A800FFF756FD019B00282ED1009A7261002B1B
:1089B8000CBF01240224B3613461DFB9089A06EBC5
:1089C8008403A0F2324010601869FFF723FD099B69
:1089D800C0EB44101860304602B0BDE8F08101A831
:1089E800FFF736FD01231C463361019B736120307C
:1089F800002FE3D0089AA7F23348C0F1350340446A
:108A08001060099A1360E6E7C0F12001009A03FAA2
:108A180001F123FA00F30A4301937261C7E700BF2B
:108A28002DE9F04383B0884669460646FFF746FFBE
:108A38000D46044601A94046FFF740FFD6F810C08E
:108A4800D8F810E02F462646CEEB0C0E0B4689468A
:108A5800024680469DE80300C1EB000C0CEB4E1E5D
:108A6800BEF1000FC3BF05EB0E5724463D46A3EBEE
:108A78000E59DCBF12464B462046294601F05CFAE7
:108A880003B0BDE8F08300BF172810B504460CDD1D
:108A980000210020C3F6F07100230022C4F2240351
:108AA80001F020F9013CF7D110BD034B03EBC004E2
:108AB800D4E9040110BD00BF907C050870B40139E9
:108AC800156902F114034E11013602EB85051435C0
:108AD80000EB8606AB420CD2014653F8044B9D428C
:108AE80041F8044BF9D8AB1A153B23F003030433C0
:108AF800C018864204D9002340F8043B8642FBD8BC
:108B080070BC704730B44B11046900F114029C42E8
:108B1800B8BF234600DB11DC043300EB8300031DE0
:108B28009A4218D253F8043C2BB9824213D250F817
:108B3800043D002BF9D0012030BC704711F01F0113
:108B4800EAD000EB8304646924FA01F505FA01F11F
:108B5800A142F0D1E0E70020EEE700BF0020C7F611
:108B6800C070704780EA010212F0030F40F03A80AB
:108B780010F0030220F0030021F0030150F804CBA9
:108B880008BF51F8043B0DD082F003024FEAC2023D
:108B98006FF07F4323FA02F251F8043B4CEA020CCF
:108BA80043EA0203ACF101329C4501BF22EA0C0200
:108BB80012F0803F50F804CB51F8043BF2D04FEA52
:108BC8000C604FEA1C2C012828BFB0EB036F08BFCC
:108BD8001B0AF4D003F0FF034FEA1060A0EB030078
:108BE800704700BF10F0030F0AD010F8012B11F8DE
:108BF800013B012A28BF9A42F4D0A2EB0300704738
:108C08004DF8045D4DF8044D4FF0010242EA02228E
:108C180042EA024201F0030C21F0030150F8044B30
:108C280051F8045BBCF1020F26D04BD824F07F4CDE
:108C3800BCEB152FA4EB020323EA04030DD113EABE
:108C4800C21308BF51F8045B0AD18CEA040CBCEBD0
:108C5800056F0CD150F8044BE8E74FEA15255CE0A6
:108C680033F07F4352D10D784FEA146C55E04FEA48
:108C7800146C05F0FF0550E04FEA044CA4EB020326
:108C88004FEA1C4C23EA0403BCEB154F17D113EA37
:108C9800C21308BF51F8045B07D18CEA040CBCEB83
:108CA800054F08D150F8044BE6E71B042ED10D8878
:108CB8004FEA144C31E04FEA05454FEA144C4FEAAD
:108CC80015452AE004F0FF0CBCEB156FA4EB02037A
:108CD80023EA04030DD113EAC21308BF51F8045B59
:108CE8000AD18CEA040CBCEB052F0AD150F8044BCE
:108CF800E8E74FEA156510E014F0FF0F06D051F8C9
:108D0800045B4FEA142C25F07F4506E04FF0000085
:108D18005DF8044B5DF8045B70470CF0FF0205F04A
:108D2800FF00012828BF904204BF4FEA1C2C2D0ADF
:108D3800F3D0A2EB00005DF8044B5DF8045B7047CC
:108D480070B4002A45D041EA000313F0030329D187
:108D5800032A27D905680C68A54223D1141F3AD0E5
:108D6800A5F1013222EA050515F0803F0DD03AE061
:108D78005B686A68A3F10135934225EA03052ED1A1
:108D8800043C28D015F0803F27D10D460346043116
:108D98000430032CECD8661E2CB91C792A79A01A49
:108DA80070BC7047561E04780A789442F7D1C6B151
:108DB8008CB101368B1C891904E08B4203F1010345
:108DC8000BD044B110F8014F13F8012C9442F4D0A1
:108DD800E5E71046E4E72046E2E70020E0E7661E04
:108DE800E1E73046DCE71846DAE700BF10B501FBDB
:108DF80002F100F02BF8044670B150F8042C22F070
:108E08000302043A242A1CD8132A98BF034605D81B
:108E180000221A605A609A60204610BD00211B2A61
:108E2800016098BF00F108034160F1D9242A8160EC
:108E3800C16011BF00F11003016100F11803416125
:108E4800E6E70021FDF7DCF8204610BD2DE9F04FDC
:108E580001F10B04162C83B006462DD924F0070423
:108E6800E30F8C422CBF194643F0010100292CD195
:108E7800304600F0A3FAB4F5FC7F2BD24FEAD40CAD
:108E8800B94F07EBCC02D368934200F000825968CF
:108E980003F10808DA68304621F0030499681B19C1
:108EA8005C68CA6044F0010491605C6000F088FA74
:108EB800404603B0BDE8F08F002310248C422CBF3D
:108EC800194643F001010029D2D00C234FF00008C5
:108ED8003360EDE75FEA542C04BF4FEAD40C4FEA45
:108EE8004C0540F08980A04F07EB8505EB689D4253
:108EF80006D10DE0002A80F24981DB689D4207D047
:108F0800596821F003010A1B0F2AF3DD0CF1FF3C1D
:108F18000CF1010C944A3B6902F1080E734508BF35
:108F2800D2F8049022D0586820F00300011B0F29C2
:108F380000F379810029C2F814E0C2F810E066DA7B
:108F4800B0F5007F80F04581C1084FF0010802EBC1
:108F5800C100891008FA01F851688568D86048EAA4
:108F68000109C2F804909D60EB60836001224FEA1A
:108F7800AC0302FA03F34B4554D819EA030F0DD199
:108F880093402CF0030C19EA030F0CF1040C05D1E3
:108F98005B000CF1040C19EA030FF9D007EBCC09BC
:108FA800E0464846C268904207D150E1002980F265
:108FB8007881D268904200F04A81556825F003050F
:108FC800291B0F29F2DD90461319D56844F00100DA
:108FD80058F8084F41F0010C50603046C3F804C0FF
:108FE800E560AC607B613B61C3F80CE0C3F808E066
:108FF800595000F0E5F95BE7BCF1040F00F2D580A9
:109008004FEA941C0CF1380C4FEA4C056BE71A1820
:1090180003F108083046536843F00103536000F039
:10902800CFF945E7BD686B6823F003094C4504D8C0
:10903800C4EB09030F2B00F39B80DFF830A105EB8D
:109048000902D7F80814DAF800300131234408BFC0
:1090580003F1100B06D003F580530F3323F47F631D
:1090680023F00F0B30465946019200F0ABF9019AF4
:10907800B0F1FF3F804600F05B81824200F2278119
:10908800DAF8043042455B44CAF8043000F05981EC
:10909800D7F808143046013117BFC2EB0802324B2B
:1090A8009B18CAF8043008BFC3F8088418F00703EF
:1090B8001FBFC3F10802C3F58053904403F10802AF
:1090C80008EB0B0308BF4FF480521B051B0DC3EBC5
:1090D800020B594600F076F9431C00F03E81C8EBBC
:1090E80000025A4442F00102DAF80430BD42C7F8DF
:1090F80008805B44C8F80420CAF8043017D0B9F1D6
:109108000F0F40F20481A9F10C02696822F00702EE
:109118004FF0050EA8180F2A01F0010142EA0101DB
:109128006960C0F804E0C0F808E000F21A81DAF8D3
:109138002C20BD68934284BF0C4AD362DAF83020F1
:10914800934284BF094A13636A6822F00302944277
:10915800C4EB020301D80F2B0ADC30464FF000089D
:1091680000F02EF9A4E600BFE4070020FC0D002063
:109178002A1943F0010344F0010430466C6005F1FC
:1091880008085360BA6000F01BF991E65918DA68CC
:109198009C6830464D6803F1080845F00105E26017
:1091A80094604D6000F00CF982E6BCF1140F9CBF8E
:1091B8000CF15B0C4FEA4C057FF695AEBCF1540FF1
:1091C80000F28E804FEA143C0CF16E0C4FEA4C050D
:1091D80089E6420A042A73D9142A9CBF02F15B0962
:1091E8004FEA490508D9542A00F2C3804FEA1039DA
:1091F80009F16E094FEA490507EB8505DFF8B481E7
:10920800AA68AA4276D0516821F00301884202D2A6
:1092180092689542F7D1D068D7F80490D8609A60E0
:10922800D3608360A2E61D1941F00107556144F03F
:109238000104156130465C6003F10808C5F80CE0CC
:10924800C5F808E06F60695000F0BAF830E608F138
:109258000108083018F0030F7FF4A4AE4A461CF04A
:10926800030FA2F108010CF1FF3C00F09A8012688C
:109278008A42F4D07A685B0093423FF6D3AE002B63
:109288003FF4D0AE1A4200F09180C44686E603F15E
:1092980008025B699A4208BF0CF1020C3FF43AAE2F
:1092A800F5E590465519D368304658F8082F69688F
:1092B800D36041F001019A60696000F081F8F7E538
:1092C8004FEA901909F138094FEA490594E7BD4278
:1092D8003FF4D6AE374B9D686A6822F0030236E742
:1092E800BCF5AA7F19D84FEAD43C0CF1770C4FEAA9
:1092F8004C05F8E50125D8F804104FEAA9091046ED
:1093080005FA09F545EA0109C8F8049086E701233A
:109318004546C8F80430002219E740F254539C45EA
:109328000BD84FEA944C0CF17C0C4FEA4C05DAE56B
:10933800BD686A6822F0030209E7FC254FF07E0C3D
:10934800D1E51105090D00297FF4A2AEBA680BEB2F
:10935800090141F001015160E9E601224FF0000BDB
:10936800C2E6304605F1080100F08AF8124B5B6846
:10937800DDE6B2F5AA7F06D84FEAD03909F17709B8
:109388004FEA490538E740F25451FC258A424FF02C
:109398007E099EBF4FEA904909F17C094FEA4905C9
:1093A8002AE77A6822EA03027A6064E75B0008F138
:1093B800040867E7E4070020FC0D0020704700BFA1
:1093C800704700BF38B50546064C084600232360A1
:1093D8003DF0C4FE431C00D038BD2368002BFBD0F1
:1093E8002B6038BDA8650120F8B50F46214D04460D
:1093F800FFF7E4FFAB685E6826F0030606F6EF7336
:10940800DF1B3F0B013F3F03B7F5805F07DB002100
:109418002046FFF7D7FFAB689B19984204D0204637
:10942800FFF7CEFF0020F8BD79422046FFF7CAFFBC
:1094380001300DD0104BF61BA968204646F00106F6
:109448001A684E60D71B1F60FFF7BAFF0120F8BDEE
:1094580000212046FFF7B6FFAB68C21A0F2ADEDDEF
:1094680042F001025A60054B1B68C01A024B186093
:10947800D5E700BFE4070020000E0020EC0B002019
:10948800F8B50D460646002955D0FFF797FF55F861
:10949800041CDFF868C1A5F1080421F00103E218F3
:1094A800DCF808005768904227F0030764D011F0F1
:1094B8000101576032D00021D0194068C00706D496
:1094C800DB199068002949D0D268C260906043F0E7
:1094D8000102E3506260E1B9B3F5007F2CD35A0A68
:1094E800042A65D89809383041000CEB810C4349AF
:1094F800DCF80820624566D0516821F003018B42F0
:1095080002D292689445F7D1D368E360A260D46030
:109518009C603046BDE8F840FFF752BF55F8080C8C
:109528000CF10805241A1B18A068A8423ED0E5686B
:10953800C560A860C0E7F8BDDB080121DCF80400BD
:109548000CEBC3029B1001FA03F3E2609168184325
:10955800CCF80400A160CC609460DAE7284DA842FA
:10956800B2D1CCF8144043F00102CCF81040E060CE
:10957800A0606260E350CCE7FF18CB0707D455F82A
:10958800083CE41AFF18A268E368D3609A6047F0C1
:10959800010363601B4BCCF808401B689F42B8D39B
:1095A800194B30461968FFF71FFFB2E7012183E71F
:1095B80002F15B004100142A97D9542A0CD8180BE1
:1095C8006E30410091E701274D688010134607FA75
:1095D80000F005434D6098E7B2F5AA7F03D8D80B91
:1095E8007730410081E740F254518A4203D8980C01
:1095F8007C30410079E7FC217E2076E7E4070020F3
:10960800EC070020F00B0020FC0D002038B50C46BC
:109618000968054609B1FFF7F9FF28462146BDE864
:109628003840FFF72DBF00BF214B70B505461B68BA
:10963800984230D0C26CA2B100231E4652F82310C3
:1096480039B10C682846FFF71BFF2146002CF8D1DA
:10965800EA6C0136202E3346F0D128461146FFF732
:109668000FFF296C11B12846FFF70AFFD5F84811FA
:1096780051B105F5A676B14206D00C682846FFF729
:10968800FFFEA6422146F8D1696D11B12846FFF7C1
:10969800F7FEAB6B03B970BDEB6B28469847D5F85E
:1096A800E0120029F7D02846BDE87040FFF7AEBFAA
:1096B80010030020F8B50746B8B1D7F8486176B16D
:1096C80075686C1E08D4023506EB850555F8043D0F
:1096D800013C9847631CF9D13668002EF0D1FB6B2A
:1096E80013B138469847F8BDF8BD014B1F68E4E749
:1096F80010030020000000004A1E08BF7047C0F099
:109708002481884240F21681114200F01781B0FA94
:1097180080F3B1FA81F2A2EB0303C3F11F0304A2A1
:1097280002EB03134FF000029F4600BFAFF3008027
:10973800B0EBC17F00BF42EB020228BFA0EBC170B3
:10974800B0EB817F00BF42EB020228BFA0EB817023
:10975800B0EB417F00BF42EB020228BFA0EB417093
:10976800B0EB017F00BF42EB020228BFA0EB017003
:10977800B0EBC16F00BF42EB020228BFA0EBC16093
:10978800B0EB816F00BF42EB020228BFA0EB816003
:10979800B0EB416F00BF42EB020228BFA0EB416073
:1097A800B0EB016F00BF42EB020228BFA0EB0160E3
:1097B800B0EBC15F00BF42EB020228BFA0EBC15073
:1097C800B0EB815F00BF42EB020228BFA0EB8150E3
:1097D800B0EB415F00BF42EB020228BFA0EB415053
:1097E800B0EB015F00BF42EB020228BFA0EB0150C3
:1097F800B0EBC14F00BF42EB020228BFA0EBC14053
:10980800B0EB814F00BF42EB020228BFA0EB8140C2
:10981800B0EB414F00BF42EB020228BFA0EB414032
:10982800B0EB014F00BF42EB020228BFA0EB0140A2
:10983800B0EBC13F00BF42EB020228BFA0EBC13032
:10984800B0EB813F00BF42EB020228BFA0EB8130A2
:10985800B0EB413F00BF42EB020228BFA0EB413012
:10986800B0EB013F00BF42EB020228BFA0EB013082
:10987800B0EBC12F00BF42EB020228BFA0EBC12012
:10988800B0EB812F00BF42EB020228BFA0EB812082
:10989800B0EB412F00BF42EB020228BFA0EB4120F2
:1098A800B0EB012F00BF42EB020228BFA0EB012062
:1098B800B0EBC11F00BF42EB020228BFA0EBC110F2
:1098C800B0EB811F00BF42EB020228BFA0EB811062
:1098D800B0EB411F00BF42EB020228BFA0EB4110D2
:1098E800B0EB011F00BF42EB020228BFA0EB011042
:1098F800B0EBC10F00BF42EB020228BFA0EBC100D2
:10990800B0EB810F00BF42EB020228BFA0EB810041
:10991800B0EB410F00BF42EB020228BFA0EB4100B1
:10992800B0EB010F00BF42EB020228BFA0EB010021
:10993800104670470CBF012000207047B1FA81F231
:10994800C2F11F0220FA02F0704708B14FF0FF3051
:1099580000F00EB80029F8D02DE90340FFF7CCFE3F
:10996800BDE8064002FB00F3A1EB0301704700BF0E
:10997800704700BF81F0004102E000BF83F0004360
:1099880030B54FEA41044FEA430594EA050F08BF92
:1099980090EA020F1FBF54EA000C55EA020C7FEA56
:1099A800645C7FEA655C00F0E2804FEA5454D4EBD3
:1099B8005555B8BF6D420CDD2C4480EA020281EA9D
:1099C800030382EA000083EA010180EA020281EAD5
:1099D8000303362D88BF30BD11F0004F4FEA013127
:1099E8004FF4801C4CEA113102D0404261EB410136
:1099F80013F0004F4FEA03334CEA133302D05242BC
:109A080063EB430394EA050F00F0A780A4F1010477
:109A1800D5F1200E0DDB02FA0EFC22FA05F28018B1
:109A280041F1000103FA0EF2801843FA05F3594197
:109A38000EE0A5F120050EF1200E012A03FA0EFC16
:109A480028BF4CF0020C43FA05F3C01851EBE37140
:109A580001F0004507D54FF0000EDCF1000C7EEB5D
:109A680000006EEB0101B1F5801F1BD3B1F5001F9B
:109A78000CD349085FEA30004FEA3C0C04F10104BA
:109A88004FEA445212F5800F80F09A80BCF1004FE3
:109A980008BF5FEA500C50F1000041EB045141EA65
:109AA800050130BD5FEA4C0C404141EB010111F466
:109AB800801FA4F10104E9D191F0000F04BF014611
:109AC8000020B1FA81F308BF2033A3F10B03B3F1EF
:109AD80020020CDA0C3208DD02F1140CC2F10C027F
:109AE80001FA0CF021FA02F10CE002F11402D8BFDD
:109AF800C2F1200C01FA02F120FA0CFCDCBF41EAA9
:109B08000C019040E41AA2BF01EB0451294330BD77
:109B18006FEA04041F3C1CDA0C340EDC04F1140454
:109B2800C4F1200220FA04F001FA02F340EA03002B
:109B380021FA04F345EA030130BDC4F10C04C4F171
:109B4800200220FA02F001FA04F340EA0300294651
:109B580030BD21FA04F0294630BD94F0000F83F49B
:109B6800801306BF81F480110134013D4EE77FEA7E
:109B7800645C18BF7FEA655C29D094EA050F08BFCA
:109B880090EA020F05D054EA000C04BF19461046AB
:109B980030BD91EA030F1EBF0021002030BD5FEAEF
:109BA800545C05D14000494128BF41F0004130BD17
:109BB80014F580043CBF01F5801130BD01F000456B
:109BC80045F0FE4141F470014FF0000030BD7FEADE
:109BD800645C1ABF194610467FEA655C1CBF0B46D9
:109BE800024650EA013406BF52EA033591EA030FF0
:109BF80041F4002130BD00BF90F0000F04BF0021E8
:109C0800704730B54FF4806404F132044FF000051A
:109C18004FF0000150E700BF90F0000F04BF002193
:109C2800704730B54FF4806404F1320410F00045F9
:109C380048BF40424FF000013EE700BF42004FEAF4
:109C4800E2014FEA31014FEA02701FBF12F07F4371
:109C580093F07F4F81F06051704792F0000F14BF6E
:109C680093F07F4F704730B54FF4607401F00045B2
:109C780021F0004120E700BF50EA010208BF704709
:109C880030B54FF000050AE050EA010208BF7047FE
:109C980030B511F0004502D5404261EB41014FF467
:109CA800806404F132045FEA915C3FF4DCAE4FF06B
:109CB80003025FEADC0C18BF03325FEADC0C18BF52
:109CC800033202EBDC02C2F1200300FA03FC20FAA3
:109CD80002F001FA03FE40EA0E0021FA02F11444F0
:109CE800C1E600BF70B54FF0FF0C4CF4E06C1CEA05
:109CF80011541DBF1CEA135594EA0C0F95EA0C0F7A
:109D080000F0DEF82C4481EA030621EA4C5123EAEC
:109D18004C5350EA013518BF52EA033541F480111B
:109D280043F4801338D0A0FB02CE4FF00005E1FBCE
:109D380002E506F00042E0FB03E54FF00006E1FB18
:109D480003569CF0000F18BF4EF0010EA4F1FF045B
:109D5800B6F5007F64F5407404D25FEA4E0E6D419B
:109D680046EB060642EAC62141EA55514FEAC520AC
:109D780040EA5E504FEACE2EB4F1FD0C88BFBCF528
:109D8800E06F1ED8BEF1004F08BF5FEA500E50F1D9
:109D9800000041EB045170BD06F0004646EA01019F
:109DA80040EA020081EA0301B4EB5C04C2BFD4EBD1
:109DB8000C0541EA045170BD41F480114FF0000ECA
:109DC800013C00F3AB8014F1360FDEBF002001F038
:109DD800004170BDC4F10004203C35DA0C341BDCB2
:109DE80004F11404C4F1200500FA05F320FA04F084
:109DF80001FA05F240EA020001F0004221F00041B8
:109E080010EBD37021FA04F642EB06015EEA430E2A
:109E180008BF20EAD37070BDC4F10C04C4F120055A
:109E280000FA04F320FA05F001FA04F240EA02000D
:109E380001F0004110EBD37041F100015EEA430EDE
:109E480008BF20EAD37070BDC4F1200500FA05F2FE
:109E58004EEA020E20FA04F301FA05F243EA02037D
:109E680021FA04F001F0004121FA04F220EA02008C
:109E780000EBD3705EEA430E08BF20EAD37070BDD2
:109E880094F0000F0FD101F00046400041EB0101B2
:109E980011F4801F08BF013CF7D041EA060195F094
:109EA800000F18BF704703F00046520043EB03034E
:109EB80013F4801F08BF013DF7D043EA060370473B
:109EC80094EA0C0F0CEA135518BF95EA0C0F0CD046
:109ED80050EA410618BF52EA4306D1D181EA03018C
:109EE80001F000414FF0000070BD50EA410606BF86
:109EF8001046194652EA430619D094EA0C0F02D1CB
:109F080050EA013613D195EA0C0F05D152EA03360F
:109F18001CBF104619460AD181EA030101F000412D
:109F280041F0FE4141F470014FF0000070BD41F076
:109F3800FE4141F4780170BD70B54FF0FF0C4CF450
:109F4800E06C1CEA11541DBF1CEA135594EA0C0F6F
:109F580095EA0C0F00F0A7F8A4EB050481EA030EBC
:109F680052EA03354FEA013100F088804FEA0333A3
:109F78004FF0805545EA131343EA12634FEA022271
:109F880045EA111545EA10654FEA00260EF0004132
:109F98009D4208BF964244F1FD0404F5407402D284
:109FA8005B084FEA3202B61A65EB03055B084FEA15
:109FB80032024FF480104FF4002CB6EB020E75EB12
:109FC800030E22BFB61A754640EA0C005B084FEA3A
:109FD8003202B6EB020E75EB030E22BFB61A7546B7
:109FE80040EA5C005B084FEA3202B6EB020E75EB02
:109FF800030E22BFB61A754640EA9C005B084FEA7A
:10A008003202B6EB020E75EB030E22BFB61A754686
:10A0180040EADC0055EA060E18D04FEA051545EA75
:10A0280016754FEA06164FEAC30343EA52734FEA1E
:10A03800C2025FEA1C1CC0D111F4801F0BD141EA97
:10A0480000014FF000004FF0004CB6E711F4801FFC
:10A0580004BF01430020B4F1FD0C88BFBCF5E06FDC
:10A068003FF6AFAEB5EB030C04BFB6EB020C5FEAEC
:10A07800500C50F1000041EB045170BD0EF0004E41
:10A088004EEA113114EB5C04C2BFD4EB0C0541EA73
:10A09800045170BD41F480114FF0000E013C90E670
:10A0A80045EA060E8DE60CEA135594EA0C0F08BF34
:10A0B80095EA0C0F3FF43BAF94EA0C0F0AD150EA33
:10A0C80001347FF434AF95EA0C0F7FF425AF1046C6
:10A0D80019462CE795EA0C0F06D152EA03353FF4EE
:10A0E800FDAE1046194622E750EA410618BF52EA6B
:10A0F80043067FF4C5AE50EA41047FF40DAF52EA3F
:10A1080043057FF4EBAE12E74FF0FF3C06E000BFDB
:10A118004FF0010C02E000BF4FF0010C4DF804CDE8
:10A128004FEA410C7FEA6C5C4FEA430C18BF7FEAA8
:10A138006C5C1BD001B050EA410C0CBF52EA430CD6
:10A1480091EA030F02BF90EA020F0020704710F156
:10A15800000F91EA030F58BF994208BF90422CBFE5
:10A16800D8176FEAE37040F0010070474FEA410CDE
:10A178007FEA6C5C02D150EA013C07D14FEA430CFC
:10A188007FEA6C5CD6D152EA033CD3D05DF8040B6D
:10A19800704700BF8446104662468C46194663469F
:10A1A80000E000BF01B5FFF7B7FF002848BF10F176
:10A1B800000F01BD4DF808EDFFF7F4FF0CBF0120BB
:10A1C80000205DF808FB00BF4DF808EDFFF7EAFF37
:10A1D80034BF012000205DF808FB00BF4DF808EDF2
:10A1E800FFF7E0FF94BF012000205DF808FB00BFE7
:10A1F8004DF808EDFFF7CEFF94BF012000205DF871
:10A2080008FB00BF4DF808EDFFF7C4FF34BF01207D
:10A2180000205DF808FB00BF4FEA410212F500126A
:10A2280015D211D56FF47873B3EB625212D94FEA95
:10A23800C12343F0004343EA505311F0004F23FA7F
:10A2480002F018BF404270474FF00000704750EAD4
:10A25800013005D111F0004008BF6FF00040704791
:10A268004FF00000704700BF4A0011D212F50012EB
:10A2780011D20DD56FF47873B3EB62520ED44FEA56
:10A28800C12343F0004343EA505323FA02F07047D6
:10A298004FF00000704750EA013002D14FF0FF3014
:10A2A80070474FF0000070474FEA4102B2F1E043B7
:10A2B80024BFB3F5001CDCF1FE5C0DD901F0004CA5
:10A2C8004FEAC0024CEA5070B2F1004F40EB8300F5
:10A2D80008BF20F00100704711F0804F21D113F121
:10A2E8003872BCBF01F00040704741F480114FEA5A
:10A2F8005252C2F11802C2F1200C10FA0CF320FAE3
:10A3080002F018BF40F001004FEAC1234FEAD323FF
:10A3180003FA0CFC40EA0C0023FA02F34FEA430369
:10A32800CCE77FEA625307D150EA01331EBF4FF0F2
:10A33800FE4040F44000704701F0004040F0FE400D
:10A3480040F40000704700BF80F0004002E000BF0A
:10A3580081F0004142001FBF5FEA410392EA030F08
:10A368007FEA226C7FEA236C6AD04FEA1262D2EB52
:10A378001363C1BFD218414048404140B8BF5B4257
:10A38800192B88BF704710F0004F40F4000020F0F0
:10A398007F4018BF404211F0004F41F4000121F006
:10A3A8007F4118BF494292EA030F3FD0A2F1010250
:10A3B80041FA03FC10EB0C00C3F1200301FA03F18E
:10A3C80000F0004302D5494260EB4000B0F5000FB1
:10A3D80013D3B0F1807F06D340084FEA310102F170
:10A3E8000102FE2A51D2B1F1004F40EBC25008BF22
:10A3F80020F0010040EA03007047490040EB0000EC
:10A4080010F4000FA2F10102EDD1B0FA80FCACF11A
:10A41800080CB2EB0C0200FA0CF0AABF00EBC25019
:10A4280052421843BCBFD0401843704792F0000F07
:10A4380081F4000106BF80F400000132013BB5E75A
:10A448004FEA41037FEA226C18BF7FEA236C21D0D0
:10A4580092EA030F04D092F0000F08BF0846704735
:10A4680090EA010F1CBF0020704712F07F4F04D103
:10A47800400028BF40F00040704712F100723CBF16
:10A4880000F50000704700F0004343F0FE4040F440
:10A49800000070477FEA226216BF08467FEA2363FE
:10A4A8000146420206BF5FEA412390EA010F40F4E9
:10A4B800800070474FF0000304E000BF10F0004335
:10A4C80048BF40425FEA000C08BF704743F096431C
:10A4D80001464FF000001CE050EA010208BF704737
:10A4E8004FF000030AE000BF50EA010208BF7047BE
:10A4F80011F0004302D5404261EB41015FEA010CD3
:10A5080002BF84460146002043F0B64308BFA3F1CA
:10A518008053A3F50003BCFA8CF2083AA3EBC253AC
:10A5280010DB01FA02FC634400FA02FCC2F12002CB
:10A53800BCF1004F20FA02F243EB020008BF20F002
:10A548000100704702F1200201FA02FCC2F1200268
:10A5580050EA4C0021FA02F243EB020008BF20EA5D
:10A56800DC7070474FF0FF0C1CEAD0521EBF1CEA8B
:10A57800D15392EA0C0F93EA0C0F6FD01A4480EA79
:10A58800010C400218BF5FEA41211ED04FF0006362
:10A5980043EA501043EA5111A0FB01310CF000408E
:10A5A800B1F5000F3EBF490041EAD3715B0040EAB4
:10A5B800010062F17F02FD2A1DD8B3F1004F40EB84
:10A5C800C25008BF20F00100704790F0000F0CF057
:10A5D800004C08BF49024CEA502040EA51207F3A1B
:10A5E800C2BFD2F1FF0340EAC250704740F40000F6
:10A5F8004FF00003013A5DDC12F1190FDCBF00F0E7
:10A6080000407047C2F10002410021FA02F1C2F194
:10A61800200200FA02FC5FEA310040F1000053EA30
:10A628004C0308BF20EADC70704792F0000F00F07E
:10A63800004C02BF400010F4000F013AF9D040EA84
:10A648000C0093F0000F01F0004C02BF490011F418
:10A65800000F013BF9D041EA0C018FE70CEAD15316
:10A6680092EA0C0F18BF93EA0C0F0AD030F0004C96
:10A6780018BF31F0004CD8D180EA010000F000404A
:10A68800704790F0000F17BF90F0004F084691F008
:10A69800000F91F0004F14D092EA0C0F01D1420242
:10A6A8000FD193EA0C0F03D14B0218BF084608D10B
:10A6B80080EA010000F0004040F0FE4040F4000055
:10A6C800704740F0FE4040F4400070474FF0FF0CE8
:10A6D8001CEAD0521EBF1CEAD15392EA0C0F93EA2F
:10A6E8000C0F69D0A2EB030280EA010C49024FEA81
:10A6F800402037D04FF0805343EA111143EA10133A
:10A708000CF000408B4238BF5B0042F17D024FF4F1
:10A71800000C8B4224BF5B1A40EA0C00B3EB510FCC
:10A7280024BFA3EB510340EA5C00B3EB910F24BFB5
:10A73800A3EB910340EA9C00B3EBD10F24BFA3EB3A
:10A74800D10340EADC001B0118BF5FEA1C1CE0D102
:10A75800FD2A3FF650AF8B4240EBC25008BF20F0B5
:10A76800010070470CF0004C4CEA50207F32C2BF09
:10A77800D2F1FF0340EAC250704740F400004FF0A6
:10A788000003013A37E792F0000F00F0004C02BFD7
:10A79800400010F4000F013AF9D040EA0C0093F0A1
:10A7A800000F01F0004C02BF490011F4000F013BFB
:10A7B800F9D041EA0C0195E70CEAD15392EA0C0F63
:10A7C80008D142027FF47DAF93EA0C0F7FF470AF9B
:10A7D800084676E793EA0C0F04D14B023FF44CAFDE
:10A7E80008466EE730F0004C18BF31F0004CCAD173
:10A7F80030F000427FF45CAF31F000437FF43CAFAF
:10A808005FE700BF4FF0FF3C06E000BF4FF0010CD0
:10A8180002E000BF4FF0010C4DF804CD4FEA4002B2
:10A828004FEA41037FEA226C18BF7FEA236C11D0FC
:10A8380001B052EA530C18BF90EA010F58BFB2EBAF
:10A84800030088BFC81738BF6FEAE17018BF40F02F
:10A85800010070477FEA226C02D15FEA402C05D1E3
:10A868007FEA236CE4D15FEA412CE1D05DF8040B68
:10A87800704700BF844608466146FFE70FB5FFF7FB
:10A88800C9FF002848BF10F1000F0FBD4DF808EDB3
:10A89800FFF7F4FF0CBF012000205DF808FB00BFA4
:10A8A8004DF808EDFFF7EAFF34BF012000205DF8FE
:10A8B80008FB00BF4DF808EDFFF7E0FF94BF01204B
:10A8C80000205DF808FB00BF4DF808EDFFF7D2FF48
:10A8D80094BF012000205DF808FB00BF4DF808ED8B
:10A8E800FFF7C8FF34BF012000205DF808FB00BF58
:10A8F8004FEA4002B2F1FE4F0FD34FF09E03B3EB85
:10A9080012620DD94FEA002343F0004310F0004FC4
:10A9180023FA02F018BF404270474FF0000070471A
:10A9280012F1610F01D1420205D110F0004008BFB9
:10A938006FF0004070474FF00000704742000ED2A1
:10A94800B2F1FE4F0BD34FF09E03B3EB126209D462
:10A958004FEA002343F0004323FA02F070474FF018
:10A968000000704712F1610F01D1420202D14FF08D
:10A97800FF3070474FF00000704700BF80B5A2B0AD
:10A9880000AF4FF0C80047F2E103C0F6050398474F
:10A998004FF00003C7F884304DF62903C0F60103D1
:10A9A8009847C7F88400D7F88430002B11D14DF6AA
:10A9B8002133C0F601039847C7F8840007F1040360
:10A9C800D7F8840019464DF28533C0F6010398473D
:10A9D80000E000BF4FF000004DF61553C0F601032C
:10A9E80098474FF00103184607F18807BD4680BD18
:10A9F80080B400AF46F61873C2F200031846BD468D
:10AA080080BC704780B582B000AF786078684FF03E
:10AA180000014FF0320246F20903C0F601039847DD
:10AA28007B684FF0010283F820207B684FF0010219
:10AA380083F829207B684FF0000242F00F0283F868
:10AA480021204FF0000283F822204FF0000283F803
:10AA580023204FF0000283F824207B684FF0000287
:10AA680042F00F0283F827204FF0000283F82820D5
:10AA78007B684FF0FF3283F82A204FF0FF3283F8CB
:10AA88002B204FF0FF3283F82C204FF0FF3283F851
:10AA98002D207B684FF0000242F00A0283F82E2036
:10AAA8004FF0000283F82F204FF0000283F8302087
:10AAB8004FF0000283F831204FF00003184607F1E9
:10AAC8000807BD4680BD00BF80B586B000AF78607E
:10AAD8004FF00003FB6007F10C034FF48010194698
:10AAE8004EF6C553C0F60203984738613B69002B00
:10AAF80010D078684AF60D23C0F6010398474FF046
:10AB08002C0039694EF26D23C0F60103984740F2D4
:10AB1800426334E04FF032037B61FB68012B02D1C2
:10AB28004FF02E037B617B6978684FF480111A46D9
:10AB38004EF69563C0F60203984738613B69002BCF
:10AB480010D078684AF60D23C0F6010398474FF0F5
:10AB58002C0039694EF26D23C0F60103984740F284
:10AB680042630CE0FB68032B07DCFB687868194636
:10AB78004AF69133C0F6010398474FF00003184690
:10AB880007F11807BD4680BD80B483B000AF786078
:10AB980039603B68012B12D17B684FF0000242F00C
:10ABA800140283F82E204FF0000283F82F204FF074
:10ABB800000283F830204FF0000283F831204FF074
:10ABC8000003184607F10C07BD4680BC704700BF5C
:10ABD80090B585B000AF786078684FF480114FF079
:10ABE80032024FF004034EF63D44C0F60204A0477B
:10ABF800F860FB68002B01D0FB6800E0FB68184692
:10AC080007F11407BD4690BD80B400AF4FF00003B4
:10AC18001846BD4680BC704780B500AF4CF6E96366
:10AC2800C0F6010398470346D3F83A35184680BD65
:10AC380080B582B000AF786078684FF000014FF0BF
:10AC4800680246F20903C0F6010398474FF0000373
:10AC5800184607F10807BD4680BD00BF80B584B01F
:10AC680000AF78607B68002B02D140F2853373E037
:10AC78004CF6E963C0F6010398470346D3F83A3522
:10AC8800C72B02D940F25C6366E07B68B3F90030F9
:10AC98009BB21BB218464BF21913C0F60103984732
:10ACA800F860FB68002B2EDA4CF6E963C0F6010366
:10ACB80098470346D3F83A35FB604CF6E963C0F68B
:10ACC800010398470346D3F83A2502F10102C3F875
:10ACD8003A257B6803F1490318464FF000014FF00D
:10ACE800070246F20903C0F6010398477B6803F19F
:10ACF8005C0318464FF000014FF0070246F20903C3
:10AD0800C0F6010398477868F96840F64963C0F6C9
:10AD180003039847B860BB68002B08D04FF00F00BA
:10AD2800B9684DF64573C0F60103984713E04FF430
:10AD380080304DF2D503C0F601039847B860BB6870
:10AD4800002B08D04FF00F00B9684DF64573C0F6D8
:10AD58000103984700BFBB68184607F11007BD46B6
:10AD680080BD00BF80B596B000AF786039603B68A1
:10AD7800012B6ADC07F10803184679684FF00402D2
:10AD880045F67573C0F60103984778684FF00001DF
:10AD98004FF0680246F20903C0F6010398473A8962
:10ADA8007B681A807B6803F1020207F1080303F14C
:10ADB80002031046194646F24D23C0F60103984790
:10ADC800BA7E7B6883F82220FA7E7B6883F823208A
:10ADD800BA8B7B689A84FA8B7B68DA8497F8202090
:10ADE8007B6883F82820B7F921309AB27B68A3F8EA
:10ADF800292097F823207B6883F82B207A6A7B68C0
:10AE0800DA62BA6A7B681A637B6803F1340307F174
:10AE18002C02106818609188927999809A717B68E1
:10AE280003F13B0307F133021168196091889279A5
:10AE380099809A717B6803F1420307F13A0211681D
:10AE480019609188927999809A713B68022B15DC78
:10AE58007B684FF0000283F864204FF0000283F80B
:10AE680065204FF0000283F866204FF0000283F857
:10AE780067207B684FF0000283F863204FF00003DF
:10AE8800184607F15807BD4680BD00BF90B583B08E
:10AE980000AF786039603B68002B02D140F28533FF
:10AEA80018E07B68002B0ADB7C684CF6E963C0F687
:10AEB800010398470346D3F83A359C4202D340F23F
:10AEC800853307E03868796840F64963C0F60303BC
:10AED80098470346184607F10C07BD4690BD00BFCA
:10AEE80080B582B000AF4CF6E963C0F6010398471D
:10AEF80003464FF0000283F83A254FF0000283F82A
:10AF08003B254FF0000283F83C254FF0000283F800
:10AF18003D254FF480304DF2D503C0F60103984724
:10AF280078607B68002B08D04FF00F0079684DF6E9
:10AF38004573C0F60103984700BF7B68184607F1C0
:10AF48000807BD4680BD00BF90B5A1B000AF03465D
:10AF5800FB804FF00003FB674FF00003BB6718E06E
:10AF680007F10C031846B96F4FF0680240F6F57305
:10AF7800C0F603039847F867FB6F002B61D1BB89C4
:10AF8800B7F906201BB29A420FD0BB6F03F1010339
:10AF9800BB67BC6F4CF6E963C0F6010398470346EC
:10AFA800D3F83A359C42DBD300E000BF4CF6E963A6
:10AFB800C0F6010398470346D3F83A3503F1FF3347
:10AFC8007B67BA6F7B6F9A421BDA07F10C0318464E
:10AFD800796F4FF0680240F6F573C0F6030398479F
:10AFE800F867FB6F002B2ED107F10C031846B96FD9
:10AFF80040F64963C0F603039847F867FB6F002BD8
:10B0080023D14CF6E963C0F6010398470346D3F809
:10B018003A2502F1FF32C3F83A254FF480304DF259
:10B02800D503C0F601039847F867FB6F002B0DD0D6
:10B038004FF00F00F96F4DF64573C0F601039847BE
:10B0480004E000BF02E000BF00E000BFFB6F18464D
:10B0580007F18407BD4690BD90B585B000AF786014
:10B0680039604FF00003FB601DE03868F9684FF065
:10B07800680240F6F573C0F603039847B860BB68EA
:10B08800002B01D0BB681BE03B68B3F900309BB2D2
:10B098001AB27B689A4202D14FF0000310E0FB68B5
:10B0A80003F10103FB60FC684CF6E963C0F6010399
:10B0B80098470346D3F83A359C42D6D340F28E33AC
:10B0C800184607F11407BD4690BD00BF80B582B091
:10B0D80000AF786039607B68002B06DB7B68B3F5CE
:10B0E800937F02D83B68002B02D140F2853309E0F8
:10B0F800386879684FF0680240F6F573C0F60303C4
:10B1080098470346184607F10807BD4680BD00BFAB
:10B1180090B59FB000AF78604FF000037B671BE0ED
:10B1280007F108031846796F4FF0680240F6F57387
:10B13800C0F60303984738673B6F002B01D03B6F7D
:10B1480017E03B891AB27B689A4201D17B6F10E005
:10B158007B6F03F101037B677C6F4CF6E963C0F6F4
:10B16800010398470346D3F83A359C42D8D34FF0A9
:10B17800FF33184607F17C07BD4690BDF0B58BB08C
:10B1880004AF78607B6893F838301A467B6893F888
:10B198003930796891F83A10084607F108010090AB
:10B1A800084647F23C21C0F6050141F2A114C0F659
:10B1B8000404A0477B6893F83F301A467B6893F8ED
:10B1C8004030796891F84110084607F1080100906D
:10B1D800084647F23C21C0F6050141F2A114C0F629
:10B1E8000404A0477B6893F846301A467B6893F8B6
:10B1F8004730796891F84810084607F1080100902F
:10B20800084647F23C21C0F6050141F2A114C0F6F8
:10B218000404A0477B68B3F849309BB21A467B68A0
:10B2280093F84B30796891F84C100E46796891F88C
:10B238004D100D46796891F84E100C46796891F8D2
:10B248004F10084607F108010096019502940390F3
:10B25800084647F24C21C0F6050141F2A114C0F698
:10B268000404A0477B68B3F85C309BB21A467B683D
:10B2780093F85E30796891F85F100E46796891F816
:10B2880060100D46796891F861100C46796891F85C
:10B298006210084607F10801009601950294039090
:10B2A800084647F24C21C0F6050141F2A114C0F648
:10B2B8000404A04707F11C07BD46F0BD80B582B065
:10B2C80000AF786078684FF000014FF4C17246F221
:10B2D8000903C0F6010398477B6818464BF2F92327
:10B2E800C0F60103984707F10807BD4680BD00BFB7
:10B2F80080B582B000AF786078684FF000014FF4F5
:10B30800AA7246F20903C0F6010398477B684FF01A
:10B31800300283F846217B684FF0FF3283F84921D9
:10B328004FF0FF3283F84A217B684FF0010283F81F
:10B338004B2107F10807BD4680BD00BF90B583B01B
:10B3480000AF4FF000037B604CF6E963C0F60103E1
:10B3580098470346D3F82235002B2FD04FF000032F
:10B368003B6020E03B684FF4C17202FB03F246F6F3
:10B378005C73C2F20003D318184639684EF6C973D5
:10B38800C0F602039847786078684DF6BD53C0F65A
:10B398000103984741F23143C0F6020398473B68DE
:10B3A80003F101033B603C684CF6E963C0F6010316
:10B3B80098470346D3F822359C42D3D37B68184676
:10B3C80007F10C07BD4690BD80B584B000AF78602A
:10B3D8007B684FF4C17202FB03F246F65C73C2F25B
:10B3E8000003D318184679684EF6C973C0F60203ED
:10B3F8009847F860F8684DF6BD53C0F601039847C2
:10B40800FB68184607F11007BD4680BD90B589B0A6
:10B4180000AF4FF00003FB614CF6E963C0F601038F
:10B4280098470346D3F822353B613B69002B40F32C
:10B43800F8814FF0FF333B603B4618464FF4A85164
:10B44800C0F210014FF27513C0F602039847F86076
:10B45800F8684DF6BD53C0F601039847FB68002B0A
:10B4680002D04FF00D033B604FF4AA737B613B6839
:10B47800012B03D14FF0DB037B614BE03B68022BD0
:10B4880003D14FF0DD037B6144E03B68032B03D11C
:10B498004FF0DE037B613DE03B68042B03D14FF4A2
:10B4A8009F737B6136E03B68052B03D14FF4A07393
:10B4B8007B612FE03B68062B03D140F243137B618D
:10B4C80028E03B68072B03D140F245137B6121E05C
:10B4D8003B68082B03D140F249137B611AE03B68B3
:10B4E800092B03D140F24B137B6113E03B680A2B15
:10B4F80003D14FF4A6737B610CE03B680B2B03D19F
:10B508004FF4A6737B6105E03B680C2B02D14FF426
:10B51800A6737B617B69B3F5AA7F02D04FF0010364
:10B52800FB614CF6E963C0F60103984703464FF008
:10B53800000283F822254FF0000283F823254FF0FC
:10B54800000283F824254FF0000283F825254FF0E8
:10B558000003BB6160E141F23143C0F60203984742
:10B56800BB694FF4C17202FB03F246F65C73C2F288
:10B578000003D31818464BF2C523C0F601039847B9
:10B58800BB694FF4C17202FB03F246F65C73C2F268
:10B598000003D3181846B9697A694FF22123C0F617
:10B5A80002039847F860F8684DF6BD53C0F60103EA
:10B5B8009847FB68002B08D04FF01F00F9684EF23F
:10B5C8006D23C0F60103984722E13B680C2B11DC80
:10B5D800BB694FF4C17202FB03F246F65C73C2F218
:10B5E8000003D2183B68104619464BF66903C0F6AB
:10B5F80001039847BB694FF4C17202FB03F303F5DB
:10B60800A87246F65C73C2F20003D31803F1040370
:10B6180018464FF000014FF0070246F20903C0F642
:10B62800010398474CF6E963C0F6010398470346BF
:10B63800D3F8F630002B62D04CF6E963C0F601036C
:10B6480098470346D3F8FA30BB6046F65C73C2F2FB
:10B658000003BA694FF4C17101FB02F29B181B8801
:10B668001AB2BB689A424AD146F65C73C2F200032A
:10B67800BA694FF4C17101FB02F29B1803F1500340
:10B68800D3F801404CF6E963C0F601039847034636
:10B69800D3F8FE2013464FEAC3739B1A4FEA4303BD
:10B6A800E3187B607B68C3F100037B60BB694FF4E0
:10B6B800C17202FB03F303F5A87246F65C73C2F28B
:10B6C8000003D31803F1040318464FF63D13C0F6E0
:10B6D80003039847BB694FF4C17202FB03F303F5F8
:10B6E800A87246F65C73C2F20003D31803F1040390
:10B6F8001846796840F23133C0F604039847BB69AD
:10B708004FF4C17202FB03F246F65C73C2F2000307
:10B71800D31818464BF6A523C0F60103984746F6FA
:10B728005C73C2F20003BA694FF4C17101FB02F203
:10B738009B189B78002B3BD146F65C73C2F2000342
:10B74800BA694FF4C17101FB02F29B1803F5A073AB
:10B758001B79022B0ED146F65C73C2F20003BA695C
:10B768004FF4C17101FB02F29B1803F5BC733A4A0E
:10B77800C3F8052046F65C73C2F20003BA694FF4B9
:10B78800C17101FB02F29B1803F5A0731B79032B0F
:10B798000ED146F65C73C2F20003BA694FF4C17168
:10B7A80001FB02F29B1803F5BC732C4AC3F8052071
:10B7B8004CF6E963C0F6010398470346D3F82225FF
:10B7C80002F10102C3F8222546F65C73C2F20003B7
:10B7D800BA694FF4C17101FB02F29B181B881BB2B6
:10B7E8004FF0130019464EF23D43C0F60103984747
:10B7F800BB694FF4C17202FB03F246F65C73C2F2F6
:10B808000003D31818464DF28523C0F60103984764
:10B81800BB6903F10103BB61BA693B699A42FFF650
:10B828009AAE4CF6E963C0F6010398470346D3F88D
:10B8380022253B699A4202D040F2436307E0FB6944
:10B84800002B02D14FF0000301E040F25A63184682
:10B8580007F12407BD4690BD00FF7F4700000000A8
:10B86800B0B5BCB000AF786039607B6807F10801FB
:10B878001A464FF0DE03084611461A4645F6757318
:10B88800C0F6010398473B68012B07D14FF000032E
:10B8980087F8E3304FF0000387F8E4303B68022B69
:10B8A80003DC4FF0010387F8E5303B68032B00F316
:10B8B800B98097F8E3207B6883F8642097F8E42040
:10B8C8007B6883F8652097F8E5207B6883F8662015
:10B8D8007B6803F167031D4607F16C040FCC2860F1
:10B8E8006960AA60EB6023782B74D7F87E207B68A8
:10B8F800C3F87920D7F882307A68C2F87D30D7F853
:10B9080086307A68C2F88130D7F88A307A68C2F807
:10B918008530D7F88E307A68C2F88930D7F89230F7
:10B928007A68C2F88D3097F896207B6883F8912062
:10B9380097F897207B6883F8922097F898207B687F
:10B9480083F8932097F899207B6883F8942097F8D8
:10B958009A207B6883F895204FF00003C7F8EC30F5
:10B968004BE0D7F8EC3003F164034FEA430307F1E7
:10B97800F002D31833F8E13C99B27B68D7F8EC2091
:10B9880002F1980223F812104FF00003C7F8E830CC
:10B9980029E0D7F8EC2013464FEA83039B18D7F821
:10B9A800E8209B1803F144034FEA430307F1F00230
:10B9B800D31833F8DD3C99B27868D7F8EC201346F1
:10B9C8004FEA83039B18D7F8E8209B1803F1740308
:10B9D8004FEA4303C3180A465A80D7F8E83003F100
:10B9E8000103C7F8E830D7F8E830042BD1DDD7F8E1
:10B9F800EC3003F10103C7F8EC30D7F8EC30052B35
:10BA0800AFDD7B684FF0000283F896204FF000020C
:10BA180083F897204FF0000283F898204FF0000237
:10BA280083F899203B68042B10DC7B684FF00002F8
:10BA380083F83F214FF0000283F840214FF00002C5
:10BA480083F841214FF0000283F842213B68072B1D
:10BA580008DC7B684FF0FF3283F849214FF0FF3252
:10BA680083F84A213B68092B04DC7B684FF001020C
:10BA780083F84B213B680C2B07DC7B68064AC3F82C
:10BA88004C217B68044AC3F850214FF00003184644
:10BA980007F1F007BD46B0BD0000000080B584B0D6
:10BAA80000AF78604FF00003FB607B689B78082B41
:10BAB8001BD17B68D3F84D3018464BF2E503C0F62E
:10BAC80002039847B860B86842F66113C0F60203EB
:10BAD8009847F860FB68002B07D04FF02700F968FB
:10BAE8004EF26D23C0F601039847FB68184607F12C
:10BAF8001007BD4680BD00BF80B584B000AF786038
:10BB08004FF00003FB607B689B78082B1BD17B6898
:10BB1800D3F84D3018464BF2E503C0F602039847B8
:10BB2800B860B86842F69513C0F602039847F86003
:10BB3800FB68002B07D04FF02800F9684EF26D2300
:10BB4800C0F601039847FB68184607F11007BD4681
:10BB580080BD00BF80B500AF4CF6E963C0F60103B5
:10BB680098470346D3F82235184680BD80B584B07F
:10BB780000AF4BF65D33C0F60103984778604FF08D
:10BB88000003BB604FF00003FB6018E0F8684BF659
:10BB9800F173C0F60103984738603B68002B09D061
:10BBA8003B6893F86630002B05D0BB6803F10103AE
:10BBB800BB6000E000BFFB6803F10103FB60FA68AB
:10BBC8007B689A42E2DBBB68184607F11007BD465E
:10BBD80080BD00BF80B586B000AF78607B68002B61
:10BBE80002D140F28533D9E07B68B3F900309BB2CB
:10BBF8001BB218464BF62973C0F6010398477861C3
:10BC08007B68B3F900309BB21BB218464BF68D73B4
:10BC1800C0F60103984738613B69002B48D07B691F
:10BC2800002B45DB7B68B3F900309BB21BB24FF0A9
:10BC3800120019464EF23D43C0F6010398477B684F
:10BC48009A783B699B789A4206D038694BF2C523AB
:10BC5800C0F60103984764E07B689B78062B0ED0FA
:10BC68007B68D3F84D203B69D3F84D309A4206D013
:10BC780038694BF2C523C0F60103984751E07B6849
:10BC88009B78062B4DD17B6893F85E203B6993F82F
:10BC98005E309A4205D17B681A6E3B691B6E9A42E8
:10BCA8003FD038694BF2C523C0F60103984738E006
:10BCB8004BF65D33C0F601039847B860BB683D2B6F
:10BCC80002DD40F2416369E0BB687B61BB684FF409
:10BCD800C17202FB03F246F65C73C2F20003D3188A
:10BCE8003B614CF6E963C0F6010398470346D3F875
:10BCF800222502F10102C3F822257B68B3F900303E
:10BD08009BB21BB24FF0110019464EF23D43C0F6EC
:10BD18000103984738694BF2C523C0F601039847D9
:10BD280000E000BF3B69184679684FF4AA7245F6EF
:10BD38007573C0F6010398473B6903F5AA73184663
:10BD48004FF63D13C0F6030398473B6918464BF678
:10BD5800A523C0F6010398473B69184679694EF652
:10BD6800C973C0F602039847F860FB68002B13D12B
:10BD78004FF480304DF2D503C0F601039847F860C0
:10BD8800FB68002B09D04FF00F00F9684DF645739A
:10BD9800C0F60103984700E000BFFB68184607F1AA
:10BDA8001807BD4680BD00BF80B584B000AF4FF016
:10BDB8000003BB604BF65D33C0F60103984778601B
:10BDC8004FF00003FB6015E0FB684FF4C17202FB03
:10BDD80003F246F65C73C2F20003D318BB60BB687B
:10BDE80018464BF60133C0F601039847FB6803F188
:10BDF8000103FB60FA687B689A42E5DB4CF6E9636D
:10BE0800C0F60103984703464FF0000283F8222545
:10BE18004FF0000283F823254FF0000283F8242511
:10BE28004FF0000283F825254FF00003184607F16C
:10BE38001007BD4680BD00BF90B587B000AF7860E1
:10BE48004FF000037B614FF00003FB604BF65D335E
:10BE5800C0F601039847B8604FF000033B6152E019
:10BE68003B694FF4C17202FB03F246F65C73C2F2FF
:10BE78000003D318FB60FB68B3F900309BB21AB219
:10BE88007B689A4204D03B6903F101033B613AE0C5
:10BE9800FB6818464BF60133C0F6010398474CF689
:10BEA800E963C0F6010398470346D3F8222502F157
:10BEB800FF32C3F822253C694CF6E963C0F601035A
:10BEC80098470346D3F822359C4221D2BB6803F138
:10BED800FF334FF4C17202FB03F246F65C73C2F201
:10BEE8000003D318F86819464FF4AA7245F675731B
:10BEF800C0F60103984738694BF2D133C0F6010305
:10BF08009847786104E03A69BB689A42A8DB00E088
:10BF180000BF7B69184607F11C07BD4690BD00BFEE
:10BF280080B586B000AF78604FF000033B614BF6F8
:10BF38005D33C0F601039847F8604FF000037B615A
:10BF480014E078694BF6F173C0F60103984738613D
:10BF58003B69B3F900309BB21AB27B689A4201D1AF
:10BF68007B6909E07B6903F101037B617A69FB68FE
:10BF78009A42E6DB4FF0FF33184607F11807BD4633
:10BF880080BD00BF80B586B000AF78604FF0000379
:10BF98003B614BF65D33C0F601039847F8604FF0FC
:10BFA80000037B6114E078694BF6F173C0F6010376
:10BFB800984738613B69B3F900309BB21AB27B6885
:10BFC8009A4201D13B6909E07B6903F101037B6176
:10BFD8007A69FB689A42E6DB4FF00003184607F1DE
:10BFE8001807BD4680BD00BF80B582B000AF78603D
:10BFF8007B68002B08DB4BF65D33C0F601039847DE
:10C0080002467B689A4202DC4FF0000309E07B6835
:10C018004FF4C17202FB03F246F65C73C2F20003EE
:10C02800D318184607F10807BD4680BD80B586B00D
:10C0380000AF0346FB804FF000033B614BF65D33D6
:10C04800C0F601039847F8604FF000037B6115E0E4
:10C0580078694BF6F173C0F60103984738613B697C
:10C06800B3F949319BB2B7F906201BB29A4201D104
:10C078003B6909E07B6903F101037B617A69FB682D
:10C088009A42E5DB4FF00003184607F11807BD4652
:10C0980080BD00BF80B582B000AF786078684FF08F
:10C0A80000014FF0800246F20903C0F601039847E9
:10C0B8004FF00003184607F10807BD4680BD00BFD2
:10C0C80080B586B000AF78604FF00003FB6007F1E1
:10C0D8000C034FF48060C0F2100019464EF6C553A9
:10C0E800C0F60203984778617B69002B10D0786806
:10C0F8004CF29D03C0F6010398474FF02D00796973
:10C108004EF26D23C0F60103984740F2426325E0E2
:10C118004FF080033B613B6978684FF48061C0F25F
:10C1280010011A464EF69563C0F6020398477861E7
:10C138007B69002B10D078684CF29D03C0F6010390
:10C1480098474FF02D0079694EF26D23C0F6010330
:10C15800984740F2426301E04FF00003184607F1A8
:10C168001807BD4680BD00BF90B585B000AF7860A8
:10C1780078684FF48061C0F210014FF080024FF0F0
:10C1880001034EF63D44C0F60204A047F860FB6880
:10C19800002B01D0FB6800E0FB68184607F1140784
:10C1A800BD4690BD80B584B000AF786078684FF028
:10C1B80000014FF0540246F20903C0F60103984704
:10C1C8007B684FF000021A734FF0000262F03D02E4
:10C1D8005A734FF0000242F001029A734FF00002C6
:10C1E800DA737B684FF000021A744FF000025A7439
:10C1F8004FF000029A744FF00002DA747B684FF037
:10C20800000242F001021A754FF000025A754FF011
:10C2180000029A754FF00002DA757B684FF0000251
:10C2280042F008021A764FF000025A764FF00002E8
:10C238009A764FF00002DA767B684FF0000262F0DF
:10C248007F021A774FF0000242F025025A774FF02A
:10C2580000029A774FF00002DA777B684FF000020D
:10C2680083F820204FF0000283F821204FF00002CD
:10C2780083F822204FF0000283F823207B684FF0D8
:10C28800000242F0010283F824204FF0000283F8F4
:10C2980025204FF0000283F826204FF0000283F893
:10C2A80027207B684FF0000242F0080283F828201C
:10C2B8004FF0000283F829204FF0000283F82A206B
:10C2C8004FF0000283F82B207B684FF0000242F009
:10C2D80002021A724FF000025A724FF000029A726C
:10C2E8004FF00002DA724FF00003FB6013E07A6847
:10C2F800FB68D31803F12C034FF000021A707A6818
:10C30800FB68D31803F134034FF000021A70FB687E
:10C3180003F10103FB60FB68072BE8DD7B684FF046
:10C32800000262F00B0283F83C204FF0000242F05A
:10C33800010283F83D204FF0000283F83E204FF0C1
:10C34800000283F83F207B684FF0000262F00B0286
:10C3580083F840204FF0000242F0010283F84120A8
:10C368004FF0000283F842204FF0000283F8432088
:10C378007B684FF0000283F844204FF0000283F8F6
:10C3880045204FF0000283F846204FF0000283F862
:10C3980047207B684FF0FF3283F848204FF0FF3288
:10C3A80083F849204FF0FF3283F84A204FF0FF32DC
:10C3B80083F84B207B684FF0000242F0050283F8B7
:10C3C8004C204FF0000283F84D204FF0000283F814
:10C3D8004E204FF0000283F84F207B684FF0000298
:10C3E80042F0050283F850204FF0000283F85120F4
:10C3F8004FF0000283F852204FF0000283F85320D8
:10C408004FF00003184607F11007BD4680BD00BF76
:10C4180080B586B000AF78604FF00003BB6007F1CD
:10C4280008034FF40060C0F2100019464EF6C553D9
:10C43800C0F602039847F860FB68002B10D07868B4
:10C448004CF2AD13C0F6010398474FF02E00F9687F
:10C458004EF26D23C0F60103984740F242634DE067
:10C468004FF054037B61BB68012B02D14FF04403AA
:10C478007B61BB68022B02D14FF04C037B61BB6828
:10C48800032B02D14FF044037B617B6978684FF43A
:10C498000061C0F210011A464EF69563C0F6020319
:10C4A8009847F860FB68002B10D078684CF2AD1301
:10C4B800C0F6010398474FF02E00F9684EF26D233D
:10C4C800C0F60103984740F2426317E04FF00003BB
:10C4D8003B6103E03B6903F101033B613B69072BC7
:10C4E800F8DDBB68042B07DCBB68786819464CF29A
:10C4F8001153C0F6010398474FF00003184607F19F
:10C508001807BD4680BD00BF80B485B000AF786015
:10C5180039603B68012B44DC4FF00003FB6013E0FB
:10C528007A68FB68D31803F12C034FF000021A70E5
:10C538007A68FB68D31803F134034FF000021A70CD
:10C54800FB6803F10103FB60FB68072BE8DD7B68F0
:10C558004FF0000262F0170283F83C204FF000020F
:10C5680042F0030283F83D204FF0000283F83E209A
:10C578004FF0000283F83F207B684FF0000262F022
:10C58800170283F840204FF0000242F0030283F8BC
:10C5980041204FF0000283F842204FF0000283F858
:10C5A80043203B68022B29DC7B684FF0000262F0D5
:10C5B800170283F83C204FF0000242F0030283F890
:10C5C8003D204FF0000283F83E204FF0000283F830
:10C5D8003F207B684FF0000262F0170283F840208A
:10C5E8004FF0000242F0030283F841204FF00002AE
:10C5F80083F842204FF0000283F843203B68032B66
:10C6080047DC7B684FF0000283F844204FF00002BB
:10C6180083F845204FF0000283F846204FF00002CF
:10C6280083F847207B684FF0FF3283F848204FF0AB
:10C63800FF3283F849204FF0FF3283F84A204FF049
:10C64800FF3283F84B207B684FF0000242F005026E
:10C6580083F84C204FF0000283F84D204FF0000281
:10C6680083F84E204FF0000283F84F207B684FF08C
:10C67800000242F0050283F850204FF0000283F8D0
:10C6880051204FF0000283F852204FF0000283F847
:10C6980053203B68042B00F3A8807B685B69002B60
:10C6A8000ED17B684FF0000242F001021A754FF07C
:10C6B80000025A754FF000029A754FF00002DA75C1
:10C6C8007B685B69012B0ED17B684FF0000242F05A
:10C6D80002021A754FF000025A754FF000029A755F
:10C6E8004FF00002DA757B689B69022B0ED17B68DC
:10C6F8004FF0000242F007021A764FF000025A7615
:10C708004FF000029A764FF00002DA767B689B6958
:10C71800032B0ED17B684FF0000242F008021A7614
:10C728004FF000025A764FF000029A764FF000025E
:10C73800DA767B685B6A002B12D17B684FF00002C7
:10C7480042F0010283F824204FF0000283F82520EC
:10C758004FF0000283F826204FF0000283F82720CC
:10C768007B685B6A012B12D17B684FF0000242F0B4
:10C77800020283F824204FF0000283F825204FF0AE
:10C78800000283F826204FF0000283F827207B68F8
:10C798009B6A022B12D17B684FF0000242F007021D
:10C7A80083F828204FF0000283F829204FF0000278
:10C7B80083F82A204FF0000283F82B207B689B6ABD
:10C7C800032B12D17B684FF0000242F0080283F875
:10C7D80028204FF0000283F829204FF0000283F848
:10C7E8002A204FF0000283F82B204FF00003184650
:10C7F80007F11407BD4680BC704700BF90B585B0EF
:10C8080000AF786078684FF40061C0F210014FF013
:10C8180054024FF005034EF63D44C0F60204A0470B
:10C82800B860BB68002B01D0BB680BE04FF0000379
:10C83800FB6003E0FB6803F10103FB60FB68072B67
:10C84800F8DDBB68184607F11407BD4690BD00BF68
:10C85800B0B582B000AF786078684FF000014FF053
:10C86800100246F20903C0F6010398477B684FF0AF
:10C8780000021A704FF000025A704FF000029A70CE
:10C888004FF00002DA707B684FF0000242F00102BC
:10C898001A724FF000025A724FF000029A724FF06B
:10C8A8000002DA727B684FF0000242F001021A734C
:10C8B8004FF000025A734FF000029A734FF00002D3
:10C8C800DA737B684FF0000242F050021A714FF0A1
:10C8D80000025A714FF000029A714FF00002DA71AB
:10C8E8007B684FF0000242F010021A744FF0000209
:10C8F80042F00E025A744FF000029A744FF0000290
:10C90800DA747B684FF000021A754FF000025A750E
:10C918004FF000029A754FF00002DA757B6803F158
:10C92800180247F26C23C0F6050315461C460FCCC7
:10C9380028606960AA60EB6003CC2861696122887D
:10C94800A3782A83AB764FF00003184607F108074F
:10C95800BD46B0BD80B586B000AF78604FF000032B
:10C96800FB6007F10C034FF44060C0F21000194659
:10C978004EF6C553C0F60203984778617B69002BD1
:10C9880010D078684CF65903C0F6010398474FF069
:10C998002F0079694EF26D23C0F60103984740F2E3
:10C9A800426325E04FF4CC733B613B6978684FF4F0
:10C9B8004061C0F210011A464EF69563C0F60203B4
:10C9C800984778617B69002B10D078684CF659033A
:10C9D800C0F6010398474FF02F0079694EF26D2396
:10C9E800C0F60103984740F2426301E04FF00003AC
:10C9F800184607F11807BD4680BD00BF90B585B041
:10CA080000AF786078684FF44061C0F210014FF4CD
:10CA1800CC724FF002034EF63D44C0F60204A04724
:10CA2800F860FB68002B01D0FB6800E0FB68184643
:10CA380007F11407BD4690BDB0B582B000AF78606D
:10CA480078684FF000014FF4217246F20903C0F6EE
:10CA5800010398477A6847F28823C0F6050315460C
:10CA68001C460FCC28606960AA60EB602288A37816
:10CA78002A82AB747B6803F1840247F29C23C0F6D8
:10CA8800050315461C460FCC28606960AA60EB6058
:10CA9800206828617B6803F5827247F2B023C0F6EC
:10CAA800050314461D460FCD20606160A260E36057
:10CAB80028682061AA88AB79A282A3757B6803F5F0
:10CAC800C27247F29C23C0F6050315461C460FCCDC
:10CAD80028606960AA60EB60206828617B6803F5BC
:10CAE800017247F2C823C0F60503186810601B7965
:10CAF80013717B684FF0000262F0260283F88020F1
:10CB08004FF0000242F05D0283F881204FF00002EE
:10CB180083F882204FF0000283F883204FF000034F
:10CB2800184607F10807BD46B0BD00BF80B586B0FE
:10CB380000AF78604FF00003FB6007F10C034FF47F
:10CB48008050C0F2100019464EF6C553C0F60203D5
:10CB5800984738613B69002B10D078684CF6412320
:10CB6800C0F6010398474FF0300039694EF26D2343
:10CB7800C0F60103984740F242633CE04FF421734A
:10CB88007B61FB68012B02D14FF4C2737B61FB68A8
:10CB9800022B02D14FF401737B617B6978684FF4F3
:10CBA8008051C0F210011A464EF69563C0F6020392
:10CBB800984738613B69002B10D078684CF64123C0
:10CBC800C0F6010398474FF0300039694EF26D23E3
:10CBD800C0F60103984740F242630CE0FB68022B61
:10CBE80007DCFB68786819464CF60943C0F6010370
:10CBF80098474FF00003184607F11807BD4680BD57
:10CC0800B0B483B000AF786039603B68012B0FD1B6
:10CC18007B6803F5C27247F29C23C0F605031546EC
:10CC28001C460FCC28606960AA60EB602068286108
:10CC38003B68022B0ADC7B6803F5017247F2C823C4
:10CC4800C0F60503186810601B7913714FF00003D4
:10CC5800184607F10C07BD46B0BC704790B585B0C3
:10CC680000AF786078684FF48051C0F210014FF43B
:10CC780021724FF003034EF63D44C0F60204A0476C
:10CC8800F860FB68002B01D0FB6800E0FB681846E1
:10CC980007F11407BD4690BD80B582B000AF78603B
:10CCA80078684FF000014FF01C0246F20903C0F605
:10CCB800010398474FF00003184607F10807BD46DF
:10CCC80080BD00BF80B586B000AF78604FF000032C
:10CCD800FB6007F10C034FF4A050C0F21000194696
:10CCE8004EF6C553C0F60203984738613B69002BDE
:10CCF80010D078684CF6A143C0F6010398474FF06E
:10CD0800310039694EF26D23C0F60103984740F2AD
:10CD1800426367E04FF01C037B61FB68032B02D181
:10CD28004FF010037B61FB68022B02D14FF0140314
:10CD38007B61FB68012B02D14FF018037B617B6993
:10CD480078684FF4A051C0F210011A464EF6956368
:10CD5800C0F60203984738613B69002B10D0786809
:10CD68004CF6A143C0F6010398474FF031003969EA
:10CD78004EF26D23C0F60103984740F2426331E05A
:10CD8800FB68012B0CDC7B684FF000021A744FF033
:10CD980000025A744FF000029A744FF00002DA74DD
:10CDA800FB68022B0CDC7B684FF000021A754FF011
:10CDB80000025A754FF000029A754FF00002DA75BA
:10CDC800FB68032B0CDC7B684FF000021A764FF0EF
:10CDD80000025A764FF000029A764FF00002DA7697
:10CDE8004FF00003184607F11807BD4680BD00BF85
:10CDF80090B585B000AF786078684FF4A051C0F264
:10CE080010014FF01C024FF004034EF63D44C0F6EB
:10CE18000204A047F860FB68002B01D0FB6800E023
:10CE2800FB68184607F11407BD4690BD80B500AFF2
:10CE38004CF6D840C2F200004FF0000140F23E52DA
:10CE480046F20903C0F6010398474CF6D840C2F2EF
:10CE580000004AF60D23C0F6010398470F484CF22C
:10CE68009D03C0F6010398470D484CF2AD13C0F678
:10CE7800010398470B484CF65903C0F6010398473D
:10CE880009484CF64123C0F60103984707484CF679
:10CE9800A143C0F60103984780BD00BF0ACD00201A
:10CEA8008ACD0020DECD002076CF0020FAD10020E8
:10CEB80080B582B000AF78607B68002B0AD07868B4
:10CEC8004FF000014FF4C17246F20903C0F60103A6
:10CED800984700E000BF07F10807BD4680BD00BFC6
:10CEE80080B400AF4CF6D843C2F200031846BD46E2
:10CEF80080BC704780B582B000AF4CF63563C0F691
:10CF0800010398474CF6D840C2F200004AF6D123F4
:10CF1800C0F601039847786028484CF2C903C0F668
:10CF280001039847786026484CF21943C0F601037C
:10CF38009847786023484CF65D13C0F6010398477C
:10CF4800786021484CF63533C0F60103984778607D
:10CF58001E484CF6CD43C0F60103984778607B68BD
:10CF6800002B24D14CF6D843C2F20003D3F8223563
:10CF7800002B0FD04BF21543C0F601039847786099
:10CF88007A6840F25A639A4204D14BF24533C0F6AC
:10CF9800010398474CF6D843C2F20003D3F83A3558
:10CFA800002B04D04CF6D973C0F6010398474FF014
:10CFB8000003184607F10807BD4680BD0ACD0020CA
:10CFC8008ACD0020DECD002076CF0020FAD10020C7
:10CFD80080B59EB000AF4FF0FF33BB6607F1680322
:10CFE80018464FF43541C0F210014FF27513C0F6E0
:10CFF8000203984738673B6F002B01D03B6F5FE017
:10D00800BB6E022B02DD4FF0000359E04FF04E03D8
:10D01800FB66BB6E012B03D14FF04E03FB660DE0A0
:10D02800BB6E022B03D14FF06303FB6606E04AF6A2
:10D03800E963C0F601039847034641E04CF6E9630B
:10D04800C0F6010398470346D3F83A3503F1FF3396
:10D058007B6731E03B461846796FFA6E40F6F57308
:10D06800C0F60303984738673B6F002B05D04AF694
:10D07800E963C0F60103984721E0BB6E3A461046C3
:10D0880019464AF66D53C0F6010398473B461846C1
:10D09800796F40F64963C0F60303984738673B6FDA
:10D0A800002B05D04AF6E963C0F60103984706E06D
:10D0B8007B6F03F1FF337B677B6F002BCADA3B6F13
:10D0C800184607F17807BD4680BD00BF80B584B01B
:10D0D80000AF78604FF00003FB607B68B3F5006F2A
:10D0E80032D0B3F5006F0DDC202B22D0202B04DCCE
:10D0F800022B1ED0102B1CD017E0402B2CD0802BDD
:10D108002AD012E0B3F5804F26D0B3F5804F06DC65
:10D11800B3F5805F28D0B3F5005F2DD005E0B3F5F7
:10D12800004F19D0B3F5803F2ED04FF00003FB60BD
:10D1380032E04CF6D840C2F200004AF6D933C0F6C5
:10D1480001039847F86027E016484CF27113C0F6BF
:10D1580001039847F8601FE013484CF60503C0F632
:10D1680001039847F86017E010484CF60523C0F60D
:10D1780001039847F8600FE00D484CF66543C0F688
:10D1880001039847F86007E00A484CF6F953C0F6DF
:10D1980001039847F86000BFFB68184607F11007BD
:10D1A800BD4680BD0ACD00208ACD0020DECD0020FE
:10D1B80076CF0020FAD1002080B400AF4CF6D843D7
:10D1C800C2F20003D3F81E33002B02D14FF0000344
:10D1D80008E0064B1B78002B02D14FF0000301E05A
:10D1E8004FF001031846BD4680BC704776CF00203B
:10D1F80080B400AF4CF6D843C2F20003D3F80A312A
:10D20800002B02D14FF0000313E04CF6D843C2F2D2
:10D218000003D3F80E31002B02D14FF0000308E0D1
:10D22800064B1B78002B02D14FF0000301E04FF0B2
:10D2380001031846BD4680BC704700BFF6CD0020EC
:10D2480080B483B000AF78604CF6D843C2F20003D4
:10D25800D3F82A207B681340184607F10C07BD460F
:10D2680080BC704780B483B000AF78607B68002BC7
:10D2780000BF07F10C07BD4680BC704780B483B07F
:10D2880000AF786007F10C07BD4680BC704700BF4F
:10D2980080B483B000AF786007F10C07BD4680BC4E
:10D2A800704700BF80B483B000AF786007F10C0707
:10D2B800BD4680BC704700BF80B483B000AF7860C3
:10D2C80007F10C07BD4680BC704700BF80B483B02F
:10D2D80000AF786007F10C07BD4680BC704700BFFF
:10D2E80080B483B000AF786007F10C07BD4680BCFE
:10D2F800704700BF80B483B000AF78604DF2182348
:10D30800C2F200031A687B681A434DF21823C2F26E
:10D3180000031A604FF00003184607F10C07BD46DA
:10D3280080BC704780B400AF4DF21823C2F20003EE
:10D338004FF000021A604FF000031846BD4680BC4B
:10D34800704700BF80B400AF4DF21823C2F200034B
:10D358001B68002B0CBF00230123DBB21846BD4617
:10D3680080BC704780B400AF4DF21823C2F20003AE
:10D378001B681846BD4680BC704700BF80B582B0A8
:10D3880000AF786039603B68002B00F044827B680E
:10D3980040F63602934200F0408140F6360293424E
:10D3A80059DC40F2DE52934200F0C98040F2DE526E
:10D3B800934226DCB3F58A6F00F00381B3F58A6FD8
:10D3C8000FDC40F24E42934200F0E58040F24E42BC
:10D3D800934200F3EB8040F24D42934200F0D0803C
:10D3E80096E040F25242934200F0018140F25242EC
:10D3F8009342C0F2F18040F2DD52934200F09480F3
:10D4080086E040F26E72934200F0548140F26E72F0
:10D4180093420DDCB3F5BC6F00F0A780B3F5BC6F89
:10D42800C0F2988040F26D72934200F038816FE04C
:10D43800B3F5EE6F00F05481B3F5EE6FC0F245819D
:10D4480040F27172934200F0568140F635029342E1
:10D4580000F0D8805CE0B3F5106F00F07881B3F588
:10D46800106F2DDC40F63A02934200F0028140F63C
:10D478003A0293420ADC40F63802934200F0E38015
:10D4880040F63802934200F3E980D1E040F6FD020D
:10D49800934200F03B8140F6FD02934205DC40F6E2
:10D4A8003B02934200F0F08032E040F6FE029342E5
:10D4B80000F0378140F6FF02934200F03D8127E0FB
:10D4C80040F60412934200F06E8140F60412934233
:10D4D8000ADC40F60212934200F04F8140F6021235
:10D4E800934200F355813DE140F60612934200F065
:10D4F800708140F606129342C0F2608140F607122E
:10D50800934200F0718140F60812934200F077814F
:10D51800386847F2D021C0F605017A6841F2A113B4
:10D52800C0F60403984777E1386847F2EC21C0F663
:10D53800050141F2A113C0F6040398476CE138686D
:10D5480047F20431C0F6050141F2A113C0F6040305
:10D55800984761E1386847F21C31C0F6050141F28D
:10D56800A113C0F60403984756E1386847F23431EE
:10D57800C0F6050141F2A113C0F6040398474BE138
:10D58800386847F24831C0F6050141F2A113C0F6E8
:10D598000403984740E1386847F26431C0F6050152
:10D5A80041F2A113C0F60403984735E1386847F201
:10D5B8009431C0F6050141F2A113C0F6040398475F
:10D5C8002AE1386847F2B431C0F6050141F2A113E7
:10D5D800C0F6040398471FE1386847F2D031C0F617
:10D5E800050141F2A113C0F60403984714E1386815
:10D5F80047F2EC31C0F6050141F2A113C0F604036D
:10D60800984709E1386847F20441C0F6050141F23C
:10D61800A113C0F604039847FEE0386847F220419A
:10D62800C0F6050141F2A113C0F604039847F3E0E0
:10D63800386847F25041C0F6050141F2A113C0F61F
:10D6480004039847E8E0386847F27041C0F60501DE
:10D6580041F2A113C0F604039847DDE0386847F2A9
:10D668008C41C0F6050141F2A113C0F604039847A6
:10D67800D2E0386847F2A841C0F6050141F2A1138B
:10D68800C0F604039847C7E0386847F2C041C0F6BF
:10D69800050141F2A113C0F604039847BCE03868BD
:10D6A80047F2E841C0F6050141F2A113C0F60403B0
:10D6B8009847B1E0386847F22051C0F6050141F2B9
:10D6C800A113C0F604039847A6E0386847F25451FE
:10D6D800C0F6050141F2A113C0F6040398479BE088
:10D6E800386847F2A451C0F6050141F2A113C0F60B
:10D6F8000403984790E0386847F2E851C0F60501FE
:10D7080041F2A113C0F60403984785E0386847F250
:10D718001461C0F6050141F2A113C0F6040398474D
:10D728007AE0386847F24061C0F6050141F2A1137A
:10D73800C0F6040398476FE0386847F25461C0F6B2
:10D74800050141F2A113C0F60403984764E0386864
:10D7580047F26C61C0F6050141F2A113C0F604035B
:10D76800984759E0386847F29061C0F6050141F2E0
:10D77800A113C0F6040398474EE0386847F2B06139
:10D78800C0F6050141F2A113C0F60403984743E02F
:10D79800386847F2D061C0F6050141F2A113C0F61E
:10D7A8000403984738E0386847F2E461C0F6050199
:10D7B80041F2A113C0F6040398472DE0386847F2F8
:10D7C800F861C0F6050141F2A113C0F604039847B9
:10D7D80022E0386847F21471C0F6050141F2A1133E
:10D7E800C0F60403984717E0386847F23471C0F66A
:10D7F800050141F2A113C0F6040398470CE038680C
:10D8080047F25471C0F6050141F2A113C0F60403B2
:10D81800984700BF00E000BF07F10807BD4680BD7C
:10D8280080B582B000AF4DF23C20C2F200004FF04C
:10D8380000014FF4257246F20903C0F60103984728
:10D848004FF000037B604DF23C23C2F200034FF01F
:10D858000002C3F840224DF23C23C2F200034FF00D
:10D86800FF32C3F83C224DF23C23C2F200034FF0D2
:10D8780000025A604DF23C23C2F200034FF0FF321F
:10D88800C3F828224DF23C23C2F200034FF0FF32C6
:10D89800C3F82C224DF23C23C2F200034FF0FF02E2
:10D8A80083F86F224DF23C23C2F200034FF0FF02CF
:10D8B80083F870224DF23C23C2F200034FF0FF02BE
:10D8C80083F871224DF23C23C2F200034FF0FF02AD
:10D8D80083F872224DF23C23C2F200034FF0FF029C
:10D8E80083F873224DF23C23C2F200034FF0FF028B
:10D8F80083F874224DF23C23C2F200034FF0FF027A
:10D9080083F879224DF23C23C2F200034FF0FF0264
:10D9180083F86E2241F2F143C0F60203984738605B
:10D928003B6803F1FF33052B0ED801A252F823F010
:10D9380051D9010851D9010851D9010851D9010813
:10D9480051D9010851D9010800BF4FF2E873C1F657
:10D95800FF731A684DF23C23C2F20003C3F8502249
:10D968004FF2EC73C1F6FF731A684DF23C23C2F212
:10D978000003C3F854224FF2F073C1F6FF731A681C
:10D988004DF23C23C2F20003C3F858224CF635632B
:10D99800C0F6010398474BF24933C0F60203984793
:10D9A80046F25D23C0F602039847584845F67103CE
:10D9B800C0F602039847564845F6C533C0F6020339
:10D9C800984740F6FD43C0F60203984778607B68A5
:10D9D800002B40F08E804EF69133C0F60103984735
:10D9E80041F2F143C0F60203984702464DF23C2348
:10D9F800C2F200031A6041F20553C0F602039847C9
:10DA080042F29D50C0F6030048F2E143C0F602031B
:10DA1800984740484FF63D13C0F6030398474DF228
:10DA28003C23C2F200039B89B3F5FC6F30D94DF259
:10DA38003C23C2F200039B7B002B29D04DF23C23F0
:10DA4800C2F200039B7B0C2B22D84DF23C23C2F27E
:10DA58000003DB7B002B1BD04DF23C23C2F20003FA
:10DA6800DB7B1F2B14D84DF23C23C2F200031B7C36
:10DA7800172B0DD84DF23C23C2F200035B7C3B2BE5
:10DA880006D84DF23C23C2F200039B7C3B2B31D9D4
:10DA98004DF23C23C2F2000340F2E1729A814DF24A
:10DAA8003C23C2F200034FF001029A734DF23C236B
:10DAB800C2F200034FF00102DA734DF23C23C2F2C6
:10DAC80000034FF000021A744DF23C23C2F2000327
:10DAD8004FF000025A744DF23C23C2F200034FF09B
:10DAE80000029A740B484FF63503C0F603039847B3
:10DAF80000E000BF78684DF6BD53C0F601039847B3
:10DB08007B68184607F10807BD4680BD4CD3002046
:10DB180054D2002048D2002090B589B004AF41F219
:10DB28001523C0F603039847B86041F25123C0F6A5
:10DB380003039847B8604FF00003FB604FF6791372
:10DB4800C0F6020398474FF0000300934FF000031C
:10DB580001934FF0000302934FF0000303934FF635
:10DB6800E510C0F601004FF000014FF4FA724FF0D3
:10DB7800000347F22D24C0F60404A04778607B68B0
:10DB8800012B03D040F2DD53FB60B3E04FF00003FC
:10DB980000934FF0000301934FF0000302934FF0FE
:10DBA800000303934FF67D60C0F601004FF00001BB
:10DBB8004FF4FA724FF0000347F22D24C0F6040424
:10DBC800A04778607B68012B03D040F2DF53FB60ED
:10DBD80090E04FF0000300934FF0000301934FF0E3
:10DBE800000302934FF0000303934FF62150C0F651
:10DBF80001004FF000014FF4FA724FF0000347F2B2
:10DC08002D24C0F60404A04778607B68012B03D05C
:10DC180040F2E153FB606DE04FF0000300934FF0DA
:10DC2800000301934FF0000302934FF000030393A6
:10DC38004FF68D40C0F601004FF000014FF4FA7224
:10DC48004FF0000347F22D24C0F60404A047786083
:10DC58007B68012B03D04FF4BC63FB604AE04FF0B4
:10DC6800000300934FF0000301934FF00003029369
:10DC78004FF0000303934FF66170C0F601004FF0B8
:10DC880000014FF4FA724FF0000347F22D24C0F65A
:10DC98000404A04778607B68012B03D040F2E4536A
:10DCA800FB6027E04FF0000300934FF0000301935F
:10DCB8004FF0000302934FF0000303934FF6A9704F
:10DCC800C0F601004FF000014FF4FA724FF0000364
:10DCD80047F22D24C0F60404A04778607B68012B26
:10DCE80003D040F2E253FB6004E041F2B953C0F6BE
:10DCF80001039847F8684DF6BD53C0F601039847ED
:10DD0800FB68184607F11407BD4690BD80B582B080
:10DD180000AF78607B68002B10DD4DF23C23C2F227
:10DD280000034FF0FF32C3F840224DF23C23C2F209
:10DD380000037A68C3F83C2200BF07E04FF00500F3
:10DD480041F21143C0F602039847FEE707F10807BE
:10DD5800BD4680BD80B582B000AF78604DF23C23EF
:10DD6800C2F20003D3F84032002B1DD04DF23C2301
:10DD7800C2F20003D3F83C227B68D21A4DF23C234E
:10DD8800C2F20003C3F83C224DF23C23C2F2000366
:10DD9800D3F83C32002B08DC4FF000004DF6155349
:10DDA800C0F60103984700E000BF07F10807BD4629
:10DDB80080BD00BF80B582B000AF78604DF23C23D3
:10DDC800C2F200037A685A607B68002B05D142F6DC
:10DDD800C553C0F60203984704E042F69553C0F6CF
:10DDE8000203984707F10807BD4680BD80B483B099
:10DDF80000AF78604DF23C23C2F200035B6818461E
:10DE080007F10C07BD4680BC704700BF80B483B0E3
:10DE180000AF78604DF23C23C2F200037A689A6042
:10DE280007F10C07BD4680BC704700BF80B400AF47
:10DE38004DF23C23C2F200039B681846BD4680BCE5
:10DE4800704700BF80B400AF4DF23C23C2F200031C
:10DE58001B681846BD4680BC704700BF80B584B0BB
:10DE680000AF07F1040318464FF63D13C0F603034D
:10DE7800984707F10403184609494FF63543C0F699
:10DE880003039847F8604DF23C23C2F200035B6934
:10DE9800FA68D31A184607F11007BD4680BD00BFBF
:10DEA80048D2002090B585B000AF786007F108032C
:10DEB80018464FF63D13C0F6030398474DF23C232E
:10DEC800C2F200035C6907F10803786819464FF647
:10DED8003543C0F6030398470346E2184DF23C2346
:10DEE800C2F200035A6107F11407BD4690BD00BF96
:10DEF80090B583B000AF03463960FB71FB790E48DB
:10DF080019464FF003023B6845F6A904C0F602041F
:10DF1800A047FA794DF23C23C2F20003C3F8282245
:10DF28004DF23C23C2F200033A68C3F82C2207F1F1
:10DF38000C07BD4690BD00BF4CD3002090B585B0FE
:10DF480000AF03463960FB714DF23C23C2F2000377
:10DF5800D3F82822FB799A4209D14DF23C23C2F228
:10DF68000003D3F82C223B689A4200F05B814FF003
:10DF78000003FB60FB79292B2FD14DF23C23C2F221
:10DF8800000393F87232002B03D03B68002B00F09B
:10DF98004B814DF23C23C2F2000393F87232002BFE
:10DFA80003D13B68002B40F041813B68002B14BF34
:10DFB80000230123DBB21A464DF23C23C2F20003D0
:10DFC80083F872224DF23C23C2F2000393F87232B6
:10DFD800002B02D04FF00203FB60FB79362B2FD1C8
:10DFE8004DF23C23C2F2000393F87132002B03D0A8
:10DFF8003B68002B00F01C814DF23C23C2F2000369
:10E0080093F87132002B03D13B68002B40F012814A
:10E018003B68002B14BF00230123DBB21A464DF2E4
:10E028003C23C2F2000383F871224DF23C23C2F272
:10E03800000393F87132002B02D04FF00203FB600B
:10E04800FB790C2B2FD14DF23C23C2F2000393F83D
:10E058007032002B03D03B68002B00F0ED804DF2AE
:10E068003C23C2F2000393F87032002B03D13B68C3
:10E07800002B40F0E3803B68002B14BF00230123F2
:10E08800DBB21A464DF23C23C2F2000383F8702239
:10E098004DF23C23C2F2000393F87032002B02D0F9
:10E0A8004FF00203FB60FB794A2B2FD14DF23C2342
:10E0B800C2F2000393F86F32002B03D03B68002BA9
:10E0C80000F0BE804DF23C23C2F2000393F86F3299
:10E0D800002B03D13B68002B40F0B4803B68002B39
:10E0E80014BF00230123DBB21A464DF23C23C2F2CF
:10E0F800000383F86F224DF23C23C2F2000393F829
:10E108006F32002B02D04FF00203FB60FB79092B22
:10E118002FD14DF23C23C2F2000393F87932002B41
:10E1280003D03B68002B00F08F804DF23C23C2F2F5
:10E13800000393F87932002B03D13B68002B40F0A1
:10E1480085803B68002B14BF00230123DBB21A46ED
:10E158004DF23C23C2F2000383F879224DF23C23AE
:10E16800C2F2000393F87932002B02D04FF0020379
:10E17800FB60FB794D2B1CD14DF23C23C2F200030E
:10E1880093F878321A463B689A4261D03B68DAB213
:10E198004DF23C23C2F2000383F878224DF23C236F
:10E1A800C2F2000393F87832002B02D14FF0020339
:10E1B800FB60FB79492B1AD14DF23C23C2F20003D4
:10E1C800D3F87C223B689A4244D04DF23C23C2F2F9
:10E1D80000033A68C3F87C224DF23C23C2F20003E4
:10E1E800D3F87C32002B02D14FF00203FB60FB68AE
:10E1F800DBB2FA791A4811461A463B6845F6A90473
:10E20800C0F60204A047FA794DF23C23C2F200039B
:10E21800C3F828224DF23C23C2F200033A68C3F83F
:10E228002C2218E000BF16E000BF14E000BF12E087
:10E2380000BF10E000BF0EE000BF0CE000BF0AE026
:10E2480000BF08E000BF06E000BF04E000BF02E036
:10E2580000BF00E000BF07F11407BD4690BD00BF36
:10E268004CD3002090B585B000AF03463960FB71F0
:10E278004DF23C23C2F20003D3F82822FB799A42DC
:10E2880009D14DF23C23C2F20003D3F82C223B689B
:10E298009A4200F0BD804FF00103FB60FB79432BED
:10E2A80033D14DF23C23C2F2000393F87332002BB2
:10E2B80007D13B68002B00F0AD803B68632B00F072
:10E2C800A9803B68002B03DD3B68622B40F3A480E8
:10E2D8003B68002B05DD3B68622B02DC4FF0010335
:10E2E80001E04FF00003DAB24DF23C23C2F2000322
:10E2F80083F873224DF23C23C2F2000393F8733281
:10E30800002B02D04FF00203FB60FB793F2B1CD19E
:10E318004DF23C23C2F2000393F875321A463B686B
:10E328009A427BD03B68DAB24DF23C23C2F200033A
:10E3380083F875224DF23C23C2F2000393F875323C
:10E34800002B02D14FF00203FB60FB793D2B24D157
:10E358004DF23C23C2F2000393F876321A463B682A
:10E368009A425DD03B68DAB24DF23C23C2F2000318
:10E3780083F876224DF23C23C2F2000393F87632FA
:10E38800022B07D04DF23C23C2F2000393F87632F9
:10E39800052B02D14FF00203FB60FB793B2B1CD10C
:10E3A8004DF23C23C2F2000393F877321A463B68D9
:10E3B8009A4237D03B68DAB24DF23C23C2F20003EE
:10E3C80083F877224DF23C23C2F2000393F87732A8
:10E3D800012B02D14FF00203FB60FB68DBB2FA7934
:10E3E800134811461A463B6845F6A904C0F60204CC
:10E3F800A047FA794DF23C23C2F20003C3F8282261
:10E408004DF23C23C2F200033A68C3F82C220AE01A
:10E4180000BF08E000BF06E000BF04E000BF02E064
:10E4280000BF00E000BF07F11407BD4690BD00BF64
:10E438004CD3002090B583B000AF03463960FB7120
:10E448004DF23C23C2F20003D3F82822FB799A420A
:10E4580008D14DF23C23C2F20003D3F82C223B68CA
:10E468009A422ED0FB79332B11D14DF23C23C2F2C4
:10E47800000393F86E321A463B689A4223D03B68F1
:10E48800DAB24DF23C23C2F2000383F86E22FB7924
:10E498000F4819464FF002023B6845F6A904C0F63A
:10E4A8000204A047FA794DF23C23C2F20003C3F8F4
:10E4B80028224DF23C23C2F200033A68C3F82C220A
:10E4C80002E000BF00E000BF07F10C07BD4690BDA9
:10E4D8004CD3002090B587B002AFF8607A603B60FB
:10E4E8000B46FB72FB7A3A6800920648F9681A46AE
:10E4F8007B6845F63544C0F60204A04707F11407C7
:10E50800BD4690BD54D2002080B483B000AF78607F
:10E518007B68002B02DB7B68042B02DD4FF00003D5
:10E5280008E04DF23C23C2F200037A689B1803F519
:10E53800A073DB79184607F10C07BD4680BC70470D
:10E5480090B58BB002AFF860B9607A603B60F8684C
:10E558004BF2A543C0F602039847B8614CF6E9634D
:10E56800C0F6010398470346D3F8EE30FB61FA6919
:10E5780040F2E7339A4202DC4FF47A73FB61B869E0
:10E58800F9694BF6E143C0F60203984778617B6965
:10E59800002B01D07B6951E0FB68002B1BD140F6B2
:10E5A800F433C2F200031A68BB689A420DD04CF6E5
:10E5B800E963C0F6010398470346D3F82E3018469E
:10E5C80047F20D33C0F60403984740F6F433C2F21D
:10E5D8000003BA681A60BB68DBB23A6B00927A6BC8
:10E5E8000192B86919467A683B684BF6C504C0F6CB
:10E5F8000204A0474DF23C23C2F20003FA689B18BC
:10E6080003F5A0734FF00102DA71B8694BF62913CC
:10E61800C0F60203984778614DF23C23C2F200032A
:10E62800FA689B1803F5A0734FF00002DA71B86915
:10E638004BF66153C0F6020398477B69184607F109
:10E648002407BD4690BD00BF80B588B000AFF86014
:10E65800B9607A603B60F8684BF2A543C0F60203E4
:10E668009847B8614CF6E963C0F60103984703463A
:10E67800D3F8EE30FB61FA6940F2E7339A4202DCE4
:10E688004FF47A73FB61B869F9694BF6E143C0F658
:10E698000203984778617B69002B01D07B6950E0C1
:10E6A800FB68002B1FD1BB681B781A4640F6F43371
:10E6B800C2F200031B689A420DD04CF6E963C0F61B
:10E6C800010398470346D3F82E30184647F20D3316
:10E6D800C0F604039847BB681B781A4640F6F43323
:10E6E800C2F200031A60B869B9687A684BF67D13FC
:10E6F800C0F6020398474DF23C23C2F20003FA68C1
:10E708009B1803F5A0734FF00102DA71B8693968F4
:10E71800BA6A4BF60523C0F60203984778614DF2B2
:10E728003C23C2F20003FA689B1803F5A0734FF06C
:10E738000002DA71B8694BF66153C0F602039847D4
:10E748007B69184607F12007BD4680BD80B588B0B3
:10E7580000AFF860B9607A6042F68573C0F60203CC
:10E768009847F86122E042F68573C0F6020398479D
:10E77800B861BA69FB69D21A13464FEA83039B183A
:10E788004FEA43037B617A687B699A4202D24FF46D
:10E79800627313E041F23143C0F6020398474FF029
:10E7A8000A0047F20D33C0F604039847FB681B784C
:10E7B8001A46BB689A42D6D14FF00003184607F1B3
:10E7C8002007BD4680BD00BF80B400AF4DF23C239A
:10E7D800C2F20003B3F830321846BD4680BC704719
:10E7E80080B400AF4DF23C23C2F20003B3F83232DA
:10E7F8001846BD4680BC704780B400AF4DF23C233C
:10E80800C2F20003B3F834321846BD4680BC7047E4
:10E8180080B400AF4DF23C23C2F20003B3F83632A5
:10E828001846BD4680BC704780B400AF4DF23C230B
:10E83800C2F20003B3F838321846BD4680BC7047B0
:10E8480080B400AF4DF23C23C2F20003B3F83A3271
:10E858001846BD4680BC704780B400AF4DF23C23DB
:10E86800C2F20003B3F8343203F101039AB24DF255
:10E878003C23C2F20003A3F83422BD4680BC704793
:10E8880080B400AF4DF23C23C2F20003B3F8363235
:10E8980003F101039AB24DF23C23C2F20003A3F83C
:10E8A8003622BD4680BC704780B400AF4DF23C2391
:10E8B800C2F20003B3F8383203F101039AB24DF201
:10E8C8003C23C2F20003A3F83822BD4680BC70473F
:10E8D80080B400AF4DF23C23C2F20003B3F83A32E1
:10E8E80003F101039AB24DF23C23C2F20003A3F8EC
:10E8F8003A22BD4680BC704780B483B000AF03465F
:10E90800FB804DF23C23C2F20003FA88A3F83422BC
:10E9180007F10C07BD4680BC704700BF80B483B0C8
:10E9280000AF0346FB804DF23C23C2F20003FA8895
:10E93800A3F8362207F10C07BD4680BC704700BF1C
:10E9480080B483B000AF0346FB804DF23C23C2F293
:10E958000003FA88A3F8382207F10C07BD4680BCEB
:10E96800704700BF80B483B000AF0346FB804DF210
:10E978003C23C2F20003FA88A3F83A2207F10C07F5
:10E98800BD4680BC704700BF80B400AF4DF23C2349
:10E99800C2F20003B3F8303203F101039AB24DF228
:10E9A8003C23C2F20003A3F83022BD4680BC704766
:10E9B80080B400AF4DF23C23C2F20003B3F8323208
:10E9C80003F101039AB24DF23C23C2F20003A3F80B
:10E9D8003222BD4680BC704780B483B000AF034686
:10E9E800FB804DF23C23C2F20003FA88A3F83022E0
:10E9F80007F10C07BD4680BC704700BF80B483B0E8
:10EA080000AF0346FB804DF23C23C2F20003FA88B4
:10EA1800A3F8322207F10C07BD4680BC704700BF3F
:10EA280080B582B000AF4CF6E963C0F601039847A1
:10EA38000346B3F927309BB21AB213464FEA0313C1
:10EA48009B1A4FEA830318464FF0000143F265739F
:10EA5800C0F60203984778600548796840F2E143B8
:10EA6800C0F60403984707F10807BD4680BD00BFFC
:10EA780080D4002080B500AF044840F21953C0F696
:10EA8800040398470346184680BD00BF80D4002081
:10EA980080B483B000AF78604DF23C23C2F200032B
:10EAA800D3F850227B681A607B6803F104024DF2A8
:10EAB8003C23C2F20003D3F8543213607B6803F19D
:10EAC80008024DF23C23C2F20003D3F85832136017
:10EAD80007F10C07BD4680BC704700BF80B483B007
:10EAE80000AF78604DF23422C2F2000247F2787328
:10EAF800C0F6050393E8030082E803007B68002B57
:10EB08000BD14DF23422C2F2000247F28073C0F6F4
:10EB1800050393E8030082E803007B68012B0BD10F
:10EB28004DF23422C2F2000247F28873C0F60503A0
:10EB380093E8030082E803007B68022B0BD14DF2B7
:10EB48003422C2F2000247F29073C0F6050393E83C
:10EB5800030082E803007B68032B0BD14DF23422BB
:10EB6800C2F2000247F29873C0F6050393E8030067
:10EB780082E803004DF23423C2F20003184607F17D
:10EB88000C07BD4680BC704780B5BEB000AF46F6E6
:10EB98005123C0F602039847C7F8F4006AE041F22F
:10EBA8003143C0F602039847D7F8F43003F1FF3336
:10EBB800C7F8F43007F10403D7F8F400194646F60D
:10EBC8002153C0F6020398474FF00003C7F8E4301A
:10EBD8004FF00003C7F8F03034E0D7F8F0004BF6F8
:10EBE800F173C0F601039847C7F8DC004FF0000343
:10EBF800C7F8EC3018E0D7F8DC30D7F8EC2002F191
:10EC0800980233F812309BB21A46BB881BB29A425C
:10EC180004D14FF00103C7F8E43009E0D7F8EC302D
:10EC280003F10103C7F8EC30D7F8EC30062BE2DD2E
:10EC3800D7F8E430002B10D1D7F8F03003F10103F6
:10EC4800C7F8F0304BF65D33C0F60103984702462B
:10EC5800D7F8F0309A42C0DC00E000BFD7F8E430C3
:10EC6800002B07D1BB881BB2184646F6B133C0F655
:10EC780002039847D7F8F430002B90DC46F605637A
:10EC8800C0F602039847C7F8F40051E041F2314357
:10EC9800C0F602039847D7F8F43003F1FF33C7F8FA
:10ECA800F43007F10403D7F8F400194647F281233A
:10ECB800C0F6020398474FF00003C7F8E4304FF05E
:10ECC8000003C7F8F0301DE0D7F8F0004BF6F173F9
:10ECD800C0F601039847C7F8D800D7F8D830B3F979
:10ECE80000309BB21AB2D7F806309A4204D14FF0DE
:10ECF8000103C7F8E4300FE0D7F8F03003F101035F
:10ED0800C7F8F0304BF65D33C0F60103984702466A
:10ED1800D7F8F0309A42D7DCD7F8E430002B07D187
:10ED2800BB881BB2184647F24103C0F60203984756
:10ED3800D7F8F430002BA9DC46F60563C0F60203C9
:10ED48009847C7F8F4004FF00003C7F8F03010E117
:10ED580041F23143C0F602039847D7F8F0004BF66A
:10ED6800F173C0F601039847C7F8D4004FF00003C9
:10ED7800C7F8E0304FF00003C7F8EC30E3E0D7F80D
:10ED8800D430D7F8EC2002F1980233F812309AB256
:10ED98004FF6FF739A424CD04FF00003C7F8E430A7
:10EDA8004FF00003C7F8F43021E007F10403D7F867
:10EDB800F400194646F62153C0F602039847BB886B
:10EDC8001AB2D7F8D430D7F8EC1001F1980133F81B
:10EDD80011309BB29A4204D14FF00103C7F8E430D6
:10EDE8000FE0D7F8F43003F10103C7F8F43046F622
:10EDF8005123C0F6020398470246D7F8F4309A42E6
:10EE0800D3DCD7F8E430002B13D1D7F8D420D7F8C7
:10EE1800EC3003F198034FF0FF3102F813104FEA7A
:10EE28004303D3184FF0FF325A704FF00103C7F86D
:10EE3800E0304FF00003C7F8E8307AE0D7F8D41094
:10EE4800D7F8EC2013464FEA83039B18D7F8E8203D
:10EE58009B1803F174034FEA4303CB185B889AB2FB
:10EE68004FF6FF739A425ED04FF00003C7F8E430C4
:10EE78004FF00003C7F8F4302AE007F10403D7F88D
:10EE8800F400194646F2E563C0F602039847BB88CA
:10EE980019B2D7F8D400D7F8EC2013464FEA830309
:10EEA8009B18D7F8E8209B1803F174034FEA430333
:10EEB800C3185B889BB2994204D14FF00103C7F88D
:10EEC800E4300FE0D7F8F43003F10103C7F8F43069
:10EED80046F20543C0F6020398470246D7F8F430D5
:10EEE8009A42CADCD7F8E430002B1CD1D7F8D420DA
:10EEF800D7F8EC100B464FEA83035B18D7F8E810F5
:10EF08005B1803F174014FEA4103D3184FF0FF3047
:10EF180098704FEA4103D3184FF0FF32DA704FF080
:10EF28000103C7F8E030D7F8E83003F10103C7F868
:10EF3800E830D7F8E830042B80DDD7F8EC3003F15F
:10EF48000103C7F8EC30D7F8EC30062B7FF717AF82
:10EF5800D7F8E030002B06D0D7F8F0004BF2D133C9
:10EF6800C0F601039847D7F8F03003F10103C7F85A
:10EF7800F0304BF65D33C0F6010398470246D7F8E8
:10EF8800F0309A423FF7E4AE4FF480304DF2D503AB
:10EF9800C0F601039847C7F8D00007F1F807BD4647
:10EFA80080BD00BF80B582B000AF78607A6840F25B
:10EFB80003339A4210D14DF2F043C2F2000303F535
:10EFC8001D5303F11C034FF007021A6042F6355334
:10EFD800C0F6020398479CE07B68B3F5407F1AD1DE
:10EFE80042F66553C0F60203984742F6C553C0F689
:10EFF8000203984742F62563C0F6020398474DF28C
:10F00800F043C2F2000303F51D5303F11C034FF054
:10F0180000021A607DE07A6845F6F7239A4211D11A
:10F028004DF21C20C2F200004FF00A0140F2E14309
:10F03800C0F60403984740F6F833C2F200034FF0D5
:10F0480000021A607A6844F6A1439A421FD140F63A
:10F05800F833C2F200031B68002B57D14DF21C2075
:10F06800C2F2000040F21953C0F604039847034661
:10F07800002B07D040F6F833C2F200034FF001022C
:10F088001A6046E04FF22513C0F6010398477A68E4
:10F0980045F6F8239A4211D14DF22820C2F2000019
:10F0A8004FF00A0140F2E143C0F60403984740F6E6
:10F0B800FC33C2F200034FF000021A607A6844F68B
:10F0C800A2439A4225D140F6FC33C2F200031B68E2
:10F0D800002B1DD14DF22820C2F2000040F2195336
:10F0E800C0F6040398470346002B07D040F6FC33CC
:10F0F800C2F200034FF001021A600AE04FF000006C
:10F108004DF29943C0F60303984702E000BF00E0C0
:10F1180000BF07F10807BD4680BD00BF80B400AF3F
:10F128004DF23C23C2F200034FF0010283F8812222
:10F13800BD4680BC704700BF80B400AF4DF23C2391
:10F14800C2F2000393F881321846BD4680BC70476E
:10F1580080B400AF40F63063C2F200034FF0010202
:10F168001A60BD4680BC704780B400AF40F630637B
:10F17800C2F200031B681846BD4680BC704700BF3A
:10F1880090B5ADB004AF4FF00003C7F898304AF619
:10F198002143C0F601039847C7F89400D7F8943084
:10F1A800002B40F3488240F60043C2F200031B687C
:10F1B80003F1010240F60043C2F200031A6040F670
:10F1C8000043C2F200031A68D7F894309A4206DB6B
:10F1D80040F60043C2F200034FF000021A6040F606
:10F1E8000043C2F200031A6807F1180310461946D3
:10F1F8004BF2D503C0F601039847C7F89800D7F833
:10F208009830002B40F0178207F1180318464BF28C
:10F218008513C0F60103984797F83A30002B00F0A1
:10F228000A8297F83B30022B40F08C8007F11803D4
:10F2380018464FF25163C0F6010398470346002B66
:10F2480000F0F98107F1100318464FF63D13C0F698
:10F258000303984707F1100207F1180303F15C0351
:10F26800104619464FF63543C0F603039847C7F8CA
:10F278009000B7F8742040F2CF739A4213D9BB8F2D
:10F288001AB213464FEA03139B1A4FEA83031A462E
:10F29800B7F941309BB21BB2D31803F10102D7F87A
:10F2A80090309A421FDA07F1180318464FF2257377
:10F2B800C0F60103984707F1180303F15C031846E9
:10F2C8004FF63D13C0F60303984740F60043C2F2D9
:10F2D80000031A6807F11803104619464AF69563A1
:10F2E800C0F60103984707F1180303F150031846C5
:10F2F80040F21953C0F6040398470346002B00F068
:10F308009A8107F1180303F15C0318464FF63D1381
:10F31800C0F60303984707F1180318464FF2257300
:10F32800C0F60103984740F60043C2F200031A688A
:10F3380007F11803104619464AF69563C0F601030B
:10F34800984727E197F83B30012B40F02381FB8F4A
:10F358001BB218464BF68D73C0F601039847C7F8E1
:10F368008C00D7F88C30002B00F065814FF000033B
:10F37800C7F89C3097F84030012B09D1D7F88C306A
:10F3880093F87331062B03D14FF00103C7F89C3073
:10F3980097F84030022B09D1D7F88C3093F87331A5
:10F3A800072B03D14FF00103C7F89C3097F8403082
:10F3B800032B09D1D7F88C3093F87331052B03D17F
:10F3C8004FF00103C7F89C3097F84030042B09D15F
:10F3D800D7F88C3093F87331042B03D14FF0010325
:10F3E800C7F89C3097F84030052B09D1D7F88C30F6
:10F3F80093F87331032B03D14FF00103C7F89C3006
:10F4080097F84030062B09D1D7F88C3093F8733130
:10F41800022B03D14FF00103C7F89C3097F8403016
:10F42800072B09D1D7F88C3093F87331012B03D10E
:10F438004FF00103C7F89C30D7F89C30002B00F040
:10F44800FA8097F87B30002B30D0FA6F4AF2C54328
:10F45800C0F60103104698470146D7F88C30D3F818
:10F46800662113461A464AF25933C0F60103084684
:10F4780011469847034623F00043C7F8883049F6F9
:10F488004543C0F60103D7F88800984702460B4663
:10F498004AF20D24C0F601041046194668A3D3E9C0
:10F4A8000023A0470346002B40F0C58007F118034E
:10F4B80018464FF25163C0F6010398470346002BE4
:10F4C80000F0B980B7F941309BB21BB2002B61DD67
:10F4D800B7F861309AB240F2CF739A4218D807F160
:10F4E800180303F1490318464FF63D13C0F603030A
:10F4F800984740F60043C2F200031A6807F1180360
:10F50800104619464AF69563C0F60103984792E0FB
:10F5180007F1080318464FF63D13C0F60303984752
:10F5280007F1080207F1180303F1490310461946C9
:10F538004FF63543C0F603039847C7F88400B7F978
:10F5480041309BB21AB2D7F884309A4273DCB7F8CC
:10F5580061309AB240F2CF739A421BD907F118036F
:10F5680003F1490318464FF000014FF0070246F235
:10F578000903C0F60103984740F60043C2F20003AE
:10F588001A6807F11803104619464AF69563C0F63B
:10F598000103984797F843404CF6E963C0F6010326
:10F5A8009847034693F820309C4231D04FF001032E
:10F5B800C7F8803097F84330786C07F104013A4671
:10F5C8000090D7F88000019007F1180000F1300092
:10F5D80002904DF2D040C2F200004AF2F164C0F647
:10F5E8000204A0477B683A4600924FF000004DF2B3
:10F5F800D041C2F200011A464DF2E043C2F20003C4
:10F608004EF25164C0F60104A047C7F8980012E012
:10F618007B6C1A46BB6C002B02D04FF47F4301E091
:10F628004FF00003104619464AF21113C0F60203C0
:10F638009847C7F8980007F1A407BD4690BD00BFDA
:10F648002D431CEBE2361A3F80B588B000AF7860D6
:10F6580007F10C0318464FF63D13C0F6030398470D
:10F668004FF00003BB814FF00003BB734FF0000362
:10F67800FB7307F10C0318464FF67533C0F6030306
:10F688009847F8617B684FF0000283F83B204FF001
:10F69800000283F83C207B684FF0000283F83D208D
:10F6A8007B684FF0000283F83E207B6803F13B0340
:10F6B80018464FF67533C0F603039847B8617B6860
:10F6C8004FF0000283F842204FF0000283F84320F5
:10F6D8007B684FF0000283F844207B684FF00002FB
:10F6E80083F845207B6803F1420318464FF67533CB
:10F6F800C0F6030398477861FA69BB699A4203DB4D
:10F70800FA697B699A4202DD4FF0000301E04FF08D
:10F718000103184607F12007BD4680BD80B588B0B3
:10F7280000AF78604FF00003BB617B6893F823302B
:10F73800022B58D107F1080318464FF63D13C0F6BF
:10F74800030398473B7B4FF4616202FB03F17B7B29
:10F758001A4613464FEA03139B1A4FEA8303CA1843
:10F76800BB7BD3187B617B6893F838304FF46162B8
:10F7780002FB03F17B6893F839301A4613464FEAC7
:10F7880003139B1A4FEA8303CA187B6893F83A302D
:10F79800D3183B617B68B3F929309BB21AB23B6935
:10F7A800D318FB610DE07B68B3F924309BB21AB221
:10F7B80013464FEA03139B1A4FEA8303FA69D318D7
:10F7C800FB61FA697B699A42EDDDFA697B69D31AB4
:10F7D800BB617B6803F150031846B96940F2E14305
:10F7E800C0F60403984707F12007BD4680BD00BF57
:10F7F80080B500AF044846F2C513C0F60203984727
:10F808000346184680BD00BF54D2002090B591B081
:10F8180002AFF860B9601346FB71F8684FF47A716B
:10F828004BF6E143C0F602039847B862BB6A002B67
:10F8380001D0BB6AC1E0FB684FF000021A61FB68A7
:10F848001968FB681B691A468A18F979117003F15F
:10F858000102FB681A6142F68573C0F602039847F5
:10F8680078624FF008037B634FF000033B635CE072
:10F8780042F68573C0F60203984738623A6A7B6A93
:10F88800D21A13464FEA83039B184FEA4303FB61DE
:10F89800FB69B3F57A7F00F288804FF00003FB75AF
:10F8A800BB689B6C07F1170210464FF001014FF03F
:10F8B80000029847B862BB6A002B07D04FF00A00D5
:10F8C80047F20D33C0F6040398472EE0FB68196829
:10F8D800FB681B691A468A18F97D117003F1010249
:10F8E800FB681A61FB681A697B6B9A421DD1FB6839
:10F8F8001B6803F101031B78A3F10F03012B03D944
:10F908004FF001033B6310E0FB681B69082B08D12B
:10F91800FB681B6803F106031B7803F109037B638B
:10F9280002E04FF001033B6300BF3B6B002B9FD00D
:10F938004FF00003FB6203E0FB6A03F10103FB6283
:10F94800FB681A69FB6A9A42F6DCFB681968FB686F
:10F958001A69FB681B6807F1180000904FF0000057
:10F968004EF25164C0F60104A047B862BB6A002B8E
:10F978001AD14FF00003FB6203E0FB6A03F10103B5
:10F98800FB62BB69FA6A9A42F7DBBB68DB69984796
:10F99800BB689B699847BB68DB6CFA681168BA69F1
:10F9A80008461146984700E000BFF8684BF66153D7
:10F9B800C0F6020398474FF00003184607F13C07CA
:10F9C800BD4690BD80B400AF40F60443C2F20003C8
:10F9D8001B681846BD4680BC704700BF90B593B001
:10F9E80000AF78604FF000037B644FF00003BB6109
:10F9F80007F11803184640F2B113C0F604039847FC
:10FA08004FF000033B644FF00003FB6341F23143C6
:10FA1800C0F602039847FB6B002B0CD04FF259132A
:10FA2800C0F6010398474FF0640047F20D33C0F663
:10FA380004039847EAE74FF000037B6107F11403DA
:10FA4800184640F2B113C0F6040398477A69BB69B7
:10FA58009A420CD07B69BB617B6C03F101037B6428
:10FA68004FF001004DF65D53C0F6010398474FF281
:10FA78008913C0F6010398474FF24113C0F60103FA
:10FA880098470346002B1AD006E04FF0640047F26F
:10FA98000D33C0F6040398474CF6E963C0F601033A
:10FAA8009847034693F82930002BEED14FF6595367
:10FAB800C0F6020398474FF00103FB63A6E741F243
:10FAC800C953C0F6030398470346D3F815203B6C87
:10FAD800D31A7B637A6B41F288339A4210D941F288
:10FAE800C953C0F6030398470346D3F815303B645F
:10FAF8004FF000037B644FF65953C0F60203984752
:10FB08007B6CB3F5616F1DDD4CF6E963C0F601034C
:10FB18009847034693F82930002B13D07B6B002BB2
:10FB280010D041F2C953C0F6030398470346D3F8EF
:10FB380015303B644FF000037B644FF65953C0F611
:10FB4800020398474CF6E963C0F601039847034659
:10FB5800D3F8F630002B00F08C804CF6E963C0F641
:10FB6800010398470346D3F8FA303B633B6B1846CA
:10FB78004BF68D73C0F601039847F862FB6A002BB9
:10FB880077D0FB6AD3F85130BB6207F10C031846F3
:10FB98004FF63D13C0F60303984740F60443C2F2FC
:10FBA80000031B687B62FB6A03F5AA7307F10C026A
:10FBB800104619464FF63543C0F603039847386296
:10FBC800BA6A3B6AD41A4CF6E963C0F6010398474F
:10FBD8000346D3F8FE309C4207DC40F60443C2F2E9
:10FBE80000034FF001021A6011E04CF6E963C0F619
:10FBF800010398470346D3F802213B6A9A4206DC80
:10FC080040F60443C2F200034FF000021A6040F6C7
:10FC18000443C2F200031B687A6A9A4229D040F66C
:10FC28000443C2F200031B684FF0620019464EF20B
:10FC38003D43C0F6010398474FF00003BB6315E04E
:10FC4800BB6BFB61FB6903F10103FB6140F60443F5
:10FC5800C2F200031B68F869194642F27D13C0F628
:10FC680002039847BB6B03F10103BB63BB6B012B1A
:10FC7800E6DD4FF0640047F20D33C0F60403984701
:10FC8800C4E600BF80B586B000AF78604FF00200D0
:10FC98004BF2A543C0F602039847386141F6192391
:10FCA800C0F602039847F860FB68002B07D14FF4B1
:10FCB8007A7047F20D33C0F604039847F7E74FF020
:10FCC80000037B617B69022B0ED0FB689B69984718
:10FCD800FB68DB699847FB68DB6A4FF000009847D0
:10FCE8004FF002037B610FE0FB685B6B9847B860DD
:10FCF800BB68002B07DD3869F9684BF2CD43C0F6C5
:10FD08000203984700E000BF4FF00A0047F20D33A6
:10FD1800C0F604039847D5E780B58AB000AF78608D
:10FD28004FF001004BF2A543C0F602039847F86173
:10FD380041F64123C0F602039847B861BB69002B1E
:10FD480007D14FF47A7047F20D33C0F60403984791
:10FD5800F7E741F6B923C0F60203984778614FF0F8
:10FD680000037B624FF001004EF21153C0F601030D
:10FD780098470346002B02D04FF004037B627B6A4E
:10FD8800022B1BD0042B28D0BB699B699847BB6901
:10FD9800DB699847BB69DB6A4FF0000098477B69CD
:10FDA8009B6998477B69DB6998477B69DB6A4FF0F9
:10FDB800000098474FF002037B621AE0BB695B6B57
:10FDC800984738613B69002B12DDF869B9694BF235
:10FDD800CD43C0F6020398470BE0F869B9694BF6C2
:10FDE8008D23C0F6020398474FF000037B6200E0C2
:10FDF80000BF7B69002B35D04DF23C23C2F20003D3
:10FE080093F88032002B2DD04FF0320387F823303F
:10FE18004FF00003FB7214E07B699B6C07F10B0247
:10FE280010464FF001014FF000029847F860FB6858
:10FE3800002B16D1FB7A18464BF6D553C0F60203B1
:10FE4800984797F82330002B0CBF00230123DBB21F
:10FE580097F8232002F1FF3287F82320002BDBD10B
:10FE680000E000BF4FF0640047F20D33C0F6040312
:10FE7800984777E780B588B000AF78604FF000000A
:10FE88004BF2A543C0F602039847B86141F66923CF
:10FE9800C0F60203984778617B69002B07D14FF4BD
:10FEA8007A7047F20D33C0F604039847F7E74FF02E
:10FEB8000003FB614FF000004EF21153C0F601033E
:10FEC80098470346002B02D04FF00403FB61FB69FF
:10FED800022B1DD0042B2AD0B8694BF6C143C0F6BB
:10FEE8000203984738617B699B6998477B69DB699E
:10FEF80098477B69DB6A4FF000009847B8694BF672
:10FF08006153C0F6020398474FF00203FB611AE001
:10FF18007B695B6B9847F860FB68002B12DDB8695A
:10FF280079694BF2CD43C0F6020398470BE0B869F4
:10FF380079694BF68D23C0F6020398474FF000030A
:10FF4800FB6100E000BF4FF00A0047F20D33C0F636
:10FF580004039847AEE700BF80B584B000AF78606F
:10FF680041F69123C0F602039847F860FB68002B1E
:10FF780007D14FF47A7047F20D33C0F6040398475F
:10FF8800F7E7F8684DF2B933C0F6030398474FF026
:10FF9800640047F20D33C0F604039847F1E700BF49
:10FFA80090B5B5B002AF78604CF6E963C0F60103CE
:10FFB8009847034693F82630002B04D04EF62923A1
:10FFC800C0F6010398474FF00003C7F8BC304FF064
:10FFD8000003C7F8B830D7F8B830002B08D04FF076
:10FFE800640047F20D33C0F60403984700F035BCAF
:08FFF8004FF00A0047F20D333F
:020000040802F0
:10000000C0F6040398474CF6E963C0F6010398472D
:10001000034693F82930002B00F022844DF23C2354
:10002000C2F20003D3F89032002B20D04DF23C23D3
:10003000C2F20003D3F890320A2B0FD94DF23C23C1
:10004000C2F20003D3F89032A3F10A024DF23C232E
:10005000C2F20003C3F8902200F003BC4DF23C232F
:10006000C2F200034FF00002C3F89022F9E34FF010
:100070000003C7F8BC304FF00003C7F8C430D7E323
:100080004FF24113C0F6010398470346002B0ED0F0
:100090004CF6E963C0F60103984703464FF00002AF
:1000A00083F829204FF00103C7F8B830CDE3D7F823
:1000B000C4004BF6F173C0F601039847C7F8AC00D3
:1000C000D7F8AC30002B00F0A483D7F8AC3093F80D
:1000D0004B31002B06D1D7F8AC304FF0000283F83B
:1000E00075219FE3D7F8AC309B780D2B00F084820C
:1000F000D7F8AC309B780C2B1CD14FF00103C7F81C
:10010000BC304BF6A953C0F602039847C7F8A800C5
:10011000D7F8A830002B06DAD7F8AC304FF0000241
:1001200083F875217EE3D7F8AC30D7F8A820C3F860
:10013000622161E2D7F8AC309B78062B40F00A814F
:100140004FF00003C7F8B430D7F8AC3093F8643000
:10015000022B0BD0D7F8AC3093F86430032B05D0CA
:10016000D7F8AC3093F86430042B7AD1D7F8AC30A0
:1001700093F85E301946D7F8AC3093F85F301A46E2
:10018000D7F8AC301B6E4FF00200009007F168000A
:1001900001904FF000004EF24954C0F60104A04710
:1001A000C7F8C000BB6EC7F8B430D7F8C030002B1A
:1001B00040F09880D7F8AC3093F86430042B18D115
:1001C000D7F8AC3093F8653007F16802104619464D
:1001D00043F63D33C0F602039847C7F8A000D7F8AE
:1001E000AC00D7F8A01040F6F133C0F602039847F0
:1001F00078E0D7F8AC3093F86430032B18D1D7F8F7
:10020000AC3093F8653007F168021046194643F6A2
:100210003543C0F602039847C7F89C00D7F8AC00F6
:10022000D7F89C1040F69123C0F60203984759E096
:10023000D7F8AC3093F8653007F1680210461946DC
:1002400043F62D53C0F602039847C7F89800D7F835
:10025000AC00D7F8981040F63113C0F60203984767
:1002600040E0D7F8AC3093F85E301946D7F8AC30A0
:1002700093F85F301A46D7F8AC301B6E4FF0010090
:10028000009007F1640001904FF000004EF24954D5
:10029000C0F60104A047C7F8C0007B6EC7F8B430B1
:1002A000D7F8AC3093F86430002B0DD17B6EA7F8F3
:1002B000A630B7F9A630D7F8AC00194640F631138E
:1002C000C0F6020398470EE07B6EA7F8A430B7F89B
:1002D000A430D7F8AC00194640F69123C0F60203CB
:1002E000984700E000BFD7F8C0004DF61563C0F690
:1002F00001039847D7F8AC304FF0000283F876211D
:10030000D7F8C02040F20E739A4212D14EF6B913BC
:10031000C0F601039847D7F8B430DAB2D7F8AC305A
:1003200083F87621D7F8AC304FF0010283F87521BD
:1003300078E2D7F8C030002B00F05E814EF69113C2
:10034000C0F601039847D7F8AC304FF0010283F8AC
:10035000752167E2D7F8AC309B78082B57D1D7F8D6
:10036000AC30D3F84D2007F15C031046194649F232
:10037000C953C0F602039847C7F8C000D7F8C03089
:10038000002B06D0D7F8AC304FF0010283F875216E
:1003900048E2D7F8AC30D3F84D3003F1010207F151
:1003A00060031046194649F2C953C0F60203984744
:1003B000C7F8C000D7F8C030002B06D0D7F8AC3053
:1003C0004FF0010283F875212CE2FB6D4FEA0342E6
:1003D0003B6E1A43D7F8AC30C3F86221D7F8AC3083
:1003E000D3F84D30A3F51C43A3F1BA034FEA5303EE
:1003F000C7F89430D7F8AC30D3F86231D7F894000E
:10040000194642F61933C0F602039847F4E0D7F8CC
:10041000AC309B780B2B53D1D7F8AC30D3F84D20B0
:100420004BF22B039A424BD9D7F8AC30D3F84D207E
:100430004BF28F039A4243D8D7F8AC30D3F84D2013
:1004400007F154031046194649F2C953C0F6020396
:100450009847C7F89000D7F8AC30D3F84D3003F187
:10046000010207F1540303F104031046194649F24F
:10047000C953C0F602039847C7F88C00D7F89030EC
:10048000002B03D1D7F88C30002B06D0D7F8AC3036
:100490004FF0010283F87521C4E107F154031846B7
:1004A0004FF0030143F63D33C0F602039847C7F807
:1004B0008800D7F8AC30D7F88820C3F862219BE0D9
:1004C000D7F8AC309B78052B47D1D7F8AC30D3F8B0
:1004D0004D2049F6CE439A423FD1D7F8AC30D3F8FD
:1004E0004D2007F150031046194649F2C953C0F692
:1004F00002039847C7F8C000D7F8C030002B06D0D9
:10050000D7F8AC304FF0010283F875218AE1D7F8B3
:10051000AC30D3F84D3003F1010207F14C03104623
:10052000194649F2C953C0F602039847C7F8C000FC
:10053000D7F8C030002B06D0D7F8AC304FF001020E
:1005400083F875216EE1FB6C4FEA03423B6D1A4361
:10055000D7F8AC30C3F862214EE0D7F8AC309B78C6
:10056000002B26D14FF00003BB64D7F8AC30D3F892
:100570004D2007F148031046194649F2C953C0F609
:1005800002039847C7F8C000D7F8C030002B06D048
:10059000D7F8AC304FF0010283F8752142E1BB6C13
:1005A000D7F8AC00194640F63113C0F6020398475D
:1005B00022E0D7F8AC30D3F84D2007F144031046C1
:1005C000194649F2C953C0F602039847C7F8C0005C
:1005D000D7F8C030002B06D0D7F8AC304FF001026E
:1005E00083F875211EE17B6CA7F88630B7F9862069
:1005F000D7F8AC30C3F86221D7F8AC309B780D2B1C
:100600000CD1D7F8AC3093F88131022B0CD1D7F84C
:10061000AC304FF0020283F8752105E0D7F8AC301A
:100620004FF0020283F87521D7F8AC0045F2114370
:10063000C0F602039847D7F8AC3093F87830002B17
:1006400006D0D7F8AC0044F2D143C0F60203984775
:10065000D7F8AC30DB78002B00F0DD8007F17003B9
:1006600018464FF63D13C0F6030398474CF6E9636E
:10067000C0F601039847034693F82630002B71D04B
:100680004EF67D23C0F6010398470346002B00F089
:10069000C4804DF2F143C0F6030398474BF65D3337
:1006A000C0F601039847C7F880004FF00003C7F871
:1006B000B03046E0D7F8B0004BF6F173C0F6010356
:1006C0009847F867FB6F93F87531022B33D14FF0E1
:1006D000000387F83330FB6FB3F900309BB29BB255
:1006E000BB86FB6FD3F86631C7F83A30FB6FD3F89F
:1006F0006231C7F8363007F12C0307F1700292E837
:100700000300186003F10403198003F102034FEAA8
:1007100011421A7007F12803184640F2F923C0F677
:1007200003039847C7F8C000D7F8AC0040F6690348
:10073000C0F602039847D7F8B03003F10103C7F8B9
:10074000B030D7F8B020D7F880309A42B2DB4EF6FE
:100750002923C0F6010398474DF22553C0F6030341
:1007600098475FE0D7F8AC3093F87531022B56D13B
:10077000D7F8AC3003F5AA7307F17002104619469A
:100780004FF63543C0F603039847B867BA6FD7F8FA
:10079000AC30D3F851309A4243D3D7F8AC3003F59C
:1007A000AA7318464FF63D13C0F6030398474FF05F
:1007B0000003FB75D7F8AC30B3F900309BB29BB2A5
:1007C0003B83D7F8AC30D3F86631C7F81E30D7F882
:1007D000AC30D3F86231C7F81A3007F10C0303F1DB
:1007E000040318464FF63D13C0F60303984707F17C
:1007F0000C03184640F2F923C0F603039847C7F8E4
:10080000C000D7F8AC0040F66903C0F60203984771
:1008100008E000BF06E000BF04E000BF02E000BF48
:1008200000E000BFD7F8C43003F10103C7F8C430BB
:10083000D7F8C4404CF6E963C0F601039847034675
:10084000D3F822359C42FFF41BACD7F8BC30DAB2A7
:100850004DF23C23C2F2000383F88022FFF7BFBBB6
:1008600000BFFFF7BCBB00BF80B584B000AF7860AD
:100870007B689B78082B22D17B6893F84331002B4F
:100880001DD07B68D3F84D3018464BF2E503C0F617
:1008900002039847F860F8684FF0000142F6C91368
:1008A000C0F602039847FB6803F1FF33BB60B868EA
:1008B0004FF0000142F61933C0F6020398477B68F7
:1008C0009B78002B03D07B689B78062B25D17B6817
:1008D00093F84431012B0DD17B68124AC3F877217C
:1008E0007B684FF0000283F87B214FF0000283F811
:1008F0007C2112E07B6893F84431022B04D17B68A1
:10090000094AC3F87D2108E07B6893F84431032B42
:1009100003D17B68054AC3F87D2107F11007BD4666
:1009200080BD00BF00000000FFFF7F7FFFFF7FFF53
:1009300090B583B000AF786039607B6893F844313C
:10094000012B48D17B68D3F8774123461C464AF2F5
:10095000C543C0F601033868984702464AF25D3342
:10096000C0F6010320461146984703461A467B68A5
:10097000C3F877217B68B3F87B319BB203F10103A5
:100980009AB27B68A3F87B217B68D3F87741234632
:100990001C467B68B3F87B319BB21A464AF2C543CA
:1009A000C0F601031046984702464AF2D563C0F6E6
:1009B000010320461146984703461A464AF6F903B2
:1009C000C0F601031046984703463B607B683A68CF
:1009D000C3F8622157E07B6893F84431022B24D19D
:1009E0004AF2C543C0F601033868984701467B6860
:1009F000D3F87D2113461A464AF6A903C0F601032F
:100A00000846114698470346002B3CD04AF2C5439E
:100A1000C0F601033868984702467B68C3F87D2119
:100A20007B683A68C3F862212DE07B6893F8443113
:100A3000032B24D14AF2C543C0F601033868984716
:100A400001467B68D3F87D2113461A464AF6E50332
:100A5000C0F601030846114698470346002B12D002
:100A60004AF2C543C0F601033868984702467B68DE
:100A7000C3F87D217B683A68C3F8622103E07B6894
:100A80003A68C3F8622107F10C07BD4690BD00BF6C
:100A900090B583B000AF786039607B6893F84431DB
:100AA000012B48D17B68D3F8774123461C464AF294
:100AB000BD43C0F601033868984702464AF25D33E9
:100AC000C0F6010320461146984703461A467B6844
:100AD000C3F877217B68B3F87B319BB203F1010344
:100AE0009AB27B68A3F87B217B68D3F877412346D1
:100AF0001C467B68B3F87B319BB21A464AF2C54369
:100B0000C0F601031046984702464AF2D563C0F684
:100B1000010320461146984703461A464AF64513F4
:100B2000C0F601031046984703463B607B683A686D
:100B3000C3F8622157E07B6893F84431022B24D13B
:100B40004AF2BD43C0F601033868984701467B6806
:100B5000D3F87D2113461A464AF6A903C0F60103CD
:100B60000846114698470346002B3CD04AF2BD4345
:100B7000C0F601033868984702467B68C3F87D21B8
:100B80007B683A68C3F862212DE07B6893F84431B2
:100B9000032B24D14AF2BD43C0F6010338689847BD
:100BA00001467B68D3F87D2113461A464AF6E503D1
:100BB000C0F601030846114698470346002B12D0A1
:100BC0004AF2BD43C0F601033868984702467B6885
:100BD000C3F87D217B683A68C3F8622103E07B6833
:100BE0003A68C3F8622107F10C07BD4690BD00BF0B
:100BF00090B583B000AF786039607B6893F844317A
:100C0000012B39D17B68D3F8772113461A464AF273
:100C10005D33C0F6010310463968984703461A460B
:100C20007B68C3F877217B68B3F87B319BB203F113
:100C300001039AB27B68A3F87B217B68D3F87741E4
:100C400023461C467B68B3F87B319BB21A464AF2B6
:100C5000C543C0F601031046984702464AF2D563E1
:100C6000C0F6010320461146984703463B607B6867
:100C70003A68C3F862213DE07B6893F84431022B67
:100C800017D17B68D3F87D2113461A464AF6E5034F
:100C9000C0F601031046396898470346002B29D057
:100CA0007B683A68C3F87D217B683A68C3F86221A3
:100CB00020E07B6893F84431032B17D17B68D3F88D
:100CC0007D2113461A464AF6A903C0F601031046D1
:100CD000396898470346002B0CD07B683A68C3F804
:100CE0007D217B683A68C3F8622103E07B683A683B
:100CF000C3F8622107F10C07BD4690BD90B58BB0DB
:100D000000AF4FF000037B624DF2F040C2F20000F2
:100D10004FF0000142F2607246F20903C0F601038F
:100D200098474FF000033B620CE04DF2F043C2F2F3
:100D300000033A6A9B184FF000021A703B6A03F1F5
:100D400001033B623B6A122BEFDD4DF2F043C2F22E
:100D500000034FF001021A704DF2F043C2F200039B
:100D600003F51D5303F11C034FF000021A604DF20E
:100D7000F043C2F2000303F51D5303F11C031B688B
:100D800043F001024DF2F043C2F2000303F51D539C
:100D900003F11C031A604DF2F043C2F2000303F5A5
:100DA0001D5303F11C031B6843F002024DF2F04394
:100DB000C2F2000303F51D5303F11C031A604DF248
:100DC000F043C2F2000303F51D5303F11C031B683B
:100DD00043F004024DF2F043C2F2000303F51D5349
:100DE00003F11C031A604EF64913C0F6030398473B
:100DF00042F65563C0F6020398474EF25123C0F6FF
:100E0000030398474FF001033B6218E03B6A03F18C
:100E1000FF33FB6107F10803F869194642F61143F5
:100E2000C0F602039847BB68386A194642F61D139C
:100E3000C0F6020398473B6A03F101033B623B6A39
:100E4000042BE3DD4DF6E923C0F6030398474EF289
:100E50008503C0F6030398474FF0010042F699233B
:100E6000C0F6020398474FF48050C4F201004FF0DF
:100E7000100140F68953C0F6050398474FF0C800AB
:100E800047F2E103C0F6050398474FF000033B62C9
:100E900036E042F63553C0F6020398474FF4FA7035
:100EA00047F2E103C0F60503984742F6F553C0F652
:100EB000020398474FF4FA7047F2E103C0F60503C6
:100EC000984742F69553C0F6020398474FF4FA70DC
:100ED00047F2E103C0F60503984742F66553C0F6B2
:100EE0000203984742F62563C0F60203984742F68C
:100EF000C553C0F6020398473B6A03F101033B6206
:100F00003B6A022BC5DD42F63553C0F60203984713
:100F10004FF0190041F21143C0F6020398474FF019
:100F200001004FF000014FF2DD73C0F60303984754
:100F300003467B6244F65523C0F6040398474FF0FE
:100F400001004FF0020144F24143C0F60403984708
:100F50004FF03A0044F2D143C0F6040398474EF6EE
:100F6000D503C0F6020398474EF68923C0F6020364
:100F7000984778627B6A002B11D040F60843C2F292
:100F800000034FF001021A604EF68D03C0F6030312
:100F900098474EF60523C0F60203984778624EF64E
:100FA0003113C0F60203984778624FF0010041F216
:100FB000C523C0F6030398470346002B15D14FF015
:100FC000000041F2C523C0F6030398470346002BF7
:100FD0000BD14FF00200796A4EF26D23C0F6010387
:100FE00098474FF000037B6238E04EF60D33C0F6B1
:100FF000020398474FF6F963C0F6020398477862F8
:101000007B6A002B16D04EF60D33C0F602039847CC
:101010004FF65953C0F6020398477862786A4DF646
:10102000BD53C0F6010398477B6A002B02D04FF0F6
:1010300000037B6241F27953C0F60303984740F204
:101040004503C0F60303984740F2A903C0F6030323
:1010500098474FF65953C0F60203984741F2C953D7
:10106000C0F60303984703469B68BB6141F2F14316
:10107000C0F60203984778614FF0010079694EF29B
:101080003D43C0F6010398474FF04F004FF4C27143
:101090004EF23D43C0F60103984741F21523C0F6D6
:1010A0000303984738614FF0220039694EF23D43FF
:1010B000C0F60103984741F25123C0F60303984755
:1010C00038614FF0230039694EF23D43C0F6010309
:1010D00098474CF6FD63C0F6010398474CF6E96368
:1010E000C0F6010398470346D3F80631002B37D0EA
:1010F0004CF6E963C0F6010398470346D3F816217E
:1011000013464FEA03139B1A4FEA83031C464CF61F
:10111000E963C0F6010398470346D3F81A21134642
:101120004FEA03139B1A4FEA83032046194643F202
:101130006573C0F602039847F860B8694DF27943C9
:10114000C0F603039847F8684DF29943C0F60303CD
:1011500098473B4618464FF63D13C0F603039847A1
:1011600041F23163C0F60203984778627B6A002B34
:1011700006D0786A4DF6BD53C0F60103984740E1AA
:1011800041F29573C0F60203984778627B6A002BA0
:101190000ED04FF01400796A4EF23D43C0F60103C1
:1011A0009847786A4DF6BD53C0F60103984728E189
:1011B00041F61903C0F60203984778627B6A002B58
:1011C0000ED04FF01500796A4EF23D43C0F6010390
:1011D0009847786A4DF6BD53C0F60103984710E171
:1011E00041F69913C0F60203984778627B6A002B98
:1011F0000ED04FF05A00796A4EF23D43C0F601031B
:101200009847786A4DF6BD53C0F601039847F8E059
:1012100041F2E553C0F60203984778627B6A002BDF
:1012200006D0786A4DF6BD53C0F601039847E8E052
:1012300046F2D923C0F60203984778627B6A002BF6
:101240000DD04FF01800796A4EF23D43C0F601030D
:101250009847786A4DF6BD53C0F60103984746F6A5
:101260001D13C0F60203984778627B6A002B0DD0ED
:101270004FF01D00796A4EF23D43C0F601039847D6
:10128000786A4DF6BD53C0F60103984744F62D1316
:10129000C0F60403984741F6E123C0F602039847DD
:1012A00078627B6A002B10D04FF00300796A4EF20F
:1012B0003D43C0F601039847786A4DF6BD53C0F62A
:1012C000010398474FF000037B6241F68D33C0F66F
:1012D0000203984778627B6A002B10D04FF004001D
:1012E000796A4EF23D43C0F601039847786A4DF69D
:1012F000BD53C0F6010398474FF000037B6241F6EF
:101300002953C0F60203984778627B6A002B10D0FD
:101310004FF01000796A4EF23D43C0F60103984742
:10132000786A4DF6BD53C0F6010398474FF00003AD
:101330007B6241F61943C0F60203984778627B6AE4
:10134000002B10D04FF00500796A4EF23D43C0F6F5
:1013500001039847786A4DF6BD53C0F601039847DC
:101360004FF000037B6241F6A143C0F602039847A9
:1013700078627B6A002B10D04FF05B00796A4EF2E6
:101380003D43C0F601039847786A4DF6BD53C0F659
:10139000010398474FF000037B6241F6A573C0F646
:1013A0000203984778627B6A002B10D04FF006004A
:1013B000796A4EF23D43C0F601039847786A4DF6CC
:1013C000BD53C0F6010398474FF000037B6242F221
:1013D0009503C0F60203984778627B6A002B10D011
:1013E0004FF00700796A4EF23D43C0F6010398477B
:1013F000786A4DF6BD53C0F6010398474FF00003DD
:101400007B627B6A184607F12C07BD4690BD00BF82
:1014100080B582B000AF78607B68184644F6F95317
:10142000C0F60403984707F10807BD4680BD00BF1A
:1014300080B500AF44F6E953C0F60403984780BD79
:1014400080B586B000AF78604FF000037B617B68A9
:101450009B6D4FF0580098477B68DB6D98470346BB
:101460003B610FE04FF0010047F2E103C0F60503D6
:1014700098477B6903F101037B617B68DB6D9847CB
:1014800003463B613B69002B04D07A6940F2E733A5
:101490009A42E7DD3B69002B0BD07B6893F8213043
:1014A00018464FF0020144F6B923C0F604039847EA
:1014B0001AE07B681B6E98470346FB737B6893F8C2
:1014C0002320FB7B1340DAB27B6893F824309A42E6
:1014D0000AD07B6893F8213018464FF0020144F699
:1014E000B923C0F60403984707F11807BD4680BD2D
:1014F00080B500AF4BF62963C0F604039847034656
:10150000184680BD80B500AF4BF6DD63C0F604031E
:10151000984780BD80B483B000AF4FF000037B607C
:101520004FF000033B6014E04DF2F043C2F20003C1
:101530003A689B181B78012B07D14FF001023B68DA
:1015400002FA03F37A6813437B603B6803F10103FB
:101550003B603B68122BE7DD7B68184607F10C0700
:10156000BD4680BC704700BF80B483B000AF7860D8
:1015700039607B68002B12DB7B68122B0FDC3B6829
:10158000012B02D03B68002B0BD13B68DAB24DF245
:10159000F043C2F2000379685B181A7002E000BFE2
:1015A00000E000BF07F10C07BD4680BC704700BFDC
:1015B00080B483B000AF78607B68002B02DB7B686F
:1015C000122B02DD4FF0000306E04DF2F043C2F2B1
:1015D00000037A689B181B78184607F10C07BD4674
:1015E00080BC704780B582B000AF104B7B607868DC
:1015F00048F21513C0F60403984703463B603B6866
:10160000002B06D14DF2F043C2F200034FF001026D
:101610005A7138684DF6BD53C0F6010398473B68D0
:10162000184607F10807BD4680BD00BFE4D600207C
:1016300080B584B000AF564BBB604FF00003FB6039
:101640004CF6E963C0F6010398470346D3F8C2306D
:10165000002B10D14CF6E963C0F60103984703460E
:10166000D3F8CA30082B02D14FF0030301E04FF04A
:101670000203FB600FE04CF6E963C0F601039847F4
:101680000346D3F8CA30082B02D14FF0040301E01F
:101690004FF00303FB604CF6E963C0F60103984783
:1016A0000346D3F8BE301A46BB681A604CF6E963AD
:1016B000C0F6010398470346D3F8C230DAB2BB68DC
:1016C0001A774CF6E963C0F6010398470346D3F84E
:1016D000C630012B0CBF00230123DBB21A46BB68C6
:1016E0005A77FB68DAB2BB689A77BB684FF00E0294
:1016F000DA77BB684FF00E0283F82020BB684FF00A
:10170000010283F82120B86842F6A523C0F604033D
:10171000984778607B68002B06D14DF2F043C2F207
:1017200000034FF001025A704CF6E963C0F6010362
:1017300098470346D3F8C230002B23D04CF6E96318
:10174000C0F6010398470346D3F8CA30082B19D1D5
:101750004FF46050C4F2010040F226614FF00002E5
:1017600045F2C933C0F6050398474FF46050C4F200
:10177000010040F225514FF0000245F2C933C0F696
:10178000050398477B68184607F11007BD4680BDE2
:1017900004D5002080B582B000AF1E4B7B607B6813
:1017A0004FF0020283F821207B684FF4E1321A6087
:1017B0007B684FF496421A607B684FF000021A77FC
:1017C0007B684FF000025A777B684FF003029A77EC
:1017D0007B684FF000025A66786842F6A523C0F68F
:1017E0000403984738603B68002B06D14DF2F04364
:1017F000C2F200034FF00102DA703B6818464DF662
:10180000BD53C0F6010398473B68184607F1080727
:10181000BD4680BDF4D5002080B584B000AF5D4BDF
:10182000BB604CF6E963C0F6010398470346D3F862
:10183000CE301A46BB681A604FF00003FB604CF6CE
:10184000E963C0F6010398470346D3F8D230002B72
:1018500010D14CF6E963C0F6010398470346D3F86C
:10186000DA30082B02D14FF0030301E04FF00203FE
:10187000FB600FE04CF6E963C0F6010398470346AE
:10188000D3F8DA30082B02D14FF0040301E04FF017
:101890000303FB604CF6E963C0F601039847034677
:1018A000D3F8D230DAB2BB681A774CF6E963C0F6E7
:1018B000010398470346D3F8D630012B0CBF002311
:1018C0000123DBB21A46BB685A77FB68DAB2BB6801
:1018D0009A77BB684FF00E02DA77BB684FF00E02C2
:1018E00083F82020BB684FF0030283F82120BA68F8
:1018F00041F68973C0F602035366B86842F6A52321
:10190000C0F60403984778607B68002B0ED14DF237
:10191000F043C2F200034FF001021A714DF2F0439E
:10192000C2F200034FF0000283F8E4224CF6E963B0
:10193000C0F6010398470346D3F8D230002B23D0DA
:101940004CF6E963C0F6010398470346D3F8DA3052
:10195000082B19D14FF49040C4F2000040F22661E8
:101960004FF0000245F2C933C0F6050398474FF423
:101970009040C4F2000040F225514FF0000245F2C1
:10198000C933C0F6050398477B68184607F110076E
:10199000BD4680BD6CD6002080B582B000AF1D4B27
:1019A0007B607B684FF416521A607B684FF0000230
:1019B0001A777B684FF000025A777B684FF003027A
:1019C0009A777B684FF00E02DA777B684FF00E0251
:1019D00083F820207B684FF0050283F821207B6884
:1019E0004FF000025A66786842F6A523C0F6040359
:1019F000984738603B68002B06D14DF2F043C2F2A5
:101A000000034FF001029A733B68184607F108077C
:101A1000BD4680BD5CD7002080B400AF4DF2F043DE
:101A2000C2F20003DB7A012B02D04FF0000300E08A
:101A3000024B1846BD4680BC704700BFECD8002062
:101A400080B400AF4DF2F043C2F200031B7A012BC9
:101A500002D04FF0000300E0024B1846BD4680BCA8
:101A6000704700BFD8D7002080B400AF4DF2F043DC
:101A7000C2F200035B7A012B02D04FF0000300E0BA
:101A8000024B1846BD4680BC704700BF34D80020CA
:101A900080B400AF4DF2F043C2F200039B7A012BF9
:101AA00002D04FF0000300E0024B1846BD4680BC58
:101AB000704700BF90D8002080B400AF4DF2F043D3
:101AC000C2F20003DB7B012B02D04FF0000300E0E9
:101AD000024B1846BD4680BC704700BF48D9002065
:101AE00080B586B000AF4DF2F043C2F20003DB7860
:101AF000012B02D040F6FD0340E04FF000037B6174
:101B00004CF6D963C0F602037B611F4879694CF635
:101B10002113C0F6020398474DF2F043C2F20003CE
:101B20004FF001029A7241F69123C0F602039847E2
:101B300038613B69002B0AD140F60913FB60F86855
:101B40004DF6BD53C0F601039847FB6816E04FF011
:101B5000020041F68963C0F60203984703463B60E2
:101B60003B46BB603B699B68B8689847786078687B
:101B70004DF6BD53C0F6010398477B68184607F140
:101B80001807BD4680BD00BF90D8002080B584B046
:101B900000AF4DF2F043C2F200031B79012B02D0DB
:101BA00040F6FD032FE04DF6BD13C0F602031848C2
:101BB00019464CF62113C0F6020398474DF2F04344
:101BC000C2F200034FF001025A724FF0030041F6D7
:101BD0008963C0F60203984703463B600D4B7B6068
:101BE00041F66923C0F602039847F860FB689B68DA
:101BF0003A4610469847B860B8684DF6BD53C0F6EF
:101C000001039847BB68184607F11007BD4680BD21
:101C100034D80020D4D7002080B584B000AF4DF276
:101C2000F043C2F200035B78012B02D040F6FD03C3
:101C30002EE04CF66113C0F60203184819464CF624
:101C40002113C0F6020398474DF2F043C2F200039D
:101C50004FF001021A724FF0000041F68963C0F69E
:101C60000203984703467B6041F64123C0F6020316
:101C70009847F860FB689B6807F104021046984794
:101C8000B860B8684DF6BD53C0F601039847BB680D
:101C9000184607F11007BD4680BD00BFD8D7002009
:101CA00080B584B000AF4DF2F043C2F200039B7BDD
:101CB000012B02D040F6FD032EE04DF24543C0F665
:101CC0000203184819464CF62113C0F60203984740
:101CD0004DF2F043C2F200034FF00102DA734FF00D
:101CE000050041F68963C0F60203984703467B600E
:101CF00041F6B923C0F602039847F860FB689B6879
:101D000007F1040210469847B860B8684DF6BD5315
:101D1000C0F601039847BB68184607F11007BD4697
:101D200080BD00BF48D9002080B584B000AF4DF21F
:101D3000F043C2F200035B79012B02D040F6FD03B1
:101D40002EE04EF2AD33C0F60203184819464CF6A9
:101D50002113C0F6020398474DF2F043C2F200038C
:101D60004FF00102DA724FF0040041F68963C0F6C9
:101D70000203984703467B6041F61923C0F602032D
:101D80009847F860FB689B6807F104021046984783
:101D9000B860B8684DF6BD53C0F601039847BB68FC
:101DA000184607F11007BD4680BD00BFECD80020E3
:101DB00080B400AF4FF000031846BD4680BC7047AA
:101DC00080B400AF4FF000031846BD4680BC70479A
:101DD00080B400AF4FF000031846BD4680BC70478A
:101DE00080B500AF4FF4C050C4F201004FF00801BD
:101DF00040F68953C0F60503984740F24C4047F23D
:101E0000E103C0F6050398474FF4C050C4F2010047
:101E10004FF0080140F6A553C0F6050398474FF46C
:101E20007A7047F2E103C0F6050398474FF4C050BB
:101E3000C4F201004FF0100140F6A553C0F60503AF
:101E400098474FF0FA0047F2E103C0F605039847C0
:101E50004FF00003184680BD80B500AF4FF4C0506E
:101E6000C4F201004FF0080140F6A553C0F6050387
:101E700098474FF0FA0047F2E103C0F60503984790
:101E80004FF00003184680BD80B483B000AF786087
:101E90007B68002B02DB7B68052B02DD4FF0000323
:101EA0006CE07B68052B0FD801A252F823F000BF2D
:101EB000E31E0208F71E02080B1F02081F1F02087C
:101EC000CF1E0208331F02084FF0000356E04DF208
:101ED000F043C2F200035B79002B34D14FF00003D2
:101EE0004CE04DF2F043C2F200035B78002B2CD1A2
:101EF0004FF0000342E04DF2F043C2F200039B7842
:101F0000002B24D14FF0000338E04DF2F043C2F231
:101F10000003DB78002B1CD14FF000032EE04DF2C4
:101F2000F043C2F200031B79002B14D14FF00003E1
:101F300024E04DF2F043C2F200039B7B002B0CD156
:101F40004FF000031AE000BF08E000BF06E000BF4A
:101F500004E000BF02E000BF00E000BF7A68134663
:101F60004FEA03139B1A4FEAC30303F110024DF229
:101F7000F043C2F20003D31803F10403184607F13B
:101F80000C07BD4680BC704780B400AF4DF2F043F3
:101F9000C2F200034FF0010283F8E422BD4680BC88
:101FA000704700BF90B585B000AF4FF00003BB6035
:101FB0004DF2F043C2F200034FF0FF0283F8B42465
:101FC0004DF2F043C2F200034FF001029A714FF05C
:101FD0000003FB6028E0FB687B607B6803F1010382
:101FE0007B604CF6E963C0F6010398470246FB6844
:101FF000D31803F1DE031B781C464CF6E963C0F6E8
:10200000010398470246FB68D31803F1E6031B78E7
:10201000786821461A4642F63123C0F602039847F3
:10202000FB6803F10103FB60FB68012BD3DD4FF07C
:1020300002004FF064014FF2A113C0F6030398476A
:102040004FF003004FF064014FF2A113C0F60303F9
:1020500098474FF002004FF000014FF22563C0F6A1
:10206000030398474FF003004FF000014FF2256340
:10207000C0F603039847BB68002BB8684DF6BD5304
:10208000C0F601039847BB68184607F11407BD4620
:1020900090BD00BF80B582B000AF4FF000037B6001
:1020A000114840F69E0144F66163C0F60403984768
:1020B0000E4840F69E0145F24103C0F604039847DE
:1020C0004DF2F043C2F200034FF00102DA7178687A
:1020D0004DF6BD53C0F6010398477B68184607F1DB
:1020E0000807BD4680BD00BFA6D90020E2EA002057
:1020F00080B584B000AF786039604DF2F043C2F231
:1021000000039B79012B02D040F6FD0331E04FF034
:102110000003FB603B684FF000021A607B68002BF5
:1021200002DD7B68022B03DD40F60213FB6019E041
:102130007B68BB60BB6803F1FF33BB604DF2F043CB
:10214000C2F2000393F8B4341A46BB6842FA03F3B0
:1021500003F00103002B14BF00230123DBB21A4656
:102160003B681A60F8684DF6BD53C0F60103984706
:10217000FB68184607F11007BD4680BD80B584B0E6
:1021800000AF786039604DF2F043C2F200039B79F2
:10219000012B02D040F6FD03CAE04FF00003FB60C4
:1021A0007B68002B02DD7B68022B09DD40F6021301
:1021B000FB60F8684DF6BD53C0F601039847B0E0E8
:1021C0007B68BB60BB6803F1FF33BB604DF2F0433B
:1021D000C2F2000393F8B434DAB24FF00101BB68E5
:1021E00001FA03F3DBB26FEA0303DBB21340DBB2A5
:1021F000DAB24DF2F043C2F2000383F8B4243B6834
:10220000002B15D14DF2F043C2F2000393F8B43421
:10221000DAB24FF00101BB6801FA03F3DBB21343FA
:10222000DBB2DAB24DF2F043C2F2000383F8B42419
:102230004CF6E963C0F6010398470246BB68D31821
:1022400003F1DE031B78022B14D14CF6E963C0F6D0
:102250000103984701463B68DAB2BB68CB1803F12B
:10226000E6031A704FF400404DF2D503C0F60103A7
:102270009847F86040F60843C2F200031B68012B40
:1022800022D13B68002B0FD178684EF69933C0F607
:10229000030398470346012B02D14FF0000301E0EE
:1022A00040F60313FB6035E078684EF67523C0F600
:1022B000030398470346012B02D14FF0000301E0CE
:1022C00040F60313FB6025E03B68002B11D17868D2
:1022D0004EF60D43C0F603039847F860FB68012BE8
:1022E00003D14FF00003FB6014E040F60313FB60E2
:1022F00010E078684EF6E923C0F603039847F860CB
:10230000FB68012B03D14FF00003FB6002E040F6B5
:102310000313FB60FB68002B03D040F60313FB6044
:1023200000BFF8684DF6BD53C0F601039847FB683F
:10233000184607F11007BD4680BD00BF80B588B0C4
:1023400000AF786039604DF2F043C2F200039B7930
:10235000012B02D040F6FD03B0E04FF00003FB611B
:102360003B684FF000021A607B68002B02DB7B6841
:10237000032B03DD40F60113FB6198E07B68002B23
:102380000EDB7B68032B0BDC7B6803F10103184633
:102390004EF62D23C0F60303984702463B681A60A9
:1023A0007B68032B38DD7B680B2B35DC786842F2C9
:1023B000F543C0F602039847B861BB69B3F1FF3F2C
:1023C00003D140F60113FB6171E07B680A2B02D058
:1023D0007B680B2B10D1BB699BB24FF44060C4F2F9
:1023E0000100194640F6D943C0F605039847034655
:1023F0001A463B681A600FE0BB699BB24FF4A050CD
:10240000C4F20100194640F6D943C0F605039847C7
:1024100003461A463B681A607B680B2B47DD7B68D6
:102420004B2B44DC786842F2C943C0F6020398475C
:1024300078617B68A3F10C0303F10702002BB8BF9E
:1024400013464FEAE30303F101033B613B6903F1E8
:10245000FF334FEA430303F17003FB6040F60C4087
:10246000C2F2000041F65563C0F6040398474FF0EE
:102470000003FB72FB68DAB207F10B031046194642
:1024800041F26D53C0F6040398470346FB61FB69B4
:10249000002B03D040F60413FB6108E0FB7A1A46D8
:1024A0007B6942FA03F303F001023B681A60F869A2
:1024B0004DF6BD53C0F601039847FB69184607F176
:1024C0002007BD4680BD00BF80B483B000AF7860F8
:1024D0007B68A3F10C024FEAE2734FEA5373D21800
:1024E00002F00702D31A184607F10C07BD4680BC5C
:1024F000704700BF80B483B000AF78607B68042B66
:1025000002D14FF480432BE07B68052B02D14FF4BE
:10251000005325E07B68062B02D14FF001031FE03A
:102520007B68072B02D14FF4004319E07B68082B2E
:1025300002D14FF0080313E07B68092B02D14FF062
:1025400010030DE07B680A2B02D14FF0400307E037
:102550007B680B2B02D14FF0800301E04FF0FF337B
:10256000184607F10C07BD4680BC704780B582B0A5
:1025700000AF786039604DF2F043C2F20003DB79BE
:10258000012B02D040F6FD0374E03B684FF00002DF
:102590001A607B68002B02DB7B68032B09DD4FF49C
:1025A00010604DF6BD53C0F6010398474FF4106319
:1025B00060E07B68002B20D144F68973C0F60403E9
:1025C000984700BF44F6E573C0F6040398470346F6
:1025D000002BF7D12A4840F69E0143F2D163C0F6A2
:1025E0000203984702464AF6F903C0F60103104673
:1025F000984702463B681A603AE07B68012B20D17D
:1026000045F26D13C0F60403984700BF45F2C913A5
:10261000C0F6040398470346002BF7D1194840F64B
:102620009E0143F2D163C0F60203984702464AF680
:10263000F903C0F601031046984702463B681A604A
:1026400016E07B68022B08D14DF63D63C0F603030C
:10265000984702463B681A600AE07B68032B07D163
:102660004DF61D73C0F60303984702463B681A6097
:102670004FF00003184607F10807BD4680BD00BFB4
:10268000A6D90020E2EA002080B584B000AFF8604F
:10269000B9607A607B684FF000021A60FB68002B1B
:1026A00002DBFB68022B09DD40F60E104DF6BD5330
:1026B000C0F60103984740F60E1345E0BB68002BB7
:1026C00002DBBB680A2B09DD40F60E104DF6BD5348
:1026D000C0F60103984740F60E1335E0FB68002B67
:1026E00009D14DF2F043C2F200031B7C012B02D052
:1026F00040F6FD0328E0FB68012B09D14DF2F043C1
:10270000C2F200035B7C012B02D040F6FD031BE00C
:10271000FB68022B09D14DF2F043C2F200039B7C0F
:10272000012B02D040F6FD030EE0BB68DBB2F86877
:10273000194643F28D13C0F60203984703461A4622
:102740007B681A604FF00003184607F11007BD467A
:1027500080BD00BF80B584B000AFF860B9607A601A
:102760004DF2F043C2F20003DB79012B02D040F6B8
:10277000FD035EE0BB684FF000021A60FB68002BAF
:1027800002DBFB68032B09DD4FF410604DF6BD53EF
:10279000C0F6010398474FF410634AE0FB68002B32
:1027A00021D144F68973C0F60403984700BF44F66C
:1027B000E573C0F6040398470346002BF7D11F4882
:1027C00040F69E017A6843F26953C0F602039847C7
:1027D00002464AF6F903C0F601031046984702463E
:1027E000BB681A6023E0FB68032B20D145F26D1310
:1027F000C0F60403984700BF45F2C913C0F60403AE
:1028000098470346002BF7D10D4840F69E017A68A1
:1028100043F26953C0F60203984702464AF6F903A9
:10282000C0F60103104698470246BB681A604FF095
:102830000003184607F11007BD4680BDA6D9002049
:10284000E2EA002080B582B000AF786039603B6872
:102850004FF000021A607B68002B02DB7B68012BC3
:1028600009DD40F60D104DF6BD53C0F60103984743
:1028700040F60D131CE07B68002B0AD14FF00200DC
:102880004FF29D53C0F60303984702463B681A6017
:102890000CE07B68012B09D14FF003004FF29D53F0
:1028A000C0F60303984702463B681A604FF00003E6
:1028B000184607F10807BD4680BD00BF80B485B04B
:1028C00000AFF860B9607A603B604DF2F043C2F24D
:1028D0000003FA6802F6CC1253F82220BB681A6093
:1028E0004DF2F042C2F20002FB6803F6CE134FEA4B
:1028F0008303D3185A687B681A604DF2F043C2F222
:102900000003FA6802F6D21253F822203B681A60DC
:1029100007F11407BD4680BC704700BF80B584B086
:1029200000AF7860396078684EF21543C0F6030353
:1029300098470346FB60FB68002B02D04FF41163FD
:1029400008E0786839684EF21933C0F603039847F7
:102950004FF00003184607F11007BD4680BD00BFC9
:1029600080B584B000AF786078684EF2B933C0F6B5
:10297000030398470346FB60FB68002B02D040F638
:10298000111301E04FF00003184607F11007BD4690
:1029900080BD00BF80B584B000AF786078684EF22B
:1029A000B933C0F6030398470346FB60FB68002B6E
:1029B00002D040F6121301E04FF00003184607F171
:1029C0001007BD4680BD00BF80B582B000AF786003
:1029D0003960786839684EF21933C0F603039847B6
:1029E0004FF00003184607F10807BD4680BD00BF41
:1029F00080B584B000AF7860396007F1080378686B
:102A000019464EF2C523C0F6030398470346FB6000
:102A1000FB68002B02D040F6131304E0BA683B6851
:102A20001A604FF00003184607F11007BD4680BD3D
:102A300080B586B000AFF860B9607A604FF00003EF
:102A40007B61BB68012B0DD0022B15D0002B1CD154
:102A5000F8684FF0000142F27D13C0F60203984778
:102A6000786112E0F8684FF0010142F27D13C0F680
:102A700002039847786108E0F868796842F27D13AC
:102A8000C0F602039847786100BF7B69184607F1DA
:102A90001807BD4680BD00BF80B582B000AF78602A
:102AA0007B68002B10D14DF2F043C2F2000303F516
:102AB0001D5303F118034FF000021A604DF6B15395
:102AC000C0F6030398470FE04DF2F043C2F2000353
:102AD00003F51D5303F118034FF001021A604DF680
:102AE0009553C0F6030398474FF00003184607F1CB
:102AF0000807BD4680BD00BF80B400AF4DF2F04373
:102B0000C2F2000303F51D5303F118031B681846B6
:102B1000BD4680BC704700BF80B582B000AF786012
:102B200039604FF0010041F2C913C0F60503984720
:102B30007B68002B15D13B684FEA13439BB24FF0E3
:102B40000800194640F2C103C0F6050398473B68E8
:102B50009BB24FF00C00194640F2C103C0F60503CA
:102B600098477B68012B15D13B684FEA13439BB212
:102B70004FF01000194640F2C103C0F60503984714
:102B80003B689BB24FF01400194640F2C103C0F6F7
:102B9000050398477B68022B15D13B684FEA134326
:102BA0009BB24FF01800194640F2C103C0F605036E
:102BB00098473B689BB24FF01C00194640F2C10396
:102BC000C0F6050398477B68032B15D13B684FEA95
:102BD00013439BB24FF02000194640F2C103C0F6E8
:102BE000050398473B689BB24FF02400194640F21A
:102BF000C103C0F6050398474FF0000041F2C91326
:102C0000C0F60503984707F10807BD4680BD00BF21
:102C100090B583B000AF786039603B684FF0000238
:102C20001A607B68002B1DD13B681C684FF00800C0
:102C300040F2F903C0F60503984703464FEA034301
:102C400044EA03023B681A603B681C684FF00C00C2
:102C500040F2F903C0F605039847034644EA03022D
:102C60003B681A607B68012B1DD13B681C684FF0E4
:102C7000100040F2F903C0F60503984703464FEAF7
:102C8000034344EA03023B681A603B681C684FF048
:102C9000140040F2F903C0F605039847034644EADE
:102CA00003023B681A607B68022B1DD13B681C68DD
:102CB0004FF0180040F2F903C0F6050398470346A9
:102CC0004FEA034344EA03023B681A603B681C680E
:102CD0004FF01C0040F2F903C0F605039847034685
:102CE00044EA03023B681A607B68032B1DD13B68F2
:102CF0001C684FF0200040F2F903C0F60503984726
:102D000003464FEA034344EA03023B681A603B6808
:102D10001C684FF0240040F2F903C0F60503984701
:102D2000034644EA03023B681A6007F10C07BD46FC
:102D300090BD00BF80B500AF4DF2F043C2F200037A
:102D400003F51D5303F11C031B6803F00103002B63
:102D500005D04EF66D63C0F60303984700E000BF50
:102D600080BD00BF80B500AF4DF2F043C2F200035A
:102D700003F51D5303F11C031B6803F00103002B33
:102D800005D04EF68963C0F60303984700E000BF04
:102D900080BD00BF80B500AF4DF2F043C2F200032A
:102DA00003F51D5303F11C031B6803F00403002B00
:102DB00005D04EF63563C0F60303984700E000BF28
:102DC00080BD00BF80B500AF4DF2F043C2F20003FA
:102DD00003F51D5303F11C031B6803F00403002BD0
:102DE00005D04EF65163C0F60303984700E000BFDC
:102DF00080BD00BF80B500AF4DF2F043C2F20003CA
:102E000003F51D5303F11C031B6803F00203002BA1
:102E100005D04EF6A563C0F60303984700E000BF57
:102E200080BD00BF80B500AF4DF2F043C2F2000399
:102E300003F51D5303F11C031B6803F00203002B71
:102E400005D04EF6C163C0F60303984700E000BF0B
:102E500080BD00BF80B586B000AF40F63463C2F2DB
:102E600000034FF000021A604FF004004FF0010120
:102E700041F64D33C0F6050398474FF40063C4F2A2
:102E800000034FF000021A804FF40063C4F2000305
:102E90004FF000029A804FF40063C4F200034FF039
:102EA00000029A8140F68C53C2F200031A6845F280
:102EB000D523CEF60413A3FB02134FEAD3339BB200
:102EC00003F1FF33FB8240F267133B81FB8ABB8037
:102ED0004FF000037B814FF00003FB8007F10403F8
:102EE0004FF40060C4F20000194643F25123C0F6CB
:102EF000050398474FF40060C4F200004FF0010151
:102F00004FF0010243F68133C0F6050398474FF4B2
:102F10000060C4F200004FF0010143F6F123C0F657
:102F2000050398474FF01E033B744FF000037B747A
:102F30004FF00203BB744FF00103FB7407F1100361
:102F400018464BF67543C0F60403984707F1180777
:102F5000BD4680BD80B400AF40F63463C2F20003CA
:102F60001B6803F1010240F63463C2F200031A60E9
:102F70004FF40063C4F200034FF6FE721A82BD469E
:102F800080BC704780B400AF40F63463C2F20003E7
:102F90001B681846BD4680BC704700BF80B582B034
:102FA00000AF4FF01003FB714FF00103BB714FF402
:102FB0008043BB8007F104034FF4A050C4F201002A
:102FC000194640F6FD23C0F6050398474FF4A0507C
:102FD000C4F201004FF4804140F68953C0F6050366
:102FE00098474FF01003FB714FF00103BB714FF096
:102FF0000103BB8007F104034FF4A050C4F20100A9
:10300000194640F6FD23C0F6050398474FF4A0503B
:10301000C4F201004FF0010140F68953C0F60503E8
:1030200098474FF01003FB714FF00103BB714FF451
:103030000043BB8007F104034FF4A050C4F2010029
:10304000194640F6FD23C0F6050398474FF4A050FB
:10305000C4F201004FF4004140F68953C0F6050365
:1030600098474FF01003FB714FF00103BB714FF015
:103070001003BB8007F104034FF4A050C4F2010019
:10308000194640F6FD23C0F6050398474FF4A050BB
:10309000C4F201004FF0100140F68953C0F6050359
:1030A00098474FF01003FB714FF00103BB714FF4D1
:1030B0000073BB8007F104034FF44060C4F20100C9
:1030C000194640F6FD23C0F6050398474FF44060CB
:1030D000C4F201004FF4007140F68953C0F60503B5
:1030E000984707F10807BD4680BD00BF80B582B094
:1030F00000AF786039603B684FF0010202FA03F3D9
:103100009BB27868194640F68953C0F60503984784
:1031100007F10807BD4680BD80B582B000AF78607A
:1031200039603B684FF0010202FA03F39BB2786802
:10313000194640F6A553C0F60503984707F108075E
:10314000BD4680BD80B582B000AF786039603B6815
:103150004FF0010202FA03F39BB27868194640F679
:10316000D943C0F6050398470346184607F10807F8
:10317000BD4680BD80B500AF4FF020004FF001018B
:1031800041F6F923C0F60503984780BD80B586B0A7
:1031900000AF78600B46FB707B68002B02DB7B681E
:1031A000022B02DD4FF0FF3316E14FF4A053C4F2BF
:1031B00001037B617B68022B04D14FF44063C4F2AE
:1031C00001037B614FF000033B61FB784FEA03137F
:1031D000FB70FB7823F00F03FB7047F6B853C0F683
:1031E00005037A689B181B787869194643F219130E
:1031F000C0F6020398474FF00A0047F2B903C0F641
:10320000050398474FF00003FB734DE0FB785BB27A
:10321000002B0BDA4FF4A050C4F201004FF00E0166
:1032200043F2ED03C0F6020398470AE04FF4A050C2
:10323000C4F201004FF00E0143F21913C0F602036D
:1032400098474FF00A0047F2B903C0F605039847C4
:103250004FF4A050C4F201004FF0000143F2ED031F
:10326000C0F6020398474FF00A0047F2B903C0F6D0
:10327000050398474FF4A050C4F201004FF000013D
:1032800043F21913C0F6020398474FF00A0047F2C1
:10329000B903C0F605039847FB784FEA4303FB7078
:1032A000FB7B03F10103FB73FB7B072BAED94FF4D0
:1032B000A050C4F201004FF00E0143F21913C0F602
:1032C000020398474FF00003FB7327E04FF4A05030
:1032D000C4F201004FF0000143F2ED03C0F6020317
:1032E00098474FF00A0047F2B903C0F60503984724
:1032F0004FF4A050C4F201004FF0000143F2191343
:10330000C0F6020398474FF00A0047F2B903C0F62F
:1033100005039847FB7B03F10103FB73FB7B032B46
:10332000D4D94FF00A0047F2B903C0F60503984715
:103330004FF000033B614FF00003FB733AE03B6941
:103340004FEA43033B614FF4A050C4F201004FF039
:103350000D0143F24513C0F60203984703463A694C
:1033600013433B614FF4A050C4F201004FF0000141
:1033700043F2ED03C0F6020398474FF00A0047F20C
:10338000B903C0F6050398474FF4A050C4F20100FA
:103390004FF0000143F21913C0F6020398474FF0B3
:1033A0000A0047F2B903C0F605039847FB7B03F117
:1033B0000103FB73FB7B0B2BC1D947F6B853C0F657
:1033C00005037A689B181B787869194643F2ED0368
:1033D000C0F6020398473B69184607F11807BD4637
:1033E00080BD00BF80B582B000AF786078684FF0D4
:1033F0000C0143F28D13C0F60203984701464DF2CB
:10340000F043C2F200037A6802F6CC1243F82210AD
:1034100078684FF00B0143F28D13C0F60203984712
:1034200001464DF2F042C2F200027B6803F6CE1371
:103430004FEA8303D318596078684FF00D0143F2C7
:103440008D13C0F60203984701464DF2F043C2F2D5
:1034500000037A6802F6D21243F822104DF2F043CC
:10346000C2F200037A6802F6CC1253F82230022B23
:1034700002D940F60F1332E04DF2F042C2F20002E0
:103480007B6803F6CE134FEA8303D3185A6840F2E1
:10349000FD739A420ED94DF2F042C2F200027B68EF
:1034A00003F6CE134FEA8303D3185A6840F602039B
:1034B0009A4202D940F60F1311E04DF2F043C2F2E6
:1034C00000037A6802F6D21253F8222040F6FC7309
:1034D0009A4202D840F60F1301E04FF0000318465D
:1034E00007F10807BD4680BD80B485B000AF7860A5
:1034F0007B68FB607B68BB600FE0BB681A78FB6889
:103500001A70BB6803F10103BB60FB681B78202BBA
:1035100003D0FB6803F10103FB60BB681B78002B41
:10352000EBD1FB684FF000021A7007F11407BD469B
:1035300080BC704780B483B000AF78607B68002B9C
:1035400002DB7B68062B02DD4FF000037B6040F658
:103550002843C2F200037A6853F82230184607F174
:103560000C07BD4680BC704780B588B000AFF860DE
:10357000B9607A602F4BFB61FB68002B02D0BB68FF
:10358000002B01DC2B4B4FE04FF00003BB6122E02E
:10359000BB694FEA4303FA68D3181B887B617A69D9
:1035A0007B68D31A7B617B697A6902FB03F24AF27A
:1035B000C543C0F601031046984702464AF25D3300
:1035C000C0F60103F869114698470346FB61BB69E1
:1035D00003F10103BB61BA69BB689A42D8DB4AF2C6
:1035E000C543C0F60103B868984702464AF2D5635E
:1035F000C0F60103F869114698470346FB6149F696
:103600004543C0F60103F869984702460B46104649
:10361000194645F6C943C0F6010398474AF2B1235B
:10362000C0F6010398470346184607F12007BD4638
:1036300080BD00BF0000000090B583B000AF03461E
:10364000FB80FA8849F62143C0F6010310469847EB
:1036500002460B4649F6ED44C0F6010410461946F1
:103660004FF000024FF0804303F50023A0470246CD
:103670000B4649F64174C0F601041046194612A3E0
:10368000D3E90023A04702460B4649F64174C0F631
:103690000104104619464FF000024FF07F5303F526
:1036A0000013A04702460B46104619464AF2B123C2
:1036B000C0F6010398470346184607F10C07BD46BC
:1036C00090BD00BFAFF300800000000000FEAF40DF
:1036D00080B584B000AF78603960214BFB607B68B7
:1036E000002B02D03B68002B01DC1D4B33E04FF078
:1036F0000003BB601AE0BB684FEA43037A68D31843
:103700001B881A464AF2C543C0F601031046984783
:1037100002464AF25D33C0F60103F8681146984745
:103720000346FB60BB6803F10103BB60BA683B68FA
:103730009A42E0DB4AF2C543C0F601033868984775
:1037400002464AF2D563C0F60103F868114698476D
:103750000346FB60FB68184607F11007BD4680BDB5
:103760000000000080B586B000AF7860396007F1D6
:10377000080318464FF63D13C0F6030398473B7BFA
:103780004FF4616202FB03F17B7B1A4613464FEA5A
:1037900003139B1A4FEA8303CA18BB7BD3187B61C0
:1037A0007B697A6893FBF2F2796801FB02F29B1A5B
:1037B0003B617A683B69D21A3B68D318184607F117
:1037C0001807BD4680BD00BF2DE9F04FA7B00EAF72
:1037D000F86007F1280318464FF63D13C0F60303BF
:1037E000984707F1280318464FF67533C0F60303D0
:1037F00098470346BB644FF00003FB646FE007F19A
:1038000024034FF00000194642F26D53C0F6020344
:1038100098477B6AFA6DD318FB6507F124034FF0D4
:103820000100194642F26D53C0F6020398477B6AC5
:10383000BA6DD318BB6507F124034FF00200194697
:1038400042F26D53C0F6020398477B6A7A6DD31833
:103850007B6507F124034FF00300194642F26D53D4
:10386000C0F6020398477B6A3A6DD3183B65B96D81
:103870007A6D3B6D084611461A4643F62523C0F67D
:10388000020398470346FB65796DFA6D3B6D084668
:1038900011461A4643F62523C0F60203984703460D
:1038A000BB65B96D3A6DFB6D084611461A4643F685
:1038B0002523C0F60203984703467B65F96D7A6DB0
:1038C000BB6D084611461A4643F62523C0F602038F
:1038D000984703463B65FB6C03F10103FB64FB6CFB
:1038E000092B8CDD3B6D4FEA0342FB6D13437B6478
:1038F0007B6D4FEA0342BB6D13433B64B86C796C3C
:103900003A6C43F62523C0F602039847F863786CB7
:10391000B96C3A6C43F62523C0F602039847B863A6
:10392000386C396CBA6C43F62523C0F6020398470D
:103930007863F86BB96B7A6B43F62523C0F6020304
:1039400098473863386B46F2A103C0F601039847E5
:103950004FF00003FB6416E046F2B903C0F6010322
:10396000984702464FEAE2734FEA1363D218D2B285
:10397000D31ADAB207F11401FB6CCB181A70FB6C86
:1039800003F10103FB64FB6C0F2BE5DD3B7D1E4661
:103990007B7D1D46BB7D1946FB7D1C463B7EBB6087
:1039A0007B7E7B60BB7E3B60FB7E9B463B7F9A467B
:1039B0007B7F9946BB7F9846FB7F9C4697F82030DB
:1039C0009E4697F82130184697F822301A4697F805
:1039D000233000910194B9680291796803913968A4
:1039E0000491CDF814B0CDF818A0CDF81C90CDF806
:1039F0002080CDF824C0CDF828E00B900C920D93D8
:103A0000F86847F2D871C0F6050132462B4641F2FC
:103A1000A114C0F60404A04707F16407BD46BDE841
:103A2000F08F00BF80B485B000AFF860B9607A60F5
:103A3000FA68BB68D31AFB60FA687B68D31AFB602C
:103A40007B684FEA5333FA685340FB60BA687B687F
:103A5000D31ABB60BA68FB68D31ABB60FB684FEA35
:103A60000323BA685340BB607A68FB68D31A7B6053
:103A70007A68BB68D31A7B60BB684FEA53337A68B5
:103A800053407B60FA68BB68D31AFB60FA687B68B6
:103A9000D31AFB607B684FEA1333FA685340FB602C
:103AA000BA687B68D31ABB60BA68FB68D31ABB607C
:103AB000FB684FEA0343BA685340BB607A68FB680F
:103AC000D31A7B607A68BB68D31A7B60BB684FEA05
:103AD00053137A6853407B60FA68BB68D31AFB6063
:103AE000FA687B68D31AFB607B684FEAD303FA68F5
:103AF0005340FB60BA687B68D31ABB60BA68FB6846
:103B0000D31ABB60FB684FEA8323BA685340BB609B
:103B10007A68FB68D31A7B607A68BB68D31A7B60CB
:103B2000BB684FEAD3337A6853407B607B681846A2
:103B300007F11407BD4680BC704700BF80B487B052
:103B400000AF78600B46FB707B681B684FEA13235D
:103B5000FB757B681B68BB757B6803F104031B68FE
:103B60004FEA13237B757B6803F104031B683B75E5
:103B70002F4BFB6007F10C033B61FB78012B12D14B
:103B80003B6903F103033A7D1A703B6903F10203B9
:103B90007A7D1A703B6903F10103BA7D1A703B69A3
:103BA000FA7D1A703DE0FB78022B12D13B6903F1DC
:103BB0000303BA7D1A703B6903F10203FA7D1A70A0
:103BC0003B6903F101033A7D1A703B697A7D1A70F3
:103BD00027E0FB78032B12D13B6903F103037A7DC5
:103BE0001A703B6903F102033A7D1A703B6903F1D5
:103BF0000103FA7D1A703B69BA7D1A7011E03B69C6
:103C000003F10303FA7D1A703B6903F10203BA7DE5
:103C10001A703B6903F101037A7D1A703B693A7DA2
:103C20001A70FB68184607F11C07BD4680BC704738
:103C30000000000080B487B000AF78600B46FB70D6
:103C40007B681B684FEA1323FB757B681B68BB7599
:103C50007B6803F104031B684FEA13237B757B68C1
:103C600003F104031B683B754FF00003FB6007F191
:103C70000C033B61FB78012B12D13B6903F1030379
:103C80003A7D1A703B6903F102037A7D1A703B6931
:103C900003F10103BA7D1A703B69FA7D1A703DE0A9
:103CA000FB78022B12D13B6903F10303BA7D1A7032
:103CB0003B6903F10203FA7D1A703B6903F10103CA
:103CC0003A7D1A703B697A7D1A7027E0FB78032BE6
:103CD00012D13B6903F103037A7D1A703B6903F14A
:103CE00002033A7D1A703B6903F10103FA7D1A70F1
:103CF0003B69BA7D1A7011E03B6903F10303FA7D59
:103D00001A703B6903F10203BA7D1A703B6903F133
:103D100001037A7D1A703B693A7D1A70FB68184678
:103D200007F11C07BD4680BC704700BF80B487B058
:103D300000AF78600B46FB707B681B684FEA13236B
:103D4000FB757B681B68BB757B6803F104031B680C
:103D50004FEA13237B757B6803F104031B683B75F3
:103D60004FF00003FB6007F10C033B61FB78012B74
:103D700012D13B6903F103033A7D1A703B6903F1E9
:103D800002037A7D1A703B6903F10103BA7D1A7050
:103D90003B69FA7D1A703DE0FB78022B12D13B693A
:103DA00003F10303BA7D1A703B6903F10203FA7D44
:103DB0001A703B6903F101033A7D1A703B697A7D01
:103DC0001A7027E0FB78032B12D13B6903F1030340
:103DD0007A7D1A703B6903F102033A7D1A703B69E0
:103DE00003F10103FA7D1A703B69BA7D1A7011E084
:103DF0003B6903F10303FA7D1A703B6903F1020387
:103E0000BA7D1A703B6903F101037A7D1A703B6930
:103E10003A7D1A70FB68184607F11C07BD4680BC46
:103E2000704700BF80B5ACB000AFF860B9607A6091
:103E30003B604FF00003C7F8AC3039E0D7F8AC3046
:103E4000FA68D3181B78C7F89C3040F20C33C2F2E2
:103E500000031A68D7F89C3003F10103D3181B78CC
:103E600003F00303012B04D1D7F89C3003F12003A6
:103E700001E0D7F89C30DAB207F11401D7F8AC3082
:103E8000CB181A7007F11402D7F8AC30D3181B788E
:103E90005C2B07D107F11402D7F8AC30D3184FF0E0
:103EA0002F021A70D7F8AC3003F10103C7F8AC3019
:103EB000D7F8AC30FA68D3181B78002B03D0D7F8AA
:103EC000AC307F2BBADDD7F8AC307F2B05DDD7F8CF
:103ED000AC3003F1FF33C7F8AC3007F11402D7F868
:103EE000AC30D3184FF000021A7007F114031846D3
:103EF00046F20933C0F6010398470346C7F89830E5
:103F00004FF00003C7F8A830BB684FF000021A70EA
:103F100007F11403184647F62001C0F6050146F2E2
:103F2000AD63C0F601039847C7F89400D7F8943002
:103F3000002B0CD04FF00703C7F8A830BA6847F63B
:103F40002003C0F6050303CB1060516041E007F188
:103F50001403184647F62801C0F6050146F2AD6382
:103F6000C0F601039847C7F89400D7F89430002BA7
:103F70000ED04FF00803C7F8A830BA6847F62803F8
:103F8000C0F6050303CB106051601B78137220E06C
:103F900007F11403184647F63401C0F6050146F24E
:103FA000AD63C0F601039847C7F89400D7F8943082
:103FB000002B0ED04FF00603C7F8A830BB6847F6B9
:103FC0003402C0F6050210681860918892799980D1
:103FD0009A71D7F8A830C7F8A43005E0D7F8A43014
:103FE00003F10103C7F8A43007F11402D7F8A43095
:103FF000D3181B782F2B0BD007F11402D7F8A4305D
:10400000D3181B78002B03D0D7F8A4307F2BE5DD25
:10401000D7F8A420D7F8A830D31A03F10103C7F8C2
:10402000A030D7F8A030802B03DD4FF07F03C7F816
:10403000A030D7F8A83007F11402D218D7F8A03072
:10404000786811461A4646F26933C0F6010398476C
:10405000D7F8A03003F1FF337A68D3184FF000028D
:104060001A70D7F89820D7F8A430D31A03F10103B7
:10407000C7F8A030D7F8A030802B03DD4FF07F03C6
:10408000C7F8A030D7F8A43007F11402D218D7F837
:10409000A030386811461A4646F26933C0F601036B
:1040A0009847D7F8A03003F1FF333A68D3184FF0A0
:1040B00000021A704FF00003184607F1B007BD4622
:1040C00080BD00BF80B594B000AF786039603B68B8
:1040D0004FF000021A607A6807F10C031046194687
:1040E00048F2BD33C0F60203984738643B6C002B9E
:1040F00001D03B6CBCE007F10C03184647F6D563D2
:10410000C0F6020398474FF00003BB644FF0000372
:10411000FB634FF000037B644FF00003FB649AE005
:10412000FB6C03F00103002B6CD1FB6C4FEA4303E3
:1041300007F15002D31833F8403C1BB2BB63BB6B92
:10414000002B00F08D80BB6B18464BF68D73C0F6CC
:1041500001039847F863FB6B002B02D140F28E33CA
:1041600086E0FB6B93F87531022B02D040F2853369
:104170007EE0BB6C002B04D1FB6BD3F862317B6417
:1041800065E0BB6C012B06D1FB6BD3F862317A6C16
:1041900013407B645BE0BB6C022B06D1FB6BD3F856
:1041A00062317A6C13437B6451E0BB6C032B07D103
:1041B000FB6BD3F862217B6C02FB03F37B6446E06C
:1041C000BB6C042B07D1FB6BD3F862317A6C92FB8A
:1041D000F3F37B643BE0BB6C052B06D1FB6BD3F8A0
:1041E00062317A6CD3187B6431E0BB6C062B06D14C
:1041F000FB6BD3F862317A6CD31A7B6427E040F210
:10420000893335E0FB6C4FEA430307F15002D318C2
:1042100033F8403C1BB2BB64BB6C012B14D0BB6CAD
:10422000022B11D0BB6C032B0ED0BB6C042B0BD01C
:10423000BB6C052B08D0BB6C062B05D0BB6C002BD0
:1042400002D040F2893313E0BB6C002B0AD0FB6C28
:1042500003F10103FB64FB6C122B7FF761AF02E0FB
:1042600000BF00E000BF7A6C3B681A604FF00003AB
:10427000184607F15007BD4680BD00BF90B595B008
:1042800000AF786039603B68904A1A607A6807F13D
:104290000C031046194648F2BD33C0F60203984796
:1042A00038643B6C002B01D03B6C0AE14FF00003FB
:1042B000BB644FF00003FB63844B7B644FF000034F
:1042C000FB64F1E0FB6C03F00103002B40F0C380C2
:1042D000FB6C4FEA430307F15002D31833F8403C1C
:1042E0001BB2BB63BB6B002B00F0E380BB6B1846BB
:1042F0004BF68D73C0F601039847F863FB6B002BF8
:1043000002D140F28E33DCE0FB6B93F87531022B67
:1043100002D040F28533D4E0BB6C002B04D1FB6BA0
:10432000D3F866317B64BBE0BB6C012B1DD14AF630
:10433000F903C0F60103786C98470446FB6BD3F889
:10434000662113461A464AF6F903C0F601031046E1
:104350009847034604EA03024AF2C543C0F6010344
:104360001046984703467B649AE0BB6C022B1DD134
:104370004AF6F903C0F60103786C98470446FB6BD4
:10438000D3F8662113461A464AF6F903C0F601032C
:1043900010469847034644EA03024AF2C543C0F672
:1043A00001031046984703467B6479E0BB6C032BFE
:1043B0000ED1FB6BD3F8662113461A464AF26D53B1
:1043C000C0F60103786C1146984703467B6467E0AA
:1043D000BB6C042B0ED1FB6BD3F8662113461A4637
:1043E0004AF2D563C0F60103786C1146984703463C
:1043F0007B6455E0BB6C052B13D1FB6BD3F86221BA
:104400004AF2C543C0F601031046984702464AF2F5
:104410005D33C0F60103786C1146984703467B6410
:104420003EE0BB6C062B13D1FB6BD3F862214AF242
:10443000C543C0F601031046984702464AF2593375
:10444000C0F60103786C1146984703467B6427E069
:1044500040F2893335E0FB6C4FEA430307F1500229
:10446000D31833F8403C1BB2BB64BB6C012B14D097
:10447000BB6C022B11D0BB6C032B0ED0BB6C042B7E
:104480000BD0BB6C052B08D0BB6C062B05D0BB6CCE
:10449000002B02D040F2893313E0BB6C002B0AD012
:1044A000FB6C03F10103FB64FB6C122B7FF70AAF7B
:1044B00002E000BF00E000BF3B687A6C1A604FF07A
:1044C0000003184607F15407BD4690BD00000000E8
:1044D00080B584B000AF78607B68002B02D140F2D9
:1044E000853369E07B6893F87830022B08D17868CF
:1044F00045F2E103C0F6020398474FF000035BE08A
:104500007B6893F87830032B08D1786844F6B96358
:10451000C0F6020398474FF000034DE04FF0000350
:10452000FB60786844F2C553C0F60203984703461F
:10453000002B03D04FF00503FB6032E0786844F2B3
:10454000A163C0F6020398470346002B03D04FF047
:104550000403FB6025E0786844F64503C0F60203D7
:1045600098470346002B03D04FF00303FB6018E08D
:10457000786844F6D923C0F6020398470346002B17
:1045800003D04FF00203FB600BE0786844F67D43F4
:10459000C0F6020398470346002B02D04FF00103F8
:1045A000FB60FB68DBB27868194644F65953C0F6E5
:1045B000020398474FF00003184607F11007BD4665
:1045C00080BD00BF90B587B000AF78607B6893F87E
:1045D0009130002B02D14FF000035BE07B68D3F8F1
:1045E0007D2013461A464AF6F903C0F60103104629
:1045F000984703467B617B68D3F866313B617B68F3
:10460000D3F8814023461C464AF2C543C0F6010355
:104610007869984702464AF25933C0F601032046AA
:10462000114698470346FB607B68D3F881402346D8
:104630001C464AF2C543C0F6010378699847024612
:104640004AF25D33C0F601032046114698470346FF
:10465000BB607B6893F87331052B0CD14AF6BD0320
:10466000C0F601033869B96898470346002B0FD09C
:104670004FF001030EE04AF6A903C0F601033869C2
:10468000F96898470346002B02D04FF0010301E080
:104690004FF00003184607F11C07BD4690BD00BF50
:1046A00090B589B000AF78607B6893F89230002BAA
:1046B00002D14FF00003BEE07B68D3F87D201346A3
:1046C0001A464AF6F903C0F6010310469847034616
:1046D0007B617B68D3F866313B61594BFB617B683A
:1046E000D3F8854023461C464AF2C543C0F6010371
:1046F0007869984702464AF25D33C0F601032046C6
:10470000114698470346FB604D4BBB617B68D3F86D
:10471000854023461C464AF2C543C0F6010378692A
:10472000984702464AF25933C0F601032046114623
:1047300098470346BB607B6893F89130002B29D0E3
:104740007B68D3F8814023461C464AF2C543C0F635
:1047500001037869984702464AF25D33C0F60103C7
:104760002046114698470346FB617B68D3F8814099
:1047700023461C464AF2C543C0F6010378699847B0
:1047800002464AF25933C0F60103204611469847C3
:104790000346BB617B6893F87331042B16D14AF64C
:1047A000D103C0F601033869B96998470346002B65
:1047B0003FD04AF6BD03C0F601033869F96898474F
:1047C0000346002B35D04FF0010334E07B6893F8AB
:1047D0007331052B16D14AF6E503C0F6010338699B
:1047E000F96998470346002B23D04AF6BD03C0F66B
:1047F00001033869F96898470346002B19D04FF038
:10480000010318E04AF6D103C0F601033869B9691B
:1048100098470346002B0CD04AF6A903C0F60103C3
:104820003869B96898470346002B02D04FF001035E
:1048300001E04FF00003184607F12407BD4690BD84
:10484000FFFF7FFF90B589B000AF78607B6893F879
:104850009330002B02D14FF0000333E17B68D3F893
:104860007D2013461A464AF6F903C0F601031046A6
:1048700098470346FB607B68D3F86631BB60944B76
:10488000FB61944BBB61924B7B61924B3B617B68BC
:1048900093F89230002B2AD07B68D3F885402346CA
:1048A0001C464AF2C543C0F60103F8689847024621
:1048B0004AF25D33C0F6010320461146984703468D
:1048C000FB617B68D3F8854023461C464AF2C5430A
:1048D000C0F60103F868984702464AF25933C0F619
:1048E000010320461146984703467B612EE07B6812
:1048F00093F89130002B29D07B68D3F88140234670
:104900001C464AF2C543C0F60103F86898470246C0
:104910004AF25D33C0F6010320461146984703462C
:10492000FB617B68D3F8814023461C464AF2C543AD
:10493000C0F60103F868984702464AF25933C0F6B8
:10494000010320461146984703467B617B6893F834
:104950009430002B2AD07B68D3F8894023461C462C
:104960004AF2C543C0F60103F868984702464AF286
:104970005D33C0F601032046114698470346BB61EC
:104980007B68D3F8894023461C464AF2C543C0F6EB
:104990000103F868984702464AF25933C0F601030A
:1049A00020461146984703463B612EE07B6893F80A
:1049B0009530002B29D07B68D3F88D4023461C46C8
:1049C0004AF2C543C0F60103F868984702464AF226
:1049D0005D33C0F601032046114698470346BB618C
:1049E0007B68D3F88D4023461C464AF2C543C0F687
:1049F0000103F868984702464AF25933C0F60103AA
:104A000020461146984703463B617B6893F8733113
:104A1000032B04D07B6893F87331002B17D14AF62F
:104A2000D103C0F60103B868796998470346002BA3
:104A300046D04AF6BD03C0F60103B868B969984785
:104A40000346002B02D04FF001033BE038E07B68C7
:104A500093F87331042B04D07B6893F87331052BE2
:104A600017D14AF6E503C0F60103B868F96998471B
:104A70000346002B24D04AF6BD03C0F60103B868F4
:104A8000B96998470346002B02D04FF0010319E0A3
:104A900016E04AF6D103C0F60103B8687969984771
:104AA0000346002B0CD04AF6A903C0F60103B868F0
:104AB000396998470346002B02D04FF0010301E00B
:104AC0004FF00003184607F12407BD4690BD00BF14
:104AD000FFFF7FFFFFFF7F7F90B589B000AF786059
:104AE0007B6893F89430002B02D14FF00003BEE0B6
:104AF0007B68D3F87D2013461A464AF6F903C0F6C0
:104B000001031046984703467B617B68D3F8663102
:104B10003B617B68D3F8894023461C464AF2C54373
:104B2000C0F601037869984702464AF25D33C0F641
:104B300001032046114698470346FB604E4BFB613C
:104B40007B68D3F8894023461C464AF2C543C0F629
:104B500001037869984702464AF25933C0F60103C7
:104B60002046114698470346BB60434BBB617B68B8
:104B700093F89530002B29D07B68D3F88D402346DD
:104B80001C464AF2C543C0F60103786998470246BD
:104B90004AF25D33C0F601032046114698470346AA
:104BA000FB617B68D3F88D4023461C464AF2C5431F
:104BB000C0F601037869984702464AF25933C0F6B5
:104BC00001032046114698470346BB617B6893F872
:104BD0007331022B16D14AF6D103C0F601033869AE
:104BE000B96898470346002B3FD04AF6BD03C0F68C
:104BF00001033869F96998470346002B35D04FF017
:104C0000010334E07B6893F87331012B16D14AF627
:104C1000D103C0F601033869B96898470346002BF1
:104C200023D04AF6A903C0F601033869B969984749
:104C30000346002B19D04FF0010318E04AF6E503B4
:104C4000C0F601033869F96898470346002B0CD079
:104C50004AF6BD03C0F601033869F969984703466F
:104C6000002B02D04FF0010301E04FF00003184683
:104C700007F12407BD4690BDFFFF7F7F90B587B049
:104C800000AF78607B6893F89530002B02D14FF02D
:104C900000035BE07B68D3F87D2013461A464AF692
:104CA000F903C0F601031046984703467B617B6811
:104CB000D3F866313B617B68D3F88D4023461C46B0
:104CC0004AF2C543C0F601037869984702464AF2A2
:104CD0005933C0F601032046114698470346FB604E
:104CE0007B68D3F88D4023461C464AF2C543C0F684
:104CF00001037869984702464AF25D33C0F6010322
:104D00002046114698470346BB607B6893F8733191
:104D1000012B0CD14AF6D103C0F601033869F968BA
:104D200098470346002B0FD04FF001030EE04AF6E0
:104D3000E503C0F601033869B96898470346002BBC
:104D400002D04FF0010301E04FF00003184607F1D5
:104D50001C07BD4690BD00BF90B587B000AF78601E
:104D60000B46FB707B68002B02D140F285339DE03F
:104D7000FB78002B0AD17B68FA7883F872217B6874
:104D8000FA7883F873214FF000038FE07B6893F883
:104D90007231FA789A420CD07B6803F25B131846A2
:104DA0004FF63D13C0F6030398477B68FA7883F803
:104DB00072217B6893F87331FA789A4274D007F1C4
:104DC000080318464FF63D13C0F6030398477B6867
:104DD00003F25B1307F10802104619464FF63543FC
:104DE000C0F60303984738617B68D3F87930002B0D
:104DF00005D03A697B68D3F879309A4254D37B68FE
:104E0000FA7883F873217B68D3F862214AF2C543AC
:104E1000C0F601031046984703467B617B689B7888
:104E2000062B08D17B6893F86430042B03D17B6890
:104E3000D3F862317B617B689B78062B14D17B6849
:104E400093F86430032B04D07B6893F86430012B13
:104E50000AD17B68D3F862214AF2BD43C0F6010350
:104E60001046984703467B617B689B78082B0AD1E4
:104E70007B68D3F862214AF2BD43C0F601031046B5
:104E8000984703467B617B68B3F900309BB219B247
:104E90007B68D3F86631FA78084611467A694EF293
:104EA000DD44C0F60104A0474FF00003184607F1A7
:104EB0001C07BD4690BD00BF90B589B000AF7860BB
:104EC0007B68002B02D140F2853304E17B6893F8C4
:104ED0007431002B1BD07B68D3F86A110B4619463E
:104EE0007B68D3F8662113461A464AF69503C0F646
:104EF00001030846114698470346002B07D07B68FC
:104F00004FF0000283F872214FF00003E3E04FF00E
:104F10000003FB614FF00003BB6125E07B68D3F821
:104F2000664123461C467A68BB6903F126034FEAB3
:104F30008303D318D3F802204AF2C543C0F6010315
:104F40001046984702464AF69503C0F601032046EC
:104F5000114698470346002B02D04FF00103FB6136
:104F6000BB6903F10103BB617B68D3F89620BB6981
:104F70009A42D3DCFB69002B12D17B684FF0000210
:104F800083F872217B684FF0000283F873217B68FD
:104F9000D3F866317A68C2F86A314FF000039AE0BC
:104FA0007B6893F87231072B0DD07B6803F25B139B
:104FB00018464FF63D13C0F6030398477B684FF041
:104FC000070283F8722107F1080318464FF63D13D4
:104FD000C0F6030398477B6803F25B1307F10802EE
:104FE000104619464FF63543C0F60303984738611B
:104FF0007B68D3F87930002B05D03A697B68D3F809
:1050000079309A4265D37B68D3F862214AF2C5436E
:10501000C0F601031046984703467B617B689B7886
:10502000062B08D17B6893F86430042B03D17B688E
:10503000D3F862317B617B689B78062B14D17B6847
:1050400093F86430032B04D07B6893F86430012B11
:105050000AD17B68D3F862214AF2BD43C0F601034E
:105060001046984703467B617B689B78082B0AD1E2
:105070007B68D3F862214AF2BD43C0F601031046B3
:10508000984703467B617B68B3F900309BB21AB244
:105090007B68D3F8663110464FF007017A694EF20B
:1050A000DD44C0F60104A0477B684FF0010283F89D
:1050B00074217B68D3F866317A68C2F86A317B68FC
:1050C0004FF0000283F872217B684FF0070283F8EB
:1050D00073214FF00003184607F12407BD4690BD29
:1050E00090B58BB000AF78607B68002B02D140F2A6
:1050F000853388E17B6893F83E31002B40F0DB80FC
:105100007B6893F87431002B0DD17B68D3F866313E
:105110007A68C2F86A317B684FF0010283F8742123
:105120004FF000036FE17B68D3F86A110B46194614
:105130007B68D3F8662113461A464AF25933C0F603
:105140000103084611469847034623F00043BB611C
:1051500049F64543C0F60103B869984702460B4635
:105160004AF2D114C0F601041046194698A3D3E9B7
:105170000023A0470346002B07D07B684FF00002B6
:1051800083F872214FF000033DE17B6893F87231A0
:10519000062B0DD07B6803F25B1318464FF63D13C8
:1051A000C0F6030398477B684FF0060283F872212C
:1051B00007F1080318464FF63D13C0F6030398475E
:1051C0007B6803F25B1307F10802104619464FF69D
:1051D0003543C0F60303984778617B68D3F879308C
:1051E000002B06D07A697B68D3F879309A42C0F0F8
:1051F00008817B68D3F862214AF2C543C0F60103F7
:105200001046984703467B627B689B78062B08D143
:105210007B6893F86430042B03D17B68D3F8623148
:105220007B627B689B78062B14D17B6893F8643093
:10523000032B04D07B6893F86430012B0AD17B6880
:10524000D3F862214AF2BD43C0F6010310469847E5
:1052500003467B627B689B78082B0AD17B68D3F876
:1052600062214AF2BD43C0F6010310469847034647
:105270007B627B68B3F900309BB21AB27B68D3F8CB
:10528000663110464FF006017A6A4EF2DD44C0F6F0
:105290000104A0477B68D3F866317A68C2F86A31A6
:1052A0007B684FF0000283F872217B684FF00602A2
:1052B00083F87321A5E07B68D3F862313B627B6899
:1052C0009B78062B11D17B6893F86430042B0CD1AA
:1052D0007B68D3F8622113461A464AF64513C0F696
:1052E00001031046984703463B627B689B78062B78
:1052F0000DD17B6893F86430032B04D07B6893F85E
:105300006430012B03D17B68D3F862313B627B6848
:105310009B78082B03D17B68D3F862313B627B68B2
:1053200093F87431002B0BD17B683A6AC3F86E2175
:105330007B684FF0010283F874214FF0000362E0B4
:105340007B68D3F86E213B6A9A4207D17B684FF0A5
:10535000000283F872214FF0000354E04FF0000385
:10536000FB6142E04FF00102FB6902FA03F33B618B
:105370007B68D3F83F213B691A403B699A422FD1A1
:105380007B68D3F86E213B6A5A403B691340002B7F
:1053900027D07B68B3F900309BB21CB24AF2C543F8
:1053A000C0F60103F86998470246396A3B6919401B
:1053B0003B69994201D1084B00E0084B20464FF071
:1053C00006014EF2DD44C0F60104A04709E000BF2B
:1053D0002D431CEBE2361A3F0000803F0000000026
:1053E00000BFFB6903F10103FB61FB691F2BB9DD02
:1053F0007B683A6AC3F86E217B684FF0000283F83D
:1054000072214FF00003184607F12C07BD4690BDEE
:1054100090B591B000AF78607B68002B02D140F26C
:1054200085331CE2DFF84034FB637B689B780B2BF1
:1054300012D17B68D3F84D204BF22B039A420BD943
:105440007B68D3F84D204BF28F039A4204D87B68D7
:10545000D3F86231FB6343E07B689B780D2B04D16A
:105460007B68D3F86231FB633AE07B689B78062B5C
:105470002BD17B6893F86430032B04D07B6893F8BE
:105480006430012B0BD17B68D3F862214AF2BD4313
:10549000C0F60103104698470346FB6320E07B6893
:1054A00093F86430042B04D17B68D3F86231FB633A
:1054B00016E07B68D3F862214AF2C543C0F60103C7
:1054C000104698470346FB630AE07B68D3F86221E5
:1054D0004AF2C543C0F60103104698470346FB63F2
:1054E0007B68FA6BC3F866217B6893F86730002B02
:1054F00054D0FB6BFB617B681B6FBB617B685B6F90
:105500007B617B689A6E4AF2BD43C0F60103104688
:10551000984703463B617B68DA6E4AF2BD43C0F6AA
:105520000103104698470346FB604AF25933C0F620
:1055300001037869B969984703461C464AF2593312
:10554000C0F60103F8693969984703461A464AF2DA
:105550006D53C0F6010320461146984703461C468A
:105560004AF25933C0F60103F8683969984703468F
:105570001A464AF2D563C0F6010320461146984701
:1055800003461A464AF25D33C0F601031046B96974
:10559000984703461A467B68C3F866217B6893F8F0
:1055A0005530032B72D1FB6BBB637B6893F867307C
:1055B000002B03D07B68D3F86631BB634AF26D538E
:1055C000C0F60103B86BB96B984703461A464AF216
:1055D0006D53C0F601031046B96B98470346194650
:1055E0007B68D3F8562013461A464AF26D53C0F62C
:1055F000010308461146984703461C464AF26D537C
:10560000C0F60103B86BB96B9847034619467B682F
:10561000D3F85A2013461A464AF26D53C0F60103D6
:1056200008461146984703461A464AF25D33C0F6CB
:10563000010320461146984703461C467B68D3F871
:105640004C2113461A464AF26D53C0F60103104628
:10565000B96B984703461A464AF25D33C0F6010318
:10566000204611469847034619467B68D3F85021D7
:1056700013461A464AF25D33C0F601030846114646
:10568000984703461A467B68C3F866217B6893F8FF
:105690005530012B29D1FB6B7B637B6893F8673016
:1056A000002B03D07B68D3F866317B637B68D3F82B
:1056B000562013461A464AF26D53C0F601031046AF
:1056C000796B9847034619467B68D3F85A201346EE
:1056D0001A464AF25D33C0F6010308461146984760
:1056E00003461A467B68C3F866217B6893F85530F9
:1056F000022B40F0B280FB6B3B637B6893F8673012
:10570000002B03D07B68D3F866313B637B68D3F80A
:105710005A2013461A464AF69503C0F6010310466E
:10572000514998470346002B05D07B68D3F8563083
:105730007A68C2F866317B68D3F85A2013461A4655
:105740004AF6E503C0F60103104647499847034669
:10575000002B39D0454BBB624FF00003FB620CE0DD
:105760004AF26D53C0F60103B86A396B9847034695
:10577000BB62FB6A03F10103FB624AF2C543C0F658
:105780000103F86A984701467B68D3F85A2013460C
:105790001A464AF6A903C0F601030846114698477F
:1057A0000346002BDCD17B68D3F8562013461A46FB
:1057B0004AF26D53C0F601031046B96A9847034692
:1057C0001A467B68C3F866217B68D3F85A201346D3
:1057D0001A464AF6A903C0F6010310462249984723
:1057E0000346002B39D0214B3B624FF000037B6214
:1057F0000CE04AF26D53C0F60103386A396B9847E2
:1058000003463B627B6A03F101037B624AF2C543B4
:10581000C0F60103786A984701467B68D3F85A209E
:1058200013461A464AF6A903C0F601030846114674
:1058300098470346002BDCD17B68D3F856201346EB
:105840001A464AF2D563C0F601031046396A9847F2
:1058500003461A467B68C3F866214FF000031846DA
:1058600007F14407BD4690BD000000000000803FE6
:1058700080B483B000AF78607B684FF0000283F89B
:1058800034207B684FF0000283F835207B684FF0AE
:10589000000283F836204FF00003184607F10C078A
:1058A000BD4680BC704700BF80B58CB000AFF860CB
:1058B0007B600B46FB721346BB72FB6893F8343077
:1058C0001A46F96813464FEA43039B184FEA8303CD
:1058D0009B18CB1803F10803FA7A1A70FB6893F847
:1058E00034301A46F96813464FEA43039B184FEACF
:1058F00083039B18CB1803F10703BA7A1A70FB686D
:1059000093F834301A46F96813464FEA43039B185C
:105910004FEA83039B18CB1803F108037A68C3F896
:105920000120FB6893F834301A4613464FEA4303CC
:105930009B184FEA83039B18FA68D31818464FF652
:105940003D13C0F6030398474FF00103FB76FB6855
:1059500093F834301A4613464FEA43039B184FEA34
:1059600083039B18FA68D21807F1140310681860B3
:105970009188927999809A71FB7AC7F81E307B687A
:10598000C7F82230BB7A9BB2FB8407F1100318469C
:1059900040F2F923C0F603039847F862F86845F629
:1059A0004933C0F602039847F862FB6A002B01D026
:1059B000FB6A35E0FB6893F8343003F10103DAB297
:1059C000FB6883F83420FB6893F83430032B04D948
:1059D000FB684FF0000283F83420FB6893F8342012
:1059E000FB6893F835309A4212D1FB6893F8353052
:1059F00003F10103DAB2FB6883F83520FB6893F802
:105A00003530032B04D9FB684FF0000283F83520B2
:105A1000F86845F6A933C0F6020398474FF0000333
:105A2000184607F13007BD4680BD00BF80B584B081
:105A300000AF786039604FF00003FB607B6893F83B
:105A400035207B6893F834309A4203D140F2863394
:105A5000FB6028E07B6893F835301A4613464FEA1E
:105A600043039B184FEA83039B187A68D31838685E
:105A700019464FF00D0245F67573C0F601039847BD
:105A80007B6893F8353003F10103DAB27B6883F861
:105A900035207B6893F83530032B04D97B684FF0B1
:105AA000000283F83520FB68184607F11007BD4651
:105AB00080BD00BF80B483B000AF78607B684FF0DA
:105AC000000283F834207B684FF0000283F8352011
:105AD00007F10C07BD4680BC704700BF80B485B09D
:105AE00000AF78604FF00003FB607B6893F83420D0
:105AF0007B6893F835309A420AD27B6893F8353048
:105B0000C3F104027B6893F83430D318FB6014E0CF
:105B10007B6893F834207B6893F835309A4209D932
:105B20007B6893F834301A467B6893F83530D31A83
:105B3000FB6002E04FF00003FB60FB68184607F1D2
:105B40001407BD4680BC704780B584B000AF786054
:105B50004FF00003FB600AE04FF00A0047F20D33FC
:105B6000C0F604039847FB6803F10103FB607B6800
:105B700093F83630012B02D1FB68312BECDD7B68CA
:105B800093F83630012B02D140F2873306E07B6870
:105B90004FF0010283F836204FF00003184607F15A
:105BA0001007BD4680BD00BF80B483B000AF7860F1
:105BB0007B684FF0000283F8362007F10C07BD46E2
:105BC00080BC704780B582B000AF78607B684FF0D2
:105BD0000002C3F8F0207B684FF00002C3F8F42005
:105BE0007B6818464FF000014FF0F00246F20903BF
:105BF000C0F6010398474FF00003184607F1080765
